:020000040800F2
:100000000002002029050008C5040008810400083A
:10001000D5040008E5040008F5040008000000000D
:10002000000000000000000000000000450400087F
:100030000505000800000000290400081505000857
:100040008901000889010008890100088901000868
:100050008901000889010008CD160008CD160008A6
:10006000CD160008CD160008CD160008890100083D
:100070008901000889010008890100088901000838
:100080008901000889010008890100088901000828
:10009000890100088901000889010008CD160008BF
:1000A0008901000889010008890100088901000808
:1000B0006518000889010008890100088901000805
:1000C00089010008890100088901000889010008E8
:1000D0008901000889010008491200084F12000830
:1000E000CD1600088901000889010008890100086F
:1000F00089010008890100088901000889010008B8
:1001000089010008890100086B18000889010008AE
:100110008901000889010008890100088901000897
:100120008901000889010008890100088901000887
:100130008901000889010008890100088901000877
:100140008901000889010008890100088901000867
:100150008901000889010008890100088901000857
:100160008901000889010008890100088901000847
:1001700089010008890100088901000800000000C9
:10018000000000008901000800F0C4B900F004BBC1
:100190007047000070B50C46064600F061F9094B47
:1001A000094A1D682919914202D8084A914204D28D
:1001B0000C2333604FF0FF3500E0196000F058F970
:1001C000284670BD000200200000022000510020DF
:1001D0001946104600F0ECBA1946104600F0F0BA85
:1001E000132303604FF0FF307047132303604FF079
:1001F000FF307047132303604FF0FF307047022930
:100200004FF0000303608CBF002001207047000006
:10021000114B70B500241C60104B114D18682E68EE
:1002200000F09CF80F4B53F820301B68A3F1080234
:1002300096420FD026B13179092904BF0A213171C4
:10024000092103F8041C33F9021C074B2A601980AA
:10025000012070BD204670BDC00200209403002024
:10026000C8020020D0020020C4020020082930B5B6
:10027000037919D9082B32D842791A4B53F82250F6
:1002800000F108042DB12D68856053F822502C60D0
:1002900000E0846043F82240134C4279012303FAC2
:1002A00002F22368134319E0082B18D945790D4B46
:1002B00053F825203AB11468A2420BBF00222468EB
:1002C00043F825201460427953F822303BB9064C9C
:1002D000012303FA02F2236823EA02032360017177
:1002E00030BD00BFD00200209403002008B50A4BA7
:1002F0001B681A79082A02D95B7983420AD900F06F
:10030000BAF818B1054B01221A6008BDBDE80840D3
:1003100000F082B808BD00BFC8020020C002002063
:1003200008B500F09DF8094B094A1B88094D1BB21E
:10033000002442F82340084A286813682146013BFC
:100340001360FFF793FF2C6000F062F8C4020020F6
:1003500010030020C8020020CC0200200023C207A6
:1003600002D440080133FAE718467047134423F0DB
:10037000030310B54FF077321C1F43F8042C6207BB
:1003800042BF4FF0883243F8082CA3F108044FF025
:10039000807304E909000F4B44F80C3C002344F837
:1003A000103C032344F8143C2246022344F8183C32
:1003B000012344F81C3C42F8201D0B2342F8043D65
:1003C000013B032BFAD120466FF0020340F8443D75
:1003D00010BD00BF21030008064B0749074A1868F3
:1003E000884203D1934201D20433F8E70348C01A8C
:1003F000704700BF00000020FEE7FEE7000200207B
:10040000EFF30880704700000048704700000020AC
:1004100000F02AF801DFFEE7024A536843F08053F8
:100420005360704700ED00E0EFF3098020E9F00F22
:1004300040F804ED02490968086000F003F8000084
:10044000C8020020FFF7E4FE04480068016801C903
:10045000B1E8F00F81F3098800470000C8020020CE
:10046000EFF3108072B6704762B6EFF310807047FA
:1004700080F310887047EFF30580C0B2704700002A
:100480000D490E4A0E4B6846904203D8984201D956
:10049000002102E009468D460121042072460242F5
:1004A00002D1EFF3088001E0EFF309802DE9F00FAE
:1004B0006B4600F06FF800BF000200200000022031
:1004C0006005002008B50249042000F08DFB00BF44
:1004D000CCC7000808B50249062000F085FB00BF24
:1004E000D8C7000808B50249072000F07DFB00BF0F
:1004F000EBC7000808B50249082000F075FB00BFF3
:10050000FDC7000808B50249092000F06DFB00BFD7
:1005100011C8000808B502490A2000F065FB00BFB9
:1005200023C800087047704708B5FFF7FBFF6A460D
:10053000114B1249934202D243F8041BFAE7104AC6
:10054000104B11498B4204D252F8040F43F8040BAC
:10055000F8E70E4B0E4A0021934202D243F8041BE7
:10056000FAE7FFF7E0FF00F01FFB0AF095FCBDE89B
:10057000084000F073BB00BF00000020FEE7FEE76C
:1005800034D6000800020020C0020020C002002073
:10059000005100202DE9F04F9A46494B8FB0934609
:1005A0009A6B03925A6B04929F6ADA6A05921A6BED
:1005B000DB6B0793434B06921A68434B9A420446FF
:1005C000884602D041480AF0ADFEB8F1000F05D0D0
:1005D0003F4800250AF0A6FE2E4626E094E80E00CD
:1005E000E068D4F81C9008902069099060690A902E
:1005F00019F4007F3748A6690D930CBF04F120055C
:1006000004F124050C920B910AF08CFE089B0093D8
:100610000BA90EC930480AF0FBFDCDF80090334617
:100620000A9A09992D480AF0F3FD2D480AF07AFE3E
:1006300039462C480AF0ECFD05992B480AF0E8FDF4
:1006400006992A480AF0E4FD079929480AF0E0FDD6
:100650003A0403D5039927480AF0DAFD3B0603D58F
:10066000049925480AF0D4FD24480AF05BFE594657
:1006700023480AF0CDFDB8F1000F1BD121480AF044
:1006800051FE314620480AF0C3FD69461F4BC91A86
:1006900003D549421E480AF0BBFD20468268C36864
:1006A00001698C4641698E46AD46514691E8F00F8E
:1006B0004168006801BE1749052000F095FA00BFA7
:1006C00000ED00E000000020FEE7FEE731C8000872
:1006D00047C8000876C8000891C80008CEC80008BE
:1006E0000CC9000815C9000825C9000835C900084B
:1006F00045C9000855C9000865C9000875C9000842
:100700007AC900088CC90008BDC90008580100203A
:10071000E5C9000812CA000810B568B1012815D152
:10072000174A136823F003031360136843F400733C
:1007300043F0010313601BE0114B1A6842F00E02F4
:100740001A605A6842F480725A6011E00D4A1369C7
:1007500023F0040313610024FFF782FEBFF34F8FE1
:1007600030BFFFF785FE54B1BDE8104000F010BC6B
:10077000044A136943F0040313610124ECE710BD3C
:100780000070004000ED00E008B5FFF769FE0020B2
:10079000BDE80840FFF7C0BF034B044A4FF4E13106
:1007A000002000F0C7BC00BF04020020270E000894
:1007B0000A460146014800F041BB00BF0402002088
:1007C00010B50A460C460146002000F019FD2046EF
:1007D00010BD002000F0F0BF034B1968024611B9AC
:1007E000084600F0C9BF7047DC03002010B5094A75
:1007F00013685BB19C6881688C4202D21A461B6800
:10080000F7E703D15C6841688C42F7D90360106058
:1008100010BD00BFE8030020F0B51F4E1F4D336828
:100820001F4C013333601F4B00201A6818602B687F
:10083000226019460746B64641B1DEF800C08E6810
:10084000664503D80F4601200968F5E700B1296025
:1008500007B9F0BD00213960E2B133B15168586881
:10086000814294BF1146194600E0114608461268BD
:100870001B680AB903600BE00BB9026008E0556819
:100880005E68B54294BF15461D4605602846EEE7F2
:100890002160F0BD2360F0BDE0030020E8030020EC
:1008A000E4030020D80300202DE9F0412E4F2F4C07
:1008B00001233B6023683BB9FFF7AEFFFFF789FFD9
:1008C0000130FBD0002502E0FFF783FF05464FF023
:1008D0000008236823B9FFF77CFF854214D91AE08A
:1008E0005E68FFF776FF854208D923685E68FFF7E8
:1008F00070FFA8422CD3B042F7D329E08642F4D946
:10090000361A132EE7D8F0E7236843B9FFF761FFE3
:10091000854206460BD9FFF77FFF0025D9E75E68C1
:10092000FFF757FF063E14308642D2D309E010F19C
:10093000140F04D3FFF74DFF8642FBD9EBE74FF0CE
:10094000FF3600233B603046BDE8F041FFF744BF6F
:1009500023681A682260C3F80480C3F80880DA6844
:1009600018699047B5E700BFDC030020E4030020CE
:10097000144B1A6882420AD112681A6012B1506888
:10098000063801E04FF0FF30FFF726BF13461A6824
:1009900022B19042FAD102681A6070470A4A13687D
:1009A0001BB1984203D01A46F9E7084A05E00368EC
:1009B000136070479842FAD01A461368002BF9D199
:1009C000704700BFE4030020D8030020E8030020A4
:1009D00008B500231846054A054900F0FFFE4FF010
:1009E000FF30BDE80840FFF7F7BE00BFA9080008C8
:1009F00040420F0070B5084EFFF7EBFE3468054625
:100A0000FFF7E7FE8542F7D800222346141843F18A
:100A100000052046294670BDE0030020F8B50446D5
:100A20000D46FFF7D6FE002385420646236010D30D
:100A3000A5F10A0383420CD20A35FFF7CAFE8542AC
:100A4000FBD3FFF7C6FE8542FBD8E36820699847D1
:100A50003EE0FFF705FD63680746002B34D1A3682D
:100A6000002B31D11B4B65601A681B68B54238BF3B
:100A70000132A260A2689A4203D92046FFF7B6FE6F
:100A80001EE0B54202D9144B19460EE0134A136812
:100A900023B159688D4201D31A46F8E723601460E8
:100AA0000EE05068854203D313461A68002AF8D135
:100AB00022601C600B689C4202D1A81FFFF78CFECD
:100AC0003846FFF7D5FC03E02046FFF751FFC9E7A2
:100AD0000020F8BDE0030020E4030020D80300203C
:100AE00038B50446FFF7BCFC6368054633B9A36814
:100AF00023B92846BDE83840FFF7BABC2046FFF7C7
:100B000037FFF6E7C36870B504460D46C3B1FFF77B
:100B1000E7FF092D0CD8FFF75CFE0646FFF759FEEC
:100B2000801B8542FAD8E3682069BDE87040184709
:100B3000FFF74FFE29182046BDE87040FFF76EBF53
:100B400070BD00002DE9F04704460E4690461AB9E4
:100B5000BDE8F047FFF7D6BFFFF782FC63680746A2
:100B6000E3B9A368D3B9DFF83CA0FFF732FEDAF8A7
:100B700000508146FFF72DFE8145F6D8304408EB42
:100B80000502864288BF01326060A2602046FFF7FE
:100B90002DFE3846BDE8F047FFF76ABC2046FFF758
:100BA000E7FEE0E7E003002008B50121094800F076
:100BB0009BFC0121084800F097FC0121074800F048
:100BC00093FC0121064800F08FFCBDE8084000F0CE
:100BD00021B900BF0D0C02400C0C02400E0C02406B
:100BE0000F0C02407047000008B50F4B1A680C4606
:100BF0009AB9012203281A6003D171460B480AF002
:100C000007FB21460A480AF003FB00F04FF90948A8
:100C10000AF0FEFA08480AF0FBFAFFF721FCFFF79A
:100C2000E1FFFFF7B1FD00BFEC03002037CA000869
:100C30003BCA000863CA000857CA000808B500F09C
:100C4000B7FE03480AF0E4FA00F06CFE002008BD8D
:100C500065CA000808B500F00BF9FCE71FB5FFF7FF
:100C6000FFFB0E4B0E481B68029300240D4B0093B4
:100C70000F220C234FF48071019400F055F80A4BB9
:100C80000A481B6802930A4B009307220C234FF477
:100C9000C061019400F048F8FFF7BAFB1802002089
:100CA000F0030020550C00081C020020F004002076
:100CB0003D0C000808B5FFF7D3FB094B1B681A79F8
:100CC000082A07D95A79074B53F8221011B109683D
:100CD00043F82210FFF7CCFBBDE80840FFF79CBBB0
:100CE000C8020020D002002038B50B79082B03D9A8
:100CF00008490320FFF778FF4C7901F108020368E7
:100D00002BB113F8035CAC4201D31846F7E78B60B4
:100D1000026038BD25CA0008031F53F8042F9A4209
:100D2000FBD0181A704700000F2A2DE9F74F05462F
:100D30008B4691469A462AD810F003031BBFC3F195
:100D40000403ED180B46CB1A303B23F003031AF0D3
:100D5000080F05EB030405D02A46A24203D2126015
:100D60000432FAE72D600193FFF77AFB2749019BD4
:100D70008046012251F8227016B25FB10132212A59
:100D8000F8D14046FFF774FB6FF08A003BE06FF04C
:100D9000150038E01D490C9841F822402A46E680AB
:100DA0000D99FFF7E3FA0E9B194AA3624FF0FF3348
:100DB000E3611368206001331AF0010F6562C4F823
:100DC0002CB084F805902771A760E7602761676100
:100DD000A7612762136004D001212046FFF746FA7D
:100DE0000DE00A212046FFF741FA1AF0040F06D160
:100DF0004046FFF73DFB4846FFF778FA02E04046E1
:100E0000FFF736FB304603B0BDE8F08F100300203B
:100E1000CC02002008B500F063FE00F0B9F8BDE890
:100E2000084000F01CB838B50446043000F035FD29
:100E30000546204600F02EFE284638BDF8B504468B
:100E40000E461746051D3A463146284600F010FD6D
:100E500020B90121204600F0EDFDF4E7F8BD08B50A
:100E6000002000F01BFA0120BDE8084000F016BA8F
:100E7000F8B50D4B1E68C6F307221D4622B9F4B221
:100E8000003418BF012400E00224FFF7E9FA2B68C0
:100E90009E42074602D12046FFF73EFC3846BDE899
:100EA000F840FFF7E5BA00BF200200202DE9F04F1F
:100EB0002C4B2D4A1B882D492D482E4EDFF8CCB0E7
:100EC0008BB00DF1280906F1800A29F8043D0AF0DB
:100ED0009FF9FFF781FA0546FFF796FA0446FFF7F8
:100EE0008FFA2A46009023464FF4007122480AF0F8
:100EF0008FF925EAE5754FF4007856F8044B14B3E2
:100F00002779E26A5BF82730606A0793904406927B
:100F1000FFF702FF069AB4F90610079B101A226821
:100F20000592626A04920390E26A029262790192E7
:100F3000082FD4BF4F4609F1010700970544A26A64
:100F40000E480AF065F9B245D7D10D4B02958DE8F0
:100F500008010C4A0C4819460AF05AF90BB0BDE8D2
:100F6000F08F00BFBDCA0008ECCA0008F2CA000832
:100F7000F7CA0008140300203FCB000889CB000803
:100F8000C5CB0008C7CB0008CBCB0008C0CA0008FF
:100F900038B5FFF765FA1B4C0023E360054600F007
:100FA00037F84FF41443A360A268164B12F00C0FED
:100FB000FAD1154A40F20571116081221A601A684F
:100FC00042F480321A601A6812F4003F0D4AFAD0D7
:100FD0000E4B5360136843F0807313601168094B24
:100FE0008901FBD59A6842F002029A609A6802F081
:100FF0000C02082AFAD100F017F82846BDE838405C
:10100000FFF736BA00380240003C0240042A40078D
:10101000044B1A6842F001021A601A689207FCD564
:10102000704700BF00380240044B9A6812F00C0F62
:101030001EBF1A6822F001021A6070470038024091
:10104000034B044A00280CBF10461846704700BFE7
:1010500000BD010580DE800204281CD8DFE800F016
:1010600003080D1217000D4B1A6C1143196412E09E
:101070000A4A536C194351640DE0084A136B194333
:10108000116308E0054A536B1943516303E0034AB7
:10109000936B19439163BFF34F8F70470038024041
:1010A000042821D8DFE800F003090F151B000F4AC0
:1010B000136C23EA0101116470470C4A536C23EA54
:1010C000010151647047094A136B23EA010111635E
:1010D0007047064A536B23EA010151637047034A84
:1010E000936B23EA01019163704700BF003802400F
:1010F00038B514230C4A4343D4582568AA0608D5AA
:101100000A4B616803EBC002C9B253F83030506833
:1011100098472B0748BF6368054B1B681BB1BDE8A8
:101120003840FFF7C7BD38BD44CC0008F00A0020A6
:10113000C002002001282DE9F04780460D461746E1
:1011400003D92B490320FFF74FFDDFF8B090294A60
:10115000142404FB009442F83070E66802EBC002ED
:1011600001215360304600F0BFF9304600F09AFA92
:101170003046617C00F054FA4E464FB1D4F80890E6
:101180000021484600F0B0F9217C484600F048FABA
:10119000142303FB08F806EB080999F812A0D9F804
:1011A00004105046FFF758FF56F808400023E3604C
:1011B000504623616361FFF743FFB0FBF5F080B257
:1011C000A06077B199F8133001215AB203F01F03E0
:1011D00001FA03F35209084941F8223042F22C0384
:1011E00001E042F20803E3600020BDE8F08700BFA1
:1011F00025CA0008F00A002000E100E044CC000805
:10120000012838B505D80E4C14230A4403FB0043CB
:1012100009E00C490320FFF7E7FC25682D06FCD503
:1012200011F8015B65608A4201D01C68F5E7142360
:101230005843034B1A5813685B06FCD538BD00BFF2
:1012400044CC000825CA00080020FFF751BF012048
:10125000FFF74EBFF8B5104C04EB4014012167684E
:10126000384600F041F9A6680021304600F03CF90C
:10127000E5680121284600F037F9247D38462146EB
:1012800000F0CEF92146304600F0CAF92146284642
:10129000BDE8F84000F0C4B978CC000801282DE979
:1012A000F041044603D910490320FFF79DFC0F4B82
:1012B000DFF83C80002543F820506401FFF7CAFFA7
:1012C00008EB04031E7F9F6930463946FFF7C4FED2
:1012D00058F8043039461D603046DD615D60BDE878
:1012E000F041FFF7DDBE00BF25CA0008000B00205B
:1012F00078CC0008012870B50C4621D84A1C22D0B1
:1013000021F0FF0313F5807F11D114F0FF041AD1EF
:101310000E4B03EB40152E69731C14D0012130468F
:1013200000F0E2F8297D304600F07AF906E001216C
:10133000204600F0D9F8204600F0B4F9002070BD36
:101340004FF0FF3070BD6FF0010070BD78CC000829
:10135000042B2DE9F84304460E461546984603D95A
:1013600017490320FFF740FC1648DFF8609067013B
:10137000012100EB840000F05DFB09EB07031C7FFB
:1013800099692046FFF768FE0F4B59F8071004EBE8
:1013900084041C4416F5807F14F8082045EAC20531
:1013A00045F004050D6015BF0B684B6843F44073AE
:1013B00043F0040314BF0B604B600020BDE8F883CA
:1013C00025CA0008000B00206CCC000878CC00086F
:1013D0000B4A430110B50446D018D3588169007FE9
:1013E00000221A605A6822F004025A60FFF758FE81
:1013F000044800EB8400BDE8104000F04BBB00BF88
:1014000078CC0008000B00202DE9F843089E099FC6
:10141000884691461D4623B91EB931490320FFF77E
:10142000E3FB304B400118F5807F1C58236843F0E4
:101430004003236005D0B8F1FF3F02D0404600F0E2
:101440003AF9A6B92F44AF4206D0A3689E07FCD54F
:1014500015F8013B2373F6E7A3689807FCD5A3684A
:101460001906FCD4A368DA0720D5E368FAE70DB1C2
:10147000002319E030463744B84217D0A3689B07D1
:10148000FCD52573A368DE07FCD5237B00F8013B60
:10149000F2E7A2689007FCD5EA5C2273A268D10744
:1014A000FCD5227BF2540133BB42F2D1A3689A07E8
:1014B000FCD5A3681B06FCD4B9F1000F0ED1B8F11E
:1014C000FF3F0BD0236818F5807F23F04003236093
:1014D00004D04046BDE8F84300F0E4B8BDE8F88326
:1014E00025CA000878CC0008F8B50D460126C0F3DF
:1014F000832120F00F0400F00F0706FA01F102200B
:10150000FFF7AAFD07FA06F00323216883406FEA7C
:10151000030C01EA0C012160216805F0030E0EFAAC
:1015200000FE4EEA01012160E2680CEA0202E2607C
:10153000E168C5F3810282400A43E2606268BE400E
:1015400022EA060666606268C5F30015BD401543D1
:101550006560A2681343A3600020F8BD2DE9F04147
:1015600000F00F0415462B4A42F8343002EBC40257
:10157000069B536006468846C0F383274FF480419C
:101580000120FFF769FD41463046FFF7ADFF042C0F
:10159000214B03DCA11D01228A4003E0092C03DC5E
:1015A0004FF400021A6002E04FF480725A601B4B45
:1015B0000120996800FA04F2D243114099609968B9
:1015C00005EA000E0EFA04FE4EEA01019960D968A0
:1015D0000A40DA60C540DA68A54004F00C0404F162
:1015E000804404F59C341543DD6006F00302A568D1
:1015F00092000F21914025EA0101A160A168974066
:10160000B0400F43A76058611A681043186000206B
:10161000BDE8F081080B002000E100E0003C014043
:1016200020F00F0300F00F02F0B51E6857000325ED
:10163000BD4026EA05051D601D680224072A04FA3C
:1016400007F444EA050494BF002201221C6003EB66
:10165000820300F007001C6A80000F22824024EA07
:1016600002021A621A6A814041EA02001862F0BD61
:10167000044900F00F000B68012202FA00F0034356
:101680000B607047003C0140054900F00F000B68FB
:10169000012202FA00F023EA00030B60704700BF4A
:1016A000003C014020F00F02012300F00F0003FA7C
:1016B00000F09061704720F00F0200F00F00103032
:1016C000012303FA00F0906170470000104B2DE9F0
:1016D000F0415E691A680F4F164000244FF0010870
:1016E0001D4608FA04F31E4206D06B6107EBC403E3
:1016F00057F83420586890470134102CF1D1064B2C
:101700001B681BB1BDE8F041FFF7D4BABDE8F0811A
:10171000003C0140080B0020C00200202DE9F843E6
:10172000124ADFF8508003010746D5582E69EB684E
:1017300000241E4008EBC0090223A3401E4209D02A
:10174000EA68D9F8040022EA0303EB60214658F85E
:10175000373098470134042CEED1054B1B681BB180
:10176000BDE8F843FFF7A6BABDE8F883B8CC000897
:10177000C0020020880B0020032910B516D80D4B9D
:1017800000011C181B586068024001F10C0003EBBB
:10179000800042601869022202FA01F120EA010287
:1017A0001A61DA681143D960002010BD4FF0FF3094
:1017B00010BD00BFB8CC00080001024B1B58586A8E
:1017C000704700BFB8CC0008034B00011A581368DB
:1017D00043F0010313607047B8CC000801282DE9DD
:1017E000F8430546884630D81A4E1B49040137197C
:1017F00041F8302097F80C9001EBC00148464B604F
:10180000B968FFF729FC36597B68002434604846E4
:101810007460F362FFF714FC104B7A7B13F8093005
:101820005843B0FBF8F3013BB36251B2012302F01D
:101830001F02736149099340094A284642F8213042
:10184000FFF7C2FF2046BDE8F8834FF0FF30BDE848
:10185000F88300BFB8CC0008880B0020D8CC000863
:1018600000E100E00020FFF759BF0120FFF756BF5D
:1018700070B513467BB18568C468A5420BD08468F7
:101880000668651C85604568013D2C40013B345D60
:1018900001F8014BEEE7D01A70BDC368426830B55D
:1018A00084681B1B934208D0C3680468013A5D1C1E
:1018B0001340C560E154002030BD4FF0FF3030BD13
:1018C000024A137801331370704700BFA00B002049
:1018D00007B50D4800900D4B01220021FFF73EFE99
:1018E000002804DA0A4809F01DFD012009E0094832
:1018F00009F08EFC084B00201860084B1870084B4C
:10190000186003B05DF804FB08000240C11800082D
:10191000DACC000816CD0008980B0020A00B0020A0
:101920009C0B002080B5FFF7D3FF194E0025194C02
:10193000174F0020FFF740FF3368C01AA042F7D9C5
:101940001548DFF86490DFF86480FFF79DFE134BC5
:1019500000201C78124B93FBF4F4FFF72DFF3B683B
:10196000C01AB4FBF0F499F8000044430020C8F812
:101970000040FFF721FFD8F800103860094889F8C7
:10198000005009F045FC0448FFF772FECFE700BFA6
:101990009C0B00203F420F00080002402402002060
:1019A000008793033CCD0008A00B0020980B00207B
:1019B00008B5002006F05EFEFFF70AF802F060FEB0
:1019C00003F042F804F0F2FB00F064FA06F02CFB9E
:1019D00000F006F800F07CFFBDE8084003F052B8C4
:1019E00013B50E4C0E490F4807F022F90D49204659
:1019F00002F07EFB002806DA0B48002102B0BDE8A9
:101A0000104009F005BC0094084B094802224FF42D
:101A1000806102F003FC02B010BD00BFFC0F00208B
:101A20004CCD0008A40F002064CD00089ECD000816
:101A3000A10B002070B505460C46FEF711FD2B6882
:101A400006462BB94FF0FF332B60FEF711FD18E06F
:101A5000CCB10F4B1C6802212046FEF707FC2B6817
:101A6000013305D104F108032B600023A36003E0D8
:101A700021462846FFF738F93046FEF7F9FCFEF715
:101A8000CBFC012070BDFEF7F3FC204670BD00BF0B
:101A9000C802002070B50446FEF7E2FC2568064641
:101AA0001DB16B1C05D100232360BDE87040FEF71B
:101AB000DFBC28460A2150F808392360FEF7D6FB20
:101AC000236813B94FF0FF33236015F8034C3046F9
:101AD000FEF7CEFC2046BDE87040FEF707BC0000D4
:101AE0000F4BD3F8882042F47002C3F888200D4AC7
:101AF0009A60102283F822200021DA7701F16040F9
:101B000000F561400131522980F80023F6D11A69AD
:101B100042F010021A615A6942F400725A61704729
:101B200000ED00E000000008034600201BB1DA6869
:101B30005B681044FAE7704710B50822094904466B
:101B400009F0D2F948B12378FF2B08D1607800F072
:101B50000F00831E5842584110BD012010BD0020C7
:101B600010BD00BF70CF0008002102F097BE38B54D
:101B7000CBB2002114460246084602F085FB05461A
:101B800018B92046FFF7F0FF0FE094F91030013349
:101B90000AD1A36882681B7903F03F0321462046DF
:101BA000137102F03BFC04466C60284638BD00000F
:101BB0002DE9F0478C680746104688461546FFF722
:101BC000B3FFA37940BAFF2BA0800AD12B7C023B44
:101BD000DBB2022B03D8214AD35CFF2B00D13B237D
:101BE000A371E37943B90FB9402304E0384600F00C
:101BF000CBFC90F8CA31E37104F1080610221849B1
:101C0000304609F071F98246D0B904F11809154936
:101C10001022484609F068F9014630B910223046D2
:101C200009F092FA0123E3750AE049465246384624
:101C300000F084FD014618B11022304609F086F903
:101C40004146284602F0A4FB002804DA831C08BFA2
:101C50000020BDE8F0870020BDE8F087ADCD00088A
:101C6000C0CF0008D0CF00088B6870B558800C46F4
:101C7000054600F089FC014618B919490320FEF712
:101C8000B3FF66683046FFF74FFFB1F8C83198429E
:101C900004D92046BDE87040FFF766BFD1F81C327A
:101CA0000133C1F81C323046FFF73EFFD1F8243231
:101CB0001844B1F8C631C1F82402DB0708D5234621
:101CC00040F202220749012002F078F830B9E0E73B
:101CD0002146284602F09DF80028DADD70BD00BFDD
:101CE00025CA00080000FFFF2DE9F04F85B090F9EC
:101CF0001030013300AF044689460AD18368B3F936
:101D0000026002F0D9FD00286AD043680446984674
:101D100001E080460026404602F0CEFD0546002840
:101D20005ED04445836818BF60601A461B7ED0F8B9
:101D3000048008BF0446FF2B2BD186B907F10800A9
:101D400002F096FA00284BD0002122460846B7F947
:101D50000860FFF70CFF0446002800F09380B9F1FB
:101D6000000F06D0424629463046FFF721FF0028E3
:101D700036DBA268137943F040031371304600F05C
:101D80005BFE43680133436021463046FFF76CFF3A
:101D900078E01346183310223C4918469B4609F058
:101DA000A3F840B15946002E39D1381D00F06AFC25
:101DB0000646002838D0B9F1000F06D04246294621
:101DC0003046FFF7F5FE00280ADB2846FFF7ACFE99
:101DD000002102460223084602F06EFC064608B9BE
:101DE000204619E083689846EA68A968404609F0E9
:101DF000ADF8EB686D6842461A449046002DF3D169
:101E00002046FFF7B1FE224B3146B3F9000002F045
:101E10000DF8002836DC3046FFF7A6FE32E03046EB
:101E200000F008FC0028C6D107F11001082301F8D2
:101E30000D3D32465B4607F1080005F05FFCEA46BF
:101E4000064640B1B9F1000F09D042462946FFF7D6
:101E5000AFFE002803DA2046FFF786FE11E0224697
:101E6000F97807F10800FFF782FE044648B13046D2
:101E700000F0E2FD03680133036021463046FFF7BE
:101E8000F3FED5461437BD46BDE8F08FD0CF00082D
:101E9000401000201FB50F4CB4F9003063B90E4A52
:101EA00001930E4B02920093042208234FF48061A9
:101EB0000B48FEF739FF20800A480B4B03600123D3
:101EC00003711423836008F0B3F9B4F9000004B07F
:101ED00010BD00BF40100020A8CD00088D210008D3
:101EE000421000200C10002048140020292B2DE95E
:101EF000F84381460F4614461D4606D03A2B06D0BD
:101F0000112B0CBF0423002302E0022300E0032373
:101F1000292D3B7401D03A2D03D1A74259D1012676
:101F200005E0A74202D063689F4252D100267B6839
:101F300093F91000022805D016B30121204602F0C3
:101F40009BFC1DE0294602F007FA18B986F001084B
:101F500036B101E04FF000080121204602F08CFC70
:101F6000234640F201221E4997F9100001F026FF96
:101F700010B92046FFF7F8FDB8F1000FDCD00AE0F9
:101F8000234640F201222946022001F017FF10B932
:101F90002046FFF7E9FD06B3292D07D03A2D18D1C9
:101FA00021464846BDE8F84308F004BA00232374EC
:101FB000616839B191F91030022B03D1204602F04B
:101FC0002DFAF5E7022323742046BDE8F84300F01C
:101FD0000BB804490320FEF707FEBDE8F88300BFF5
:101FE0000000FFFF25CA00082DE9F047044618B994
:101FF00064490320FEF7F8FD4FF0FF3102F0D9F9F4
:102000000546A0B18368B3F90260002EF0D03046D7
:1020100000F012FD43690133014643612046FFF79A
:1020200083FDEA688B699B1A1844886100E00646C4
:102030002746254695F91030022B08D1EB68282B4E
:1020400005D1AB681B7803F0F003602B08D0D5F8FE
:1020500004802F46B8F1000F6ED04546EAE73C46B3
:10206000D5F80880E368B8F8041049BA89B29942F3
:1020700003D2204602F0A8FB0FE022460023D068DE
:10208000034492F91000022803D1283B994204D955
:102090005DE05268002AF2D1F7E708F11809102232
:1020A0003949484608F020FF002855D04846FFF738
:1020B00043FD494600B136B9002000F0E3FA002E96
:1020C00008BF064602E0304600F0B4FAB0FA80F0ED
:1020D0004009002840D008F10800FFF72DFDB0BBF3
:1020E0004846FFF729FD90BB98F80730013BDBB26B
:1020F00088F807305BB3284602F0DEFB38B34FF0B8
:10210000FF31204602F055F9014610B1204602F099
:1021100085F921460025084602F0CEFB18B928466D
:10212000FFF722FD13E04168456005460029F2D122
:10213000BDE8F047FFF7D8BDA3681B7803F0F003B4
:10214000602B04D1204602F0B7FB074668B9204651
:10215000BDE8F047FFF708BD98F80630224639463B
:102160003046BDE8F047FFF7C1BE0222282102F049
:10217000BDFA87F81080054600287FF470AF384616
:10218000E6E700BF25CA0008D0CF000810B598B018
:10219000514B0693514B08211B88ADF81C3008A801
:1021A0000024059407F0CCFD05A9022002F0A2F856
:1021B00040F20523ADF80E3001A807F0BDFDBDF8D3
:1021C00006306FF400721344222BF5D801A252F8A6
:1021D00023F000BF61220008692200087322000872
:1021E00073220008B9210008B9210008B9210008AC
:1021F000B9210008B9210008B9210008B921000857
:10220000B9210008B9210008B9210008B921000846
:1022100083220008B92100088F220008B921000894
:10222000B9210008C7220008B92100089722000838
:10223000B9210008B9210008B9210008B921000816
:10224000B9210008B9210008B9210008B921000806
:102250009F220008A7220008AF220008BF22000822
:102260000298FFF7C1FEA7E701210298FFF73CFDA6
:10227000A2E76FF0850303A901A8049307F02EFDE0
:102280009AE7029A537E23F00803537694E7029864
:1022900000F044FF90E7029800F0CEFF8CE7029830
:1022A00005F0A6F988E7029805F0F8F984E7029BA3
:1022B000587C00F00F0003F0E5FF04747CE70298FF
:1022C00005F052FC78E7029A00231946B2F91A0089
:1022D00001F012FB70E700BF0000FFFFC402002006
:1022E0000121FFF7A7BB2DE9F84300F5E07507468C
:1022F00028468846FFF7F4FF00244FF0380909FB11
:1023000004764146304606F028F838B11022002104
:10231000304608F019FF0023337402E00134082C22
:10232000EDD12846BDE8F843FFF7B4BB08B510224D
:10233000034908F0D9FDB0FA80F0400908BD00BF9C
:10234000C0CF000810B508220949044608F0CCFDAA
:1023500048B12378FF2B08D1607800F00F00831E6E
:102360005842584110BD012010BD002010BD00BFD3
:1023700070CF00082DE9FF470026054688469246A3
:1023800099463446AF194146384605F0E6FF002825
:102390007FD13846FFF7CAFF10B1002C08BF3C467A
:1023A0003836B6F5E07FEDD12746002C71D01022EB
:1023B0004146204608F0CAFD237884F811A0FF2B7F
:1023C00084F8109016D0B5F8C631DA0712D501F0AE
:1023D000E1F8814670B105F5E0763046FFF75AFB2B
:1023E000B5F9C4014B464A46214601F083F930460F
:1023F000FFF776FF98F80030FF2B04D1237C43F0E1
:102400000103237441E04046FFF79CFF8146C8B9B1
:10241000B5F8C62102F00602062A17D105F5E076C6
:102420003046FFF737FBB5F8C631DB0706D54B461C
:102430004A464946B5F9C40101F05EFA3046FFF755
:102440004FFF03E0237C63F07F032374B5F8C631AC
:1024500003F00303012B18D040F2FF220023CDE943
:1024600000234FF080730293FF238DF80C3098F80F
:102470000D308DF80D30B8F80E30ADF80E308022EA
:10248000002369462846FFF775FF40F21123638653
:102490006463384604B0BDE8F08703885BBA23F074
:1024A0003F031B041B0C4FF6C062934209D0037814
:1024B000FF2B08D1407800F00F00052818BF0E2030
:1024C0007047052070470E2070472DE9F047002522
:1024D000804691461F460C462E464FF0010A3FB1FA
:1024E0003A780AFA05F31A421AD0237CDB0717D48C
:1024F0002046FFF71BFF98B94946204605F042FFEA
:1025000037B999F80030FF2B02D0637C834207D89B
:10251000B04205D9B8F1000F01D0C8F80040064616
:102520000135082D04F13804D9D13046BDE8F087D3
:1025300070B5134CB4F9C451A84206461ED0EDB98B
:1025400004F5E070FFF7CCFE4FF4A063A4F8C831A7
:10255000402384F8CA31A4F8C4612B46A4F8C651BC
:10256000802208492046FFF705FF04F5E070FFF7D9
:1025700091FA2046BDE8704000F06CBE70BD00BF0F
:10258000C816002090CF0008034BB3F9C421824243
:102590000CBF184600207047C8160020B0F8C6319E
:1025A000DA0707D511B143F0020301E023F002037B
:1025B000A0F8C6317047B0F8C631DB0701D505F089
:1025C00093BA70472DE9F0410D4617469846FFF73C
:1025D000DBFF044610B90020BDE8F0810029FAD0E5
:1025E0000846FFF7A3FE0028F5D1802FF3DC04F5A1
:1025F000E0763046FFF774FE43463A4629462046C9
:10260000FFF7B8FE04463046FFF744FA2046BDE81F
:10261000F081000010B520B90548B0F9C43133B1DC
:1026200001E0FFF7B1FFBDE81040FFF75CBE10BD51
:10263000C81600202DE9F8438946FFF7A5FF044698
:10264000E8B100F5E0763046FFF74AFE002504EBDE
:1026500005084946404605F080FE074628B1304649
:10266000FFF718FA4046BDE8F8833835B5F5E07F46
:10267000EDD13046FFF70EFA3846BDE8F883BDE8E5
:10268000F883000038B5084C0546B4F9C4011DB9FB
:10269000FFF7D0FF20B938BDFFF7CCFF286008B1A5
:1026A000B4F9C40138BD00BFC81600202DE9F341BC
:1026B00002AD00260E4C45F8046D8846074604F529
:1026C000E070FFF70DFE3346424621462846FFF7ED
:1026D000FCFE20B1019B3B60B4F9C44100E004461C
:1026E0000448FFF7D7F9204602B0BDE8F08100BFEB
:1026F000C8160020881800202DE9F34102AC0027FD
:10270000884644F8047DFFF73FFF00F5E075064674
:102710002846FFF7E5FD20463B4642463146FFF797
:10272000D4FE044628461CB1FFF7B4F9019802E034
:10273000FFF7B0F9204602B0BDE8F0812DE9F04F77
:1027400087B00F461546FFF71FFF00F5E073804680
:1027500018460193FFF7C4FD0122002102A808F0EA
:10276000F3FC4646C3464FF0FF3A00244FF0010900
:102770009BF80020FF2A12D05846FFF7D7FD70B90A
:1027800045B99DF8081009FA04F20A438DF80820AB
:10279000A24604E05846FFF7D5FD0028F1D10134E8
:1027A000082C0BF1380BE3D1BAF1FF3F00F0878022
:1027B00004AD22460021284608F0C6FC3B78FF2BDA
:1027C00004D197F8019009F00F0309E03846FFF7AC
:1027D000B9FD20B93846FFF760FE009001E0022302
:1027E00000934FF000094C469DF80810012303FAAE
:1027F00004F2114232D039463046B34605F0ADFD01
:10280000002855D13046FFF79DFD18B93046FFF737
:1028100044FE00E00220009B834208D12A5D04327E
:10282000D2B22A554A4588BF4FF004090AE009D9B7
:102830002A5D0232D2B24A4513462A5538BF4B466A
:102840005FFA83F9B2694AB12A5D0132D2B24A45D0
:1028500013462A5538BF4B465FFA83F90134082CDA
:1028600006F13806C0D10122002102A808F06CFC54
:1028700000209DF80820014601246E5C4E4504BFEF
:1028800004FA01F0024301F1010104BFD2B20120B8
:102890000829F2D108B18DF8082006A8002340F8D5
:1028A0000C3D3A4602AB4146FFF70FFEDDF80CB097
:1028B000BBF1000F05D1382202FB0A8B01E04FF07B
:1028C000000B0198FFF7E6F8584607B0BDE8F08F17
:1028D0002DE9F04F8DB005A801F0CAFC0026544F39
:1028E00003900DF11205B146039B9E4200F09D80BE
:1028F00035F9020FFFF748FE0446002800F09180EA
:1029000000F5E07A5046FFF7EBFC0123B5F9000033
:10291000009300220DF1130317218DF8139001F09D
:1029200093FA86302CD09DF91330012B28D108233F
:102930000DF13008ADF818304FF6FF7328F8103D50
:10294000B7F8C631B5F9000043F003034FF0020BAE
:10295000A7F8C631002206AB0521CDF800B001F082
:1029600099FAB5F90000CDF800B0112143460022D4
:1029700001F06AFABDF82010B5F9000005F040FA40
:102980004FF00808B5F90000CDF8008006AB002232
:10299000414601F059FA00280FDB424606A90AA871
:1029A00008F0D4FA4246234908A808F0CFFA0023D9
:1029B000402208A92046FFF7DDFC0223B5F90000FC
:1029C000009300220DF11603112101F03DFA0028B9
:1029D00006DBBDF81630B3F5A06F28BFA4F8C831E8
:1029E00000231A462421B5F90000CDF8009001F02B
:1029F0002BFAB4F8C6310028CCBF43F0800323F093
:102A00008003A4F8C6315046FFF744F80121204660
:102A1000FFF7C4FDB4F8C631DB0702D5204604F049
:102A2000AFFD013607F50C775EE70DB0BDE8F08F1E
:102A3000C816002070CF000808B5FFF7A5FD00F507
:102A4000057008BD2DE9F3410746884616461C4629
:102A500007F074FE054640B9032300933246A3B243
:102A60004146384607F0FCFD20E0437E03F00703B3
:102A7000012B01D103210DE0027EA3B29A4200F1A5
:102A800010070CD031462C762246384608F05EFA04
:102A90000321284602B0BDE8F04100F08FBE224677
:102AA0003946304608F020FA0028EBD102B0BDE8E4
:102AB000F08100002DE9F04F1D46D37991B0FF2B36
:102AC0008046069116461A9F40F0B4806B78002B22
:102AD00040F0B080172F40F2AD802B7AFF2B00F032
:102AE000A98002F1080955491022484608F0FCF96E
:102AF00070B105F108014046FFF79CFD05900028E4
:102B000000F098800023183F1C4619469A461BE0A7
:102B10000D224B4906F1180008F0E6F9002800F0F4
:102B20008980E6E70AF1180205EB020BAA5C012A8C
:102B30000DD0212A08BF5C469BF801200AEBC20A8F
:102B40001FFA8AFAA7EBC207002FEBDC0BE008ABF9
:102B50002A780698009331465B4601F00DF8031E73
:102B600068DB5946E8E7404607930691FFF70CFDFE
:102B70000699079B18B933490320FEF735F808AAD0
:102B8000002942D0002C40D0B0F8C61101F003015A
:102B900003293AD12978029301924B460A460094C0
:102BA0003146404604F09AFE002304F108020F214A
:102BB000074604F079FE054617B91022494620E081
:102BC000237A83F002038DF82830637A8DF8293058
:102BD000A37A8DF82A30E37A8DF82B30237B8DF899
:102BE0002C30637B8DF82D30A37B8DF82E3008229E
:102BF000E37B8DF82F300AA90EA808F0A7F9124937
:102C000008220CA808F0A2F909E049464046FFF75F
:102C100019FF102249460CA808F098F90025337EC8
:102C20000095A3F1FF025342534105990CAA404677
:102C300000F0D4FC11B0BDE8F08F00BFC0CF000899
:102C4000B0CF000825CA000870CF00082DE9F04F6A
:102C500089B003F108099246059149461D46804610
:102C6000129E07F06BFD9AF80730FF2B40F0B580FD
:102C70006C78002C40F0B180172E40F2AE802B7A99
:102C8000FF2B00F0AA80002800F0A780183E2746FE
:102C9000002E27DD07F1180305EB030BEB5C022B7D
:102CA0000DD0212B16D10023029301932A78CDF861
:102CB00000B04B465146404604F010FE0AE006AB19
:102CC00000932A7805985B46514600F09CFF041E4D
:102CD000C0F283809BF8013007EBC307BFB2A6EBBD
:102CE000C306D5E74FF0FF31059801F062FB08B14C
:102CF000876800E007464946404607F01FFD064644
:102D000000286AD0437E03F00703022B12D127B1BB
:102D10003B7813B17B78002B31D106A9A6F81A8035
:102D20003476224606F1100008F010F92B79590686
:102D300016D512E01FB13B780BB17B7813BB002C8A
:102D400049D1377E003718BF01272B799A062AD43C
:102D50004FB3A4BB2B795B0601D5072101E01FB15E
:102D60000321304600F02AFD95F90430002B737ED4
:102D7000B4BF43F0080323F0080373762DE0002C62
:102D8000CBD12AE02CB3337E9C4209D0224606A93F
:102D900006F1100008F0A8F8B0FA80F0400900E051
:102DA00000200746D1E7002CD4D0A6F81A8034764C
:102DB000224606A906F1100008F0C8F8CAE7737E9B
:102DC00003F00703072B08D10321304600F0F6FC7F
:102DD00003E02746B9E70027B7E709B0BDE8F08F61
:102DE0002DE9F04F87B01546984681460291109F15
:102DF000FFF7CAFBB0F8C6319A07064669D5EB79EA
:102E0000FF2B66D198F80140002C62D1072F60D9C2
:102E100005F10803083F0DF1100A0393002F1FDD91
:102E200004F1080308EB030B18F80330012B0FD152
:102E300098F800200298CDF800A05B46294600F0E3
:102E40009BFE031E45DB524603994846FFF7FAFDF9
:102E50009BF8013004EBC304A4B2A7EBC307DDE782
:102E6000B6F8C63113F0040F05F1080528D013F0A9
:102E7000010F194B194C18BF1C4605F001FC06F553
:102E8000FC7780463846FDF72BFEB6F8C631DB07E7
:102E900016D52946484607F051FC88B1B8FBF4F135
:102EA00040F21523A6F80E320D4BC6F81002B3F906
:102EB000003006F5037204FB1181384605F09EFED2
:102EC0002946484607F03AFC18B1437E23F0080330
:102ED000437607B0BDE8F08F80841E0020A1070074
:102EE000401000202DE9F04F89B0924605918146AF
:102EF0001E46FFF749FB0AF1080B054608228449E4
:102F0000584607F0F1FF002840F0FF809AF808309B
:102F1000FF2B00F0FA809AF80730FF2B40F0F58085
:102F20007378002B40F0F180129B0F2B40F2ED8064
:102F30005946484607F002FC074650B90B23009358
:102F4000024603465946484607F08AFB074668B9D9
:102F5000DBE0437E190706D5F28852BA92B212B965
:102F600023F0080301E043F008037B76F3889CB26A
:102F700064B15CBA674B68491B88A4B21BB207F105
:102F80003002614307F11C0005F038FE33790BB1C4
:102F900085F8CA31B5F8C631C3F30D02A5F8C621CC
:102FA00073791B0203F440431343A5F8C631B0689C
:102FB000A8B1D5F8D03190FA80F898450FD005F037
:102FC0005FFB0A22B0FBF2F303FB1200053008FBA3
:102FD00000F0C5F8D081B0FBF2F0C5F8D401F36879
:102FE00013B11BBAC5F8D83105F5E070FEF752FDF4
:102FF000129B103B0393002302930493039B002B2B
:1030000058DD029B103306EB0308F35C052B1CD044
:1030100004D8012B0DD0032B1ED03FE0222B2AD049
:10302000232B3BD14346129A3146484604F0D4FD47
:1030300034E006AB0093327805984346514600F0E1
:103040009BFD031E049329DA5FE04246317848462F
:1030500000F013FE10BB58E042463178484600F0BD
:1030600029FE002851D0D8F804301BBAB3B19C42D5
:1030700028BF1C4612E04146307804F001FD0028CC
:1030800043D0B8F806305BBA9BB23BB13C22B4FBEC
:10309000F2F2934202D23C2202FB03F498F8013090
:1030A000029A02EBC30292B20292039AA2EBC3030A
:1030B0000393A3E7049B06AA59464846FFF7C2FCC0
:1030C00005F5EE70FDF70CFDB5F8C631DA071CD535
:1030D00004EB4404042C88BFA1084FF0000498BFFF
:1030E0000121384685F8CB4104F0B2FB3B463A4615
:1030F0002146B7F91A0000F0FDFAB5F8C6319B0772
:1031000003D501212846FFF756FA09B0BDE8F08F34
:1031100070CF0008C402002040420F002DE9F041AA
:10312000437E03F00703022B86B0044601D0052B33
:103130007BD194F89420B4F91A50012A71D9022B4A
:1031400011D14FF080730493FF238DF81430637B0B
:103150008DF8153040F2FF200021E389ADF81630DC
:10316000CDE902010BE094E8030002AB83E8030021
:1031700004F1080393E8030006AB03E90300013AF6
:1031800084F894201DBB01AE304601F071F807466B
:10319000BD4208D036F9150002AB2246002100F0EE
:1031A000A9FA0135F4E7224B04F13805B3F90060C0
:1031B0002846FDF795FC40F21223A4F84E3004F1A6
:1031C0004C0233461B49284605F018FD2DE02846E1
:1031D000FFF7DAF90646224602AB06F5E075B4F9C8
:1031E0001A00002100F086FA01212846FEF722FC91
:1031F0000F4BD6F8D871B3F9008004F13806304689
:10320000FDF76EFC40F21223A4F84E3030464346E0
:1032100004F14C02394605F0F1FC2846FEF73AFC71
:1032200003E02146284607F0B1FA06B0BDE8F08178
:103230004010002040420F00437E03F00703042BA0
:1032400003D0072B04D1032100E0052100F0B6BA1A
:103250007047000038B500F5E075044601212846A6
:10326000FEF7E8FB05F00CFA0A210A4BB0FBF1F27D
:1032700002FB11000530C4F8D0314343B3FBF1F336
:10328000C4F8D431044BC4F8D8312846BDE83840DE
:10329000FEF700BC80C3C90140420F0010B50446D0
:1032A00008462378FF2B14D000221823872107F02B
:1032B000EBF8002270B183681A715A719A71DA7151
:1032C00021686268DA609960A168E2685A611961F0
:1032D00010BD002010BD38B50B78FF2B05460C46FD
:1032E000104616D000221823882107F0CDF80022BE
:1032F00080B1836825F01F051D71DA719A715A71CA
:1033000021686268DA609960A168E2685A611961AF
:1033100038BD002038BD08B500220823852107F0FC
:10332000B3F828B1836800221A715A719A71DA7160
:1033300008BD10B5002304461046CA1D02F0F8026D
:10334000194601F0B9F920B182681470C368DB082E
:10335000537010BDF8B516460F461A46B11CFFF75C
:10336000E8FF044660B18568C2680235023A002170
:10337000284607F0E9FE32463946284607F0E6FDC2
:103380002046F8BD13460A4601460120FFF7E2BF7A
:1033900013460A4601460220FFF7DCBF2DE9F04143
:1033A00080460F4616461D460022102386210798A8
:1033B00007F06AF860B1069B846827F03F0776BA89
:1033C0002DBA1BBA84F804806771E680A560E360BB
:1033D000BDE8F0812DE9F0410746884616462021D8
:1033E000079A03201C46FFF7A4FF0546C8B1806872
:1033F00024BA0021846028F03F0800F1100436BA96
:10340000017341738173C173877080F803804660D4
:103410001022204607F098FE3A460699204604F00E
:10342000D7FF2846BDE8F08110B50A4604460821BA
:103430000520FFF77EFF28B18368002224BA9A7026
:10344000DA705C6010BD000008B51022034907F077
:103450004BFDB0FA80F0400908BD00BFC0CF0008A6
:1034600010B508220949044607F03EFD48B123780B
:10347000FF2B08D1607800F00F00831E584258419E
:1034800010BD012010BD002010BD00BF70CF00088E
:1034900070B506460846194607F080F80446A0B104
:1034A0008368FF22DA7100231A461946184600F095
:1034B000EBFE054620B92146204600F0AFFF02E0B2
:1034C00083685E804460284670BD70BD002101F0B5
:1034D000E5B90000F7B51F46537C802B05460E4624
:1034E000144603D911490320FDF77EFB1046FFF770
:1034F000ABFF08B1002017E02046FFF7B1FF00281E
:10350000F8D1217CCB07F5D43388607C626913F055
:10351000010F14BF002680268DE89000A369314377
:10352000FFF758FF2860012003B0F0BD25CA00084E
:1035300030B585B0022300930D460DF10E03002235
:103540000521044600F080FC002803DBBDF80E30A6
:10355000062B10D80823009300222B460221204678
:1035600000F072FC002802DBADF80E000EE0002334
:10357000ADF80E300AE00823009300222B46032109
:10358000204600F061FC0628E4DDEDE7BDF80E0002
:1035900005B030BD38B5002007F01AF9044658B11F
:1035A000637E03F00703013B012B03D90A4B002282
:1035B0001A600EE02046EFE7074D286807F008F98B
:1035C000034618B907F004F9034610B12B601846FA
:1035D00038BD204638BD00BFF81800202DE9F7435C
:1035E0000A9C0F46994680461646FEF7CDFFB0F876
:1035F000C631990701D4002507E04046FEF7C4FF15
:10360000B0F8C6315A07F6D580253046FFF71CFFC3
:1036100038B110223349304607F098FC022373700A
:1036200001E045F04005B9F1000F0BD06946404676
:10363000FFF77EFF30B1C1B222466846FFF7A8FE11
:1036400068B1044624B13B7CDB0758BF45F0200538
:10365000224639462846FFF73EFE814608B92046F5
:103660003BE00146002332464046FFF711FF054686
:1036700008B9484631E03B7CDFF8749013F0010F45
:1036800023D004F0FDFF184BB0FBF3F7314607FBE6
:103690001307404607F052F8044618B913490320AF
:1036A000FDF7A2FA00F154063046FDF719FA40F290
:1036B0000223A4F86A30E566B9F9003004F1680223
:1036C0003946304605F09AFA09E00146B9F900009A
:1036D00000F09FFB002802DC2846FFF7F7FE03B04E
:1036E000BDE8F08380CF000840420F0025CA0008E3
:1036F000401000202DE9FF4707460D4690469946A9
:10370000FEF742FF824618B92A490320FDF76CFAFA
:1037100035B92A4641463846FFF710F8054668B1E4
:1037200002A93846FFF704FF064650B1C1B2002295
:1037300002A8FFF727FE044620B935E006460446F6
:1037400000E00446BAF8C631DB0714D5082E0AD0CB
:103750000823009300226B440321384600F074FBD9
:1037600080B208281FD1234602AA0F21002004F0AE
:103770009BF8C0B1044621464046FFF78FFD064640
:1037800088B101462B464A463846FFF781FE04467B
:1037900008B9304608E0084B0146B3F9000000F0D4
:1037A00038FB002802DC2046FFF790FE04B0BDE89D
:1037B000F08700BF25CA0008401000202DE9F04125
:1037C000437E23F007030B4305290446437620D0AC
:1037D000072903D004294BD1264E05E0B0F91A0081
:1037E000FEF7D2FED0F8D461234B04F13805B3F9CB
:1037F00000702846FDF774F940F21723A4F84E3004
:1038000004F14C023B4631462846BDE8F04105F044
:10381000F5B9B0F91A00FEF7B7FE032306462246B3
:1038200006F5E07584F89430B4F91A0023460021B7
:10383000FFF760FF01212846FEF7FCF80E4BD6F893
:10384000D871B3F9008004F138063046FDF748F925
:1038500040F21223A4F84E303046434604F14C02A5
:10386000394605F0CBF92846BDE8F041FEF712B91C
:10387000BDE8F081404B4C00401000202DE9F341A1
:103880001B4D002918BF0D46002229468046FEF731
:1038900055FF074670B169464046FFF749FE38B10B
:1038A000C1B200226846FFF76DFD044618B91AE060
:1038B000044600E004462046FFF72DFD064688B189
:1038C00001463B462A464046FFF7E2FD044608B95A
:1038D000304608E0074B0146B3F9000000F099FAC2
:1038E000002802DC2046FFF7F1FD02B0BDE8F081C0
:1038F000A0CF0008401000202DE9F04F8BB000272A
:1039000091468A46039302900797FEF73DFE964B39
:10391000064600F5E07801214046B94508BF9946C2
:10392000FEF788F8B6F8C65115F001051BD13446EC
:1039300006F5E377B3465C4500F0ED80627C9BF8CA
:1039400011309A4240F0E4805946204604F01AFDB6
:10395000637C834200F2DC8000E01D463834A045E1
:10396000E8D1079D4FE004F0EFF8054600284AD063
:10397000846906F5E37BECB163689E4218D1AB69BC
:103980009C4200F0D780A268996892F811E0487CC8
:10399000864540F0E38010460593049204F0F2FC63
:1039A000049A059B527C824200F2D88000E01F46B8
:1039B0002468E0E74FF0010B05EBD4039A7D04F097
:1039C00007030BFA03F31A420CD0E0B202F05AFCE0
:1039D000428A417C0346007C009704F0CFF90790AF
:1039E00060B107460134102CE6D12A46A98A28691D
:1039F0003B4604F0E9F90546079020B94046FEF73A
:103A000049F8384681E0B6F8C6311B0707D5294684
:103A1000B6F8C801FFF708FD0790F8B10546BAF1FE
:103A2000000F0FD14046FEF735F8494601220298B3
:103A3000FEF784FE012182464046FDF7FBFFBAF106
:103A4000000F10D008A90298FFF772FD58B1C1B25B
:103A50002A4608A8FFF796FC079018B94046FEF7DB
:103A600019F83DE00546B6F8C62102F01004A4B2EC
:103A70000CB196F8CA4102F020039BB24BB1D6F8C4
:103A8000D4313A498B4206D84FF47A7BB3FBFBFB27
:103A900003E09B4601E0DFF8DCB002F04007BFB274
:103AA0002FB1D6F8D8714FF47A73B7FBF3F7039BB5
:103AB00013B9B6F8CC2100E0002240460392FDF78E
:103AC000E9FFB6F8C611039A01950912204600973E
:103AD0005B4601F0C001FFF761FC0446079008B99E
:103AE000284612E0014653464A460298FFF7D0FCAA
:103AF0000146079008B9204607E01D4BB3F90000C6
:103B000000F087F900282BDC0798FFF7DFFC27E09F
:103B10000BF1380B0FE72B462246394607A8FFF773
:103B2000D9FC00283FF41AAF079B002B7FF415AF98
:103B300028460DE03B46A268594607A8FFF7CAFC95
:103B400000283FF435AF079B002B7FF430AF384699
:103B5000FFF7BCFC4046FDF79DFF01E01B680FE747
:103B60000BB0BDE8F08F00BF90CF000800A493D643
:103B70004010002080EE3600F8B51E469F1C5B7892
:103B80000446154613B96FF01500F8BD01F10800A1
:103B9000FFF75AFC0028F6D17CB394F910300133BA
:103BA00004D1A3681C78022C04D001E06468F3E718
:103BB000082C06D17378012B14D0022BE3D10824F2
:103BC00011E0853D022D1BD884B9727808236FF06F
:103BD000010413FB024402FB036616F8013D2BB9F6
:103BE000013CFAE70224853D022D09D822463946D8
:103BF000069807F0ABF92046F8BD853D022DE4D9C3
:103C00006FF08500F8BD70B51D465B78044616461A
:103C100013B96FF0150070BD01F10800FFF714FC37
:103C20000028F6D1882E27D1A91CA4B194F9103010
:103C3000013304D1A3681C78022C04D001E064682D
:103C4000F3E7082C06D16B78012B0ED0022BE0D1C4
:103C500008240BE054B96C78E408023CE4B20B1978
:103C600013F8013C13B9013CF8E7022422460498FA
:103C700007F06CF9204670BD70BDF8B517460D46CB
:103C8000FEF782FC7C78012C06460FD1862D0FD1E1
:103C900000F5E07521462846FDF7CCFE7B681BBA8F
:103CA000A6F8C8312846FDF7F5FE01E00020F8BD72
:103CB0002046F8BD2DE9F0415378042B86B0074625
:103CC000154671D186294ED102F110084046FFF702
:103CD000C7FB0646002846D13846FEF755FCB0F82B
:103CE000C631DA0703D595F90330002B3BDB41469B
:103CF0003846FEF79FFC044618B1427CAB789A42E6
:103D00002AD06B6843B31022002102A807F01CFAE6
:103D1000EB785B0616D4AA78414602A804F058FB5B
:103D2000EB78AA7803F0C00302A93846FEF74AFCF4
:103D30000446002839D03846FEF726FC012103F05E
:103D4000D3FE09E00821009104AB0022384600F0C0
:103D50007BF80028DFDA28E06B6833B91CB1214614
:103D60003846FEF757FC01261FE01BBA6361AA68BC
:103D7000013312BAA2610CD00E4B69680E481B8841
:103D800009BA41431BB204F1300204F11C0004F0F3
:103D900035FF237C23F07F03DBB22374EA7822F023
:103DA0003F0213432374DEE70026304606B0BDE829
:103DB000F08100BFC402002040420F002DE9F34112
:103DC0000446884617461E4600F0C6FA0546E0B18E
:103DD0004146204600F0AEFA691E0446304600F027
:103DE0004BFD94B1B4F90810ADF802706846019625
:103DF00005F022FF002803DC0021304600F04EFDD4
:103E0000204600F0BDFA0446EBE7284602B0BDE8C4
:103E1000F08107B540F20223019101466846ADF8F2
:103E2000023005F009FF03B05DF804FB07B540F26E
:103E30000123019101466846ADF8023005F0FCFE11
:103E400003B05DF804FB000000B589B006930A9B3F
:103E5000ADF81C304FF401738DF81410ADF8162036
:103E6000ADF80630024605AB03A901A8029305F0A0
:103E700007FFBDF80E2040F205239A4203D0044903
:103E80000320FCF7B1FE049809B05DF804FB00BF05
:103E900025CA000800B589B006930A9BADF81C300E
:103EA00040F203238DF81410ADF81620ADF806305B
:103EB000024605AB03A901A8029305F0E1FEBDF897
:103EC0000E2040F205239A4203D004490320FCF758
:103ED0008BFE049809B05DF804FB00BF25CA0008FA
:103EE0002DE9F04384680746208F638D8FB000F082
:103EF000280EADF818304EF0010E0E4611B96FF0D5
:103F000015005DE091F91030013354D18D682B79A3
:103F10002A7813F0C00F03BF02F108035B1995F86C
:103F200001C0294B18BF4FF0020C12B105F1080176
:103F300007E0420747BF04F12E01082204F12C01DB
:103F4000022294F8360000F1010884F836800490CB
:103F50000DF12008BDF81800ADF80800ADF8040018
:103F6000CDF80CE0CDF800C0404604F08FF8814653
:103F70000028C4D0304607A900F024FA0646E8B16C
:103F8000816881E800032B7913F0C00FBB6815BF6F
:103F90001A69DA680132013214BF1A61DA602368E3
:103FA000079A1B682046984700210446304600F0D7
:103FB00075FC204604E06FF04C0001E06FF06800F3
:103FC0000FB0BDE8F08300BF6ECF00082DE9F043CD
:103FD00087683B685C68002387B01A4619463846F4
:103FE000A047041E15DD002322461946184600F09E
:103FF00063FB054668B13B6881685E6822466B4694
:104000003846B047B0F1000805DC0021284600F032
:1040100045FC002466E03E8F06F00206B6B2002E94
:104020005BD1A86804F0C6F8044608B9014637E039
:104030000146C0EB08083246284600F057FB81468F
:1040400008B90146E2E7866801AA04A9304604F0EF
:1040500027F901AA044602A9304604F0CFF8002C43
:1040600001DA00241BE00028FBDBC1B2E3B204AAA2
:1040700002A800F009F906460028F2D0022C0CD163
:104080009DF81030FF2B08D19DF81130FF2B01BF98
:104090008268137963F07F031371344626B90021D7
:1040A000284600F0FBFB1DE0B3689DF801209A71E3
:1040B0009DF800205A710D4A12885A8097F82830CE
:1040C0002B744946284600F0A9F9002373602B465B
:1040D0005A680AB11346FBE75E604146284600F085
:1040E00073FB2C46204607B0BDE8F083C4020020D5
:1040F000034B0360034B436081600020704700BFA7
:10410000E13E0008CD3F0008F0B5254E84683388B5
:10411000838195B00821054604A805F011FE30887A
:10412000204B6360A56000B200F090F82368204641
:104130009B68984740F2032741F23426684605F011
:10414000FBFDBDF80230BB4213D0B3F5017F08D2AE
:1041500040F202229342F1D12B68019928469847F8
:10416000EAE70AD0B342E9D123682046DB689847E2
:10417000E2E7236801995E6902E0236801991E69FC
:104180000B894A6809782046B04740F2052303901E
:1041900002A96846ADF80A3005F0A0FDCCE700BFE3
:1041A000C4020020A941000813B50346806879B90C
:1041B00041F234230190B0F90C10ADF8023068469A
:1041C00005F018FD002822DC124807F0ABF81EE0CD
:1041D000042919D0072913D0022918D14368984718
:1041E0000446A0B103460C4990F9100040F20122A8
:1041F000FFF7E4FD014650B9204600F04FFB06E012
:104200009A6901329A6102E05A6901325A6102B038
:1042100010BD00BFB0CD00080000FFFF30B585B075
:10422000089C6CB1A5685DB10293074B00930194A3
:104230000823FCF779FD0028D8BF6FF0150001E0D6
:104240006FF0120005B030BD09410008074B10B5F2
:10425000B3F90040A04201D1002010BD14B16FF0AD
:104260000B0010BD1880FEF763F9F5E7FC1800207D
:10427000044BB3F9003013B1038001207047184696
:10428000704700BFFC1800202DE9F041174603F1EC
:1042900008020A440E46002180461D4608464FF09B
:1042A000FF3300F009FA00220446F8B183681E705B
:1042B0005D705A805A719A711A71B8F1000F08D066
:1042C0003EB180680278B24203D14146083006F020
:1042D0003DFE5FB155B1A0684378AB4206D103788B
:1042E00008332A463946184406F030FE2046BDE819
:1042F000F081000008B50C4BB1F9082053F82230CA
:104300001B6A1BB909490320FCF76EFCC3B2042BDE
:104310009FBF074B53F820200A6043F8201094BF3A
:1043200000206FF0150008BD1003002025CA00080A
:1043300000190020C3B2042B09D8064B53F8200003
:1043400020B143688B4203D00068F9E77047002032
:10435000704700BF00190020C3B2042B0BD8074BD5
:1043600053F8203000202BB15A681B688A4208BFDE
:104370000130F8E770470020704700BF00190020A7
:1043800028B14368006810B142689342FAD170477F
:1043900049B190F91030032B03D0042B06D103F060
:1043A00029BE06F081B86FF0150070476FF001006C
:1043B000704728B190F910308B4201D04068F8E77F
:1043C0007047000070B504460E4619B91249032023
:1043D000FCF70AFC10B90020306070BD01460025D2
:1043E000496801350029FBD16FF00103EA0020463E
:1043F00000F062F90028EED08368002BE6D0083385
:10440000A26843F8082CE268646843F8042C083377
:10441000002CF5D1356070BD25CA000810B50446E2
:104420008C42084601D1646808E023465A682AB1E4
:10443000904201D01346F9E742685A60002141607A
:1044400000F02CFA204610BD70B5556804460846A9
:10445000EDB129464B680BB11946FBE71CB91A4967
:104460000320FCF7C1FB0028F9D0002AF7D04368ED
:104470005360844206D023465E6826B1B04219D00C
:104480003346F9E7144653684B60556015E0002C3D
:10449000E5D00029E3D0002AE1D04B6853608C427C
:1044A00006D02346596841B1884205D00B46F9E74A
:1044B000144602E05A60E6E75A600021416000F0CD
:1044C000EDF9204670BD00BF25CA000870B503464F
:1044D0001A4A072B88BF033310688CBF23F00303ED
:1044E0000823002140B34468A34202D90146006872
:1044F000F8E7E41A072C0344114E05D8046809B9FB
:10450000146011E00C600FE0C6F108051D44B5F51C
:10451000C05F02D90021116003E009B9136000E017
:104520000B60026883E81400064A9B1B11889BB24B
:10453000994201D2138070BD70BD00BF18190020D0
:104540001C1900201419002001210148FDF772BA3E
:104550001C310020204A38B5831AB3F5C05F39D228
:104560001E4D2C68002324B1844202D223462468C5
:10457000F9E707298ABF0331082121F0030104600C
:10458000141AC1F5C0522244072A98BF8918416005
:104590000BB9286011E05A6818601A44821A072A79
:1045A0000BD818B90E490320FCF71EFB02684168BE
:1045B0001A60C21A0A445A601846036853B1426826
:1045C00002449A1A072A05D81A6802601A1A5B6808
:1045D0001344436038BD00BF1C1900201819002087
:1045E00025CA00082DE9F843814614200F461646D7
:1045F0009846FFF76BFF0446D8B15EB13046FFF72F
:1046000065FF054638B920461421FFF7A3FF284669
:10461000BDE8F88335460123C4F80490A560E66040
:1046200084F81080236027B132463946284606F0C8
:104630008DFC2046BDE8F883F8B50F4D04460026F2
:10464000CCB1631BB3F5C05F03D30C490320FCF767
:10465000CBFA94E88800012B09D1E168A0682660B4
:10466000FFF778FF14212046FFF774FF01E0013BBC
:1046700023603C46E4E7F8BD1C19002025CA000869
:1046800008B5FFF761FF094A094B136018210022A2
:104690001A705A709A70DA701A7159719A71DA71C7
:1046A0000448BDE80840FDF7F5B900BF181900201F
:1046B0001C1900201C310020B2F5C05FF8B505467A
:1046C0000E4614461F460DD8FFF73EFF22463B46D6
:1046D00031462846FFF786FF04460348FDF7DAF91E
:1046E0002046F8BD0020F8BD1C31002007292DE927
:1046F000F84388BFCF1C0D468CBF27F0030708275F
:1047000004469146FFF720FF2DB124B1E3689D4296
:1047100001D8A3682BB92B48FDF7BCF90020BDE8F0
:10472000F8831420FFF7D2FE06460028F3D0E36892
:104730009D422ED0AF4202D85A1B072A29D82846BC
:10474000FFF7C4FE074610B9142130460BE0E068BD
:10475000401BFFF7BBFE804640B914213046FFF7EF
:10476000F9FE29463846FFF7F5FED4E72A46A16848
:10477000384606F0EBFBE268A168521B294440462C
:1047800006F0E4FBE168A068FFF7E4FEC4F80880E7
:1047900005E0A7689D4214BF7B190023A360E3686E
:1047A00008485B1BE360636873600123B760F560D2
:1047B00086F8109033606660FDF76CF93046BDE80E
:1047C000F88300BF1C310020072970B588BFCE1CBC
:1047D00004468CBF26F0030608260D46FFF7B4FEFC
:1047E0001CB922490320FCF7FFF9E368A06813B95C
:1047F0000028F6D106E00028F3D01D4A821AB2F54F
:10480000C05FEED29D422CD02DB930B11946FFF7D2
:10481000A1FEA56024E09D4202D8991B072917D864
:104820002846FFF753FE064620B91248FDF732F935
:104830000C2070BDA16829B1E268AA4228BF2A46AF
:1048400006F084FBE168A068FFF784FEA66007E03D
:10485000033323F003039E4202D23044FFF77AFE73
:10486000E5600448FDF716F9002070BD25CA000870
:104870001C1900201C31002038B504460D46FFF7F6
:1048800063FE24B123682B4423606468F9E702487F
:10489000BDE83840FDF7FEB81C31002010B50446D5
:1048A000FFF752FE2046FFF7C7FE0248BDE8104062
:1048B000FDF7F0B81C31002038B50446FFF744FE80
:1048C0000CB1E26822B90E48FDF7E4F8002038BDCB
:1048D0002368012B0FD994F91030A1686068FFF7A5
:1048E00081FE054610B12368013B23600448FDF7B3
:1048F000D1F8284638BD0248FDF7CCF8204638BD2F
:104900001C310020F8B50026074604463546002C29
:1049100048D02946E268294806F07AFC94F910103C
:104920004B1C052B31D8DFE803F006030F182028B5
:10493000002123482AE04FF0FF31224806F068FCAE
:10494000A06805F06BFF28E001211F4806F060FC1D
:10495000E168A06803F0BCFE1FE002211B4806F0DE
:1049600057FCA06803F008FE17E00321184806F082
:104970004FFCA06803F076FB0FE00421154806F019
:1049800047FCA06804F0E2F807E0134806F040FC9A
:104990001022E168A06803F03BFEE368646801351B
:1049A0001E44B4E7294632460C4806F031FC214645
:1049B0003846BDE8F840FFF771BF00BFD6CD00080C
:1049C000FBCD00080FCE000823CE00083BCE000828
:1049D0004ECE000863CE000875CE00088BCE0008CE
:1049E00000B595B0082104A805F0AAF96FF0850379
:1049F000039340F20523ADF80A30684605F09CF9B0
:104A0000BDF802306FF400721344032B11D8DFE8B5
:104A100003F002040B0B094800E0094806F082FC91
:104A20000198FFF76FFFE8E702A9684605F056F91D
:104A3000E3E7044806F076FCDFE700BFB8CE0008E5
:104A4000D0CE0008E7CE00081FB50A4CB4F90030FC
:104A500063B9094A0193094B029200930622082385
:104A60004FF4C0610648FCF75FF92080B4F90000FC
:104A700004B010BD203100200ECF0008E14900082D
:104A80002231002007B501A8FFF7F2FBBDF90400B1
:104A900000F006F903B05DF804FB00002DE9F043D7
:104AA000082187B07648774C774F05F049F940F2F6
:104AB0000523ADF81230264602A805F03DF9BDF8F1
:104AC0000A30B3F5017F09D840F20322934280F007
:104AD000CF8040F20122934277D0EDE7B3F5106F1B
:104AE00004D040F60112934264D0E5E7674D05F12A
:104AF000900815F8013CD3B1D5F81730022B0DD929
:104B0000042B05D8D5F813302946986900F084FAAB
:104B1000D5F81730023BC5F8173008E0D5F81390E8
:104B2000681F01F06BF80021484601F0F5F83035B8
:104B3000A845DED16378ABB394F98C30002B20DC30
:104B400096F83730022B18D894F8351051BB94F8EA
:104B50003430032B07D93C2384F8373084F83410E1
:104B600084F835101EE0013394F82920206A84F877
:104B7000343000F051FD032300E0023B84F837306D
:104B800010E0E269002ADBD1218E4FF6FF729142DC
:104B9000D6D1023B5BB2002B84F88C30D0DC394894
:104BA00001F087F8B7F90030394A3A493A4804F039
:104BB00025F881E7039800283FF47EAF4369002B76
:104BC0003FF47AAF03F064FF76E7039D1DB93349E4
:104BD0000320FCF709F802212846FFF7EAFB4FF013
:104BE000FF3180462846FFF7E4FBB8F1000FEED016
:104BF00018B18368B3F9021000E00146A868D8F83C
:104C000008204378032B2ED8DFE803F0020D182389
:104C100093885BBA9BB20093043002F11803083208
:104C200000F03CFA1FE093885BBA9BB2009304301B
:104C300002F11803083200F04DFB14E093885BBAD0
:104C40009BB20093043002F11803083200F04EFECC
:104C500009E093885BBA9BB20093043002F1180319
:104C6000083200F09DFE00212846FFF717FE23E7DB
:104C70006FF0850304A902A8059305F02FF81BE740
:104C800024370020183C00202237002075370020F0
:104C90002802002080841E000438002025CA000855
:104CA0007FB51C4CB4F90050064625BB1A4B1B4877
:104CB0001D701B4B02931B4B00930195082305228B
:104CC0004FF48061FCF730F8208000B316499B2236
:104CD000088103204A60FFF70DFB00F0A9FE134A8C
:104CE00013491448B4F9003003F088FF80222946A4
:104CF000114806F029FA0023802210493046FDF7BA
:104D000061FC00200D4900F087F9B4F9000004B0FF
:104D100070BD00BF22370020003800201838002066
:104D200026CF00089D4A0008643700202802002092
:104D300080841E0004380020A83C002016CF000804
:104D4000012380F82F30002380F82C3080F82D309C
:104D500070473C2380F82F30002380F82C3080F8F7
:104D60002D3070470021FFF799BD10F0800F4BB236
:104D700002D0002B11DA01E0002B10DB884204D2B4
:104D8000C1F1800303440F2B09DD884205D9401A85
:104D90000F28CCBF00200120704700207047012061
:104DA00070470000F8B5074615461E460C4639B94F
:104DB00020461949FDF766FC044608B9384625E047
:104DC00035B916492046FDF797FC05460028F5D071
:104DD000114A2946002E18BF3246384605F0DEFB40
:104DE00006460028EAD000231A4619461846FFF75F
:104DF0004BFA83680A495C8005464660034640F2E8
:104E000002220220FEF7DAFF20B92846BDE8F8406A
:104E1000FFF7A8BFF8BD00BF16CF000870CF00088D
:104E20000000FFFF002370B510220C46194606460D
:104E3000FFF742FC054618B93046FFF793FF24E020
:104E4000836804221A7000210E225A709970A27F82
:104E5000DA70E27F1A7194F820205A71A269B2F8D0
:104E60008A2052BADA80A269B2F8882052BA1A812E
:104E7000A269D2F884201288197352BA5A8194F820
:104E800021205A73628C52BADA81284670BD002301
:104E900070B520220E4619460446FFF70DFC054664
:104EA00018B92046FFF75EFF1EE0806808230370F4
:104EB0001E2343704023C37033695A6942609A6964
:104EC00082605B7C8370002100F1100401734173E8
:104ED0008173C1731022204606F036F933693146DA
:104EE0005A7C204603F074FA284670BD2DE9F34140
:104EF0000F460446002800F0898090F8363003F011
:104F0000020300F1080603F0FF0533B1314600202B
:104F1000FFF7BDFF0546002878D094F83630DB0750
:104F20000CD528463146FFF77DFF054600286DD099
:104F300094F8363023F0010384F836300023182229
:104F400019462846FFF7B8FB804608B9284637E0DF
:104F5000836822781A7094F82E205A7094F83220C0
:104F6000022A04D14FF0FF329A70DA7002E0228EEA
:104F700052BA5A8094F8802094F82F10D20042EA56
:104F8000C11294F825100A431A7194F824205A711A
:104F900000229A71DA713546083304F1180E2A4658
:104FA00003CA724518605960154603F10803F6D12B
:104FB000042301229B21404605F066FA28B94046A9
:104FC00002B0BDE8F041FFF7CDBE03460022D9682C
:104FD0005B680A44002BFAD10E4B17B13978FF29D0
:104FE0000DD1996901319961D9690A44DA61B4F93D
:104FF0002C1000963B460022FFF7D4FE06E019690C
:105000000131196159690A445A61F0E702B0BDE8FB
:10501000F08100BFA83C0020F0B51E4B85B00022F7
:105020000546186803900F460A239B21104605F099
:105030002BFA064658B38068002404714471042298
:1050400003A9063005F082FF32462346D168526834
:105050000B44002AFAD1104A17B13978FF290FD131
:10506000916B01319163D16B0B44D36305B108356A
:10507000002200953B4611463046FFF793FE06E0BE
:10508000116B01311163516B0B445363EEE705B0B3
:10509000F0BD00BF2ACF0008A83C002030B419485A
:1050A000BDF808505BB11978FF2908D0046A0134B3
:1050B0000462446A2C444462052D07D820E0846AC7
:1050C00001348462C46A2C44C462F5E71B780E483C
:1050D000FF2B09D143789BB190F83230022B0FD0CF
:1050E000383030BC03F0E4BC43784BB190F8363034
:1050F00043F0010380F83630114630BCFFF7F6BEAE
:1051000030BC7047A83C0020183C00202DE9F04F2F
:105110008BB00026159F07933E600C46154600F0A5
:10512000CBFE8246002800F0CF80B0464FF47A7B59
:10513000079B434540F2C8802B78082B00F2BD80C6
:10514000DFE803F0050FBBBB147698BB4C003B684F
:1051500008F1010843F001033B601FFA88F80135AC
:10516000E6E73B6843F002033B60A6E03B6843F0A0
:1051700010033B6094F8363043F0010384F8363076
:10518000688940BA80B200F05BFC10B1C4F88400BA
:1051900003E000F055FCC4F88400E87884F82600A9
:1051A00095F804E084F827E0697984F82810EB8802
:1051B0005BBAA4F88A302B895BBAA4F888306B7B81
:1051C00084F82930EA8984F83900012352BA03FAB5
:1051D0000EF36285E36384F838106EE03B68B4F93F
:1051E0002C0043F480733B6094F83630082143F080
:1051F000020384F83630009108AB0022FEF724FE4B
:10520000002802DAEB785B0657D5082208A905F1D9
:10521000100905F1180005F099FE0023AA78B4F9E9
:105220002C004946FDF7CEF9002846D0A06144E0A5
:105230003B68B4F92C1043F020033B6094F829003C
:10524000638DEA7843430BFB03F3002E08BF2E4621
:105250000493802A4FF0010394BF12060022149891
:10526000039310230190009202932A1D184804F022
:1052700086FE22E03B6843F040033B600EB9002607
:105280001BE04FF010096A79638DCDF8009053430D
:105290000BFB03F3029395F902300D48DB43DB0F60
:1052A0000193311D149B102204F0F1FE7378023338
:1052B0001E443378052BE6D0E1E76B78023398443F
:1052C0001FFA88F81D4433E750460BB0BDE8F08F55
:1052D0000C1000202DE9F04786B0174600220392FB
:1052E00004460D46BDF83860A74A5BB11B78FF2B1A
:1052F00008D01368013313605368334453601B2E86
:1053000007D83DE1936801339360D3683344D36099
:10531000F5E71C3E03A92078B6B200F0ABFB0028ED
:1053200000F0898063885BBA9BB24FF6FF729342AC
:1053300000F023812379DDF80C80C3F3C20388F8E1
:105340008030002000F07CFBC8F884004DB928466E
:105350008E49FDF797F9054618B98D490320FBF7EB
:1053600043FC2A46002304F10801039800F0B2FB35
:10537000039D06AA05F10808002342F8083D3946B6
:10538000404600F0E7FB18B9049B002B00F0F580C5
:10539000637885F82E3023790399DB0985F82F305F
:1053A000237903F0070385F825306388049A5BBAF4
:1053B000D38206AB002243F8042D0120019300970D
:1053C000334604F11802FFF7A1FE002800F0D58053
:1053D000059810F0100407D1039800F06AFC3946D4
:1053E0002046FFF719FECBE0AB6943B94146B5F95A
:1053F0002C00FDF781F9002800F0BF80A86140462D
:10540000FFF79EFC634A95F82730B2F9000095F843
:105410002820019295F826200092012202FA03F337
:1054200005F1380140F6011203F058FB049940469B
:1054300000F072FCA4E0039D002D00F0A18005F1B6
:105440000808102204F10801404605F04DFD814690
:10545000002840F09580039A237992F88020C3F3C6
:10546000C2039A4240F08C80627895F82EA01046D4
:105470005146FFF77AFCC8B195F83230012B0FD1B5
:10548000130601D5FF2A00E07F2A1ABF0132D2B2EB
:105490004A4685F82E2005F1380003F009FB0BE0A1
:1054A00085F82E20404600F015FC05E011465046D8
:1054B000FFF75BFC002837D195F83230012B0BD178
:1054C00063885BBA9BB24FF6FF72934205F13800D6
:1054D0002CD003F036FB53E006AA002342F8083D27
:1054E0003946404600F036FB049B08B9002B47D0F4
:1054F0001BB105F1380003F024FB049900293FF4A7
:105500002CAF63885BBACB82404600F005FC049B5D
:105510001A7972B963885BBA9BB24FF6FF729342F5
:105520002ED12A8E9A422BD005F1380003F0C0FA12
:1055300026E0EA69934223D15A7D63799A4202D0E8
:105540004046FFF7FDFB049B62795A752379039966
:10555000DB0985F82F30237903F0070385F8253020
:1055600006AB002243F8042D012001930097334637
:1055700004F11802FFF7CAFD10B9039800F099FB77
:1055800006B0BDE8F08700BFA83C002016CF000899
:1055900025CA000822370020F8B500230C4616461D
:1055A000194614220746FFF787F8054618B938460A
:1055B000FFF7D8FB11E0836805221A7012225A7097
:1055C00000229A70DE702146043304F1100251F873
:1055D000040B43F8040B9142F9D12846F8BDF8B505
:1055E00000230E461546194606220746FFF764F8C3
:1055F000044618B93846FFF7B5FB0AE0836806226F
:105600001A7004225A70ED0100229D70DA701A712E
:105610005E712046F8BD00002DE9F04F8DB00E46BA
:1056200006920546002800F0FD8090F83230012BEC
:1056300000F0F88021B9C669002E00F0F38005362D
:105640000CA805F108030024194640F8044D059301
:1056500009940A94FDF72AF80B9B002B00F0E280D6
:1056600001217248DFF8D8B1FCF7E4F9A0460494B0
:105670000394DBF808309C4268D2DBF8007007EB3B
:105680004417D7E9022313435ED0BB69DA070CD471
:10569000039BD3B9012206991846FFF7A0FF0A9091
:1056A00088B96248FCF7F6F9BCE0049B83B91A4656
:1056B00006991846FFF793FF804609900028F0D01E
:1056C0000123049304E0012303930DF1280901E071
:1056D0000DF124097B699A78FF2A03F1020A07D1A8
:1056E000D87800F00F00A0F10E035842584120E096
:1056F00008224F490793504605F0F6FB079B08B96F
:10570000002016E09A78FF2A04D1DB7803F00F031B
:10571000022BF5D010224749504605F0E5FB002842
:10572000EED010224449504605F0DEFB003018BF91
:10573000012048B1FA7CD9F800005146FFF72CFF50
:10574000C9F800000028ACD0013492E73748FCF7D4
:10575000A1F90A9BB8F1000F02D0C8F8043000E0AC
:10576000099380220B990998FFF716FF04460990C8
:10577000002857D095F90070002F07DA0023102277
:105780000599FEF799FF0A9030B30990DDF824805F
:105790000023042219464046FEF78EFF04460A9075
:1057A00008B9404619E083682A781A70002FB4BF00
:1057B000402200225A705A78099062F07F025A7093
:1057C00095F83320DA7000279F70022204239B2172
:1057D00004F05AFE0A9018B92046FFF7C3FA21E0F8
:1057E000099002463B46D16852680B44002AFAD120
:1057F0003278FF2A114A0ED0116D01311165516DB9
:105800000B445365059BB5F92C10009300223346D9
:10581000FFF7C8FA06E0916D01319165D16D0B4437
:10582000D365EFE70DB0BDE8F08F00BF1810002082
:1058300070CF0008C0CF0008D0CF0008A83C0020DF
:105840000C1000202DE9F7430E469146044600282F
:1058500046D090F90080B8F1000FACBF08231823A0
:1058600003229B21002004F00FFE0546002837D0BC
:10587000876823783B71B8F1000F09DA80237B71C8
:10588000102204F1080107F1080005F05FFB01E0B8
:1058900000237B71002387F80690FB712A46D168AC
:1058A00052680B44002AFAD10F4A16B13178FF2909
:1058B0000FD1916F01319167D16F0B44D367B4F968
:1058C0002C1008340094334600222846FFF76AFA69
:1058D00006E0116F01311167516F0B445367EEE71A
:1058E00003B0BDE8F08300BFA83C00202DE9FF41D4
:1058F00017460546BDF82840284A8BB11B78FF2B78
:105900000ED0136C01331364536C234453646B78CF
:1059100013F0400F0CBF082318239C423AD306E033
:10592000936C01339364D36C2344D364EFE72878FA
:1059300000F0C2F8064668B36B785B0605F1040117
:1059400006F1080801D4083C07E01022404605F0A3
:10595000CBFAF8B905F11401183C96F83220022A66
:10596000A3B217D004AA002042F8040D00970192B8
:1059700002200A463146FFF7C9FB58B195F90130BC
:10598000002B04DAEA7839463046FFF75BFF4046E1
:10599000FFF7D6F904B0BDE8F08100BFA83C0020B5
:1059A00070B5224A0446BDF81000A3B11978FF294A
:1059B00011D0116E01311166516E014451661B7890
:1059C000FF2B32D094F90130002BACBF08231823F1
:1059D00098422AD106E0916E01319166D16E014460
:1059E000D166ECE7207800F067F80546E8B194F955
:1059F0000130002B05F1080602DBE37843B90CE027
:105A00001022211D304605F06FFA0028F5D070BD38
:105A1000A27895F833309A4207D1012385F83530C2
:105A20003046BDE87040FFF794B970BDA83C002037
:105A300008B500F0A5FA014B186008BD283D00200C
:105A4000054B1B680BB900F09BBA1A8882420CBF49
:105A500018460020704700BF283D002090F83220F3
:105A6000022A02D1383003F069B80149FFF73EBA83
:105A700016CF000810B500230E4A0B6054780CB9FD
:105A80000A6004E01478844201D10A600FE00B68D8
:105A90006BB118700B68012058700B6800224FF42E
:105AA0008071A3F88A20A3F88810DA6110BD184627
:105AB00010BD00BF183C0020054A53782BB1137865
:105AC00083420CBF1046002070471846704700BF45
:105AD000183C0020F8B5044608B1407818B91B49B5
:105AE0000320FBF781F80D4604F1080701F1100EC1
:105AF000286869683E4603C6083575453746F7D1BC
:105B00004FF6FF7121861249E164142184F82610B2
:105B1000032184F827100A2184F82810052184F82D
:105B200029103C216185F020002184F8330084F89D
:105B3000321084F8241084F83410246584F8351069
:105B40002462A285A3610120F8BD00BF25CA000818
:105B50005D5A00082DE9F8430026264F166080465E
:105B60000D4614464FF0010917F8013C33B9B9F15D
:105B7000000F14D07A1F2260994610E0D7F8133036
:105B800043450CD12946384602F0E7FB38B11A4AA2
:105B9000302303FB062626600020BDE8F88301368B
:105BA000032E07F13007DFD1206800B3C0F818805A
:105BB000236800221A60D8F8143033B11A680AB189
:105BC0001346FBE722681A6002E02368C8F8143025
:105BD000236801221A7123682946053305F1100252
:105BE00051F8040B43F8040B9142F9D10120BDE8B0
:105BF000F88300BF753700207037002030B50446A9
:105C000087B018B920490320FAF7EEFF85696B6960
:105C100098422AD110221D491D4804F081FA2368B8
:105C2000D3B10020FBF7C8FD22681A4BB0FBF3F09C
:105C3000D369B5F92410181A4FF47A735843053212
:105C400001230393019210230022049000920293F7
:105C50000E4A0F4804F093F96B699C4205D1236802
:105C60006B6108E0944204D013461A68002AF9D107
:105C700001E022681A6030220021204605F064FA13
:105C8000012007B030BD00BF25CA0008C0CF000802
:105C90000C10002040420F0038B50446406920B186
:105CA0000568FFF7ABFF2846F9E74FF6FF7323853A
:105CB00038BD10B504460830FFF7EEFF04F1380098
:105CC00002F03CFF90220021204605F03DFA012021
:105CD00010BD000010B5037F01330377436904460C
:105CE00033B1FFF7D9FF102209490A4804F018FA26
:105CF000228D4FF6FF739A4208D0238504F13000BD
:105D000002F0D6FEA369052283F88C2010BD00BFE7
:105D1000C0CF00080C1000202DE9F04F0A4689B0D2
:105D20000446E1B1438C90F821105943D161416997
:105D30008A4214D1B0F9241090F8210043434FF463
:105D40007A70434305320493012303930192102395
:105D5000002200920293564A564804F010F96369F3
:105D6000228D0692002B00F099804FF0010B00224B
:105D70006669626192469146002E36D00AF1010AA8
:105D8000354600272D6801370DB9D84610E05F452C
:105D9000F8D1FAE7B8F1000F0DD12A46354636683A
:105DA000013FB9F1000F1CD0C9F80050A9461546B3
:105DB000002FEFDC01E02DB9EFE7B8F1000F12DDA5
:105DC0008DB157B1A2690793D2F884202946D268D1
:105DD000304690470028079BDFDD2A6808F1FF382E
:105DE000DFE76561E2E72E46C6E7B9F1000F01D0B3
:105DF000C9F80060BAF1010F4FEA4B0BB7DC6269DA
:105E0000D08A4FF6FF71884248D0934223D0A069D0
:105E100090F88020023A012A06D80022591DFFF787
:105E2000FBFB2046FEF78CFF638C94F82120B4F92D
:105E3000241020485A434FF47A7353436269049301
:105E40000532012303930192102300220092029352
:105E5000174A04F094F8A3696069D3F884300021EC
:105E60005B689847069B2085834203D004F130008D
:105E700002F01EFE606978B1A369228DB3F8881024
:105E8000C38AB2FBF1F2B3FBF1F39A42056801D881
:105E9000FFF7B4FE2846EEE763692BB9204609B048
:105EA000BDE8F04FFFF716BF09B0BDE8F08F00BFA7
:105EB000C0CF00080C10002070B500249C422ED2E8
:105EC0001578082D25D8DFE805F0052424240913CA
:105ED00019240E000134A4B20132EFE7012822D1C7
:105EE00055780E2D14E001281DD155781E2D0FE098
:105EF000022818D15578122D0BD914E0022812D19E
:105F000091F880505678012D14BF04251425AE4217
:105F100009D1557802352C44A4B22A44CEE70CBFEF
:105F20000120002070BD002070BD704711B970B114
:105F3000C18A00E020B183699B69B3F8880001E061
:105F40004FF480700844814201DC80B270474FF604
:105F5000FF707047C28ACB8A9A4203D38CBF01205C
:105F6000002070474FF0FF30704738B50446FFF708
:105F7000F1FF0028CCBF0846204638BD704700001E
:105F800000487047300200200021FEF787BC000067
:105F90002DE9F0419CB000230993A3F580330A93C7
:105FA0007F4B08211B88ADF82C300CA803F0C8FEED
:105FB00009A90120FEF79EF940F20523ADF816303D
:105FC00040F2032440F2012503A803F0B5FEBDF81A
:105FD0000E30B3F5017F09D8A34280F0D880AB42E0
:105FE0000CD040F2022293426ED0EDE740F225221F
:105FF0009342E9D1049800F0EDF9E1E7049D2846C9
:10600000FEF75AFC044600287ED00121FEF7D1F9A4
:10601000054608B1C3681BB92046FFF7B5FFCFE7B7
:1060200083681B78412B11D1FEF746FC05460028FA
:10603000F2D001221146FEF759FB01460028EBD0B1
:106040002046FEF7EBF90223044631E003F0D802C4
:10605000C02A03D1204600F0B1FAB1E703F0E00313
:10606000602BD9D10021022328220846FEF724FB09
:10607000079010B9079890B9CEE702AB00930023C0
:1060800021461A4607A800F0DFFC01460028F1D09F
:1060900001222046FEF72AFB014618B90798FFF7B0
:1060A00073FFB9E72046079AFEF7CEF900230446AE
:1060B0002B7440F2012223463A490220FDF77EFE6E
:1060C00000287FF47DAFA7E7049DEDB1EB68072BB7
:1060D0001AD96B68C3B193F91030022B14D128463A
:1060E000FEF7EAFB044678B18768B7F9020001F0D1
:1060F00095FE61688046002619B1CB6849681E4448
:10610000FAE7B8F1000F01D1284686E798F8043085
:1061100023B1204600F086FF70B97DE701231A46BF
:106120000846FEF7C9FA00283FF476AF636843607B
:106130006060836841221A70626800231AB1D168D6
:1061400052680B44FAE7B8F80210994208D3214686
:10615000B7F90200FDF75DFE00283FF731AF5BE7BE
:10616000114B596800297FF457AFB6F5006FBFF4A3
:1061700053AF79889A8107A840F2252219805C6084
:106180009E60ADF81E20089303F0F8FC18E76FF04E
:10619000850305A903A8069303F0A0FD10E700BF3F
:1061A000C40200200000FFFF2C3D00201FB50A4C58
:1061B000B4F9000000280DDC084B02930023019382
:1061C000074B0093032208234FF480610548FAF738
:1061D000ABFD208004B010BD3C4100202ECF000854
:1061E000915F00083C3D002038B50E4B142404FBA1
:1061F00000340546638A63B10020FBF7DDFA0A4BE1
:10620000B0FBF3F0094B53F82530834206D8002346
:106210006382637C23F01003637438BD1B1A6382AE
:1062200038BD00BF3E41002000879303804200201C
:106230002DE9F041012180461048114DFBF7FAFB92
:10624000002426462746E0B2FFF7CEFF2B7C53B151
:106250004146284602F096F82B7C834203D8B84288
:1062600084BF2E4607460134102C05F11405EAD1EF
:106270000248FBF70FFC3046BDE8F081C042002029
:106280003E4100200F2838B5044615D801210B489F
:10629000FBF7D0FB2046FFF7A7FF094B142000FBBC
:1062A000043506482C7C1CB1FBF7F4FB284638BDAE
:1062B000FBF7F0FB204638BD002038BDC04200206F
:1062C0003E4100202DE9F8430F2806468846154632
:1062D0001F469DF820903FD8002A40D00121214838
:1062E000214CFBF7A7FB002F4FF0140303FB0643E1
:1062F00008BF4FF00009802D88BF80225F828CBFCD
:106300001A741D74B9F1000F02D046F0100300E0BA
:106310003346142000FB064441466374204602F0D5
:106320001CF8014640B91022204604F00DFF227CE3
:106330004146204602F04CF80020FBF73DFA0B4B9B
:10634000B0FBF3F00A4B0744064843F82670FBF70E
:10635000A1FB2046BDE8F8830020BDE8F883104685
:10636000BDE8F883C04200203E410020008793032F
:10637000804200200021FEF791BAF8B50E46017860
:106380004378174601F10802024405460830FDF73C
:106390007BFF0446E0B18368B5F902205A802A7970
:1063A0001A716A795A71AA799A71B7424FF000014D
:1063B0003A464FF0010328BF32460846FEF77CF903
:1063C000054620B92046FFF7D5FF2846F8BD606096
:1063D0002046F8BD2DE9F04F054685B0B0F9000024
:1063E00001F01CFDD5F80480D8F8044083464FF036
:1063F000000A1CB1E36864689A44FAE7BBF1000F35
:1064000005D14046FFF7B6FFC5F804B0D0E0B5F8B7
:106410000C90B9F1000F42D1674FAE683B88D8F8B5
:10642000080001333B80CAEB06039AB2BBF8023086
:10643000043B134403F0F8039B1A1FFA83F909F194
:1064400004025146FFF799FF034600283AD04268FC
:10645000D2F808A076BAAAF800609AF8002062F094
:106460003F028AF800203A8852BAAAF80220D8F8E7
:106470000470002F7CD0FA68B9680093C4EB090659
:10648000964228BF1646201D344432465044A4B2DA
:1064900004F05CFDA145009B6AD97F68E9E7D1451E
:1064A00080F08280BBF80260D8F80800AF68053E33
:1064B00006F0F806C9F10501721D5144FFF75DFFB2
:1064C000034628B96868FFF755FF00236B606FE04B
:1064D00042689268511D009179BA1180117861F07B
:1064E0001F01117034494F440988CAEB070A49BAA1
:1064F0004FEADA0A518082F804A0D8F80470FFB19C
:10650000A1451BD0FA68A11889B2894513D2C4EB02
:1065100009041FFA84F9C9EB0204B442B96800986F
:10652000019328BF34462246494404F00FFDA4B22B
:106530007F68019B05E07F680C46E0E7002400E0EF
:106540003C46A64214D99FB1FA680193C4EB0608F1
:106550009045009BB96828BF9046181944444246AC
:10656000A4B204F0F3FCA642019B01D07F68EAE7E5
:106570001946BBF900000093FDF74BFC0028009B77
:1065800002DC1846FFF7F6FE002C9BD0AB89039582
:106590001C44AC8140F2252302A8ADF80A3003F078
:1065A000EDFAFAF787FB03E04046FFF7E3FE6C6085
:1065B00005B0BDE8F08F00BFC442002010B582686E
:1065C000137803F0F803C02B044606D0E02B0DD15E
:1065D0001379C268DB00053A02E0C2680023043A7E
:1065E00060682146806800F013F82046BDE810403E
:1065F000FFF7C0BE002203682BB119689A80DA80C9
:106600001A600160F7E7436070470021FEF746B962
:106610002DE9F04F8FB081460020924604911F462D
:106620008E68AA4DFBF7C8F8A94A834605F1900881
:106630002C46606858B1A368C3EB0B03934206D99C
:106640000292FFF7E2FF2046FFF7D4FF029A2434BC
:106650004445EED199F800B009F1080307930BF116
:1066600008034B44069399F80130029333885BBAD0
:10667000C3F30A03059373885BBAADF82630002094
:106680009BB20A93FBF798F8002308901C460393EB
:106690006A68A846002A00F02581D26805999142CF
:1066A00023D1EA8B0A998A421FD12A7F93451CD1B4
:1066B0006A7F0299914218D15A4607990B9305F1C6
:1066C0000C0004F011FC0B9B78B9029A069905F1B5
:1066D000140004F009FC0B9B38B97C4C039A24236A
:1066E00003FB0244089BA3604EE014B96A6802B938
:1066F0002C463BB1A9689A68521A76498A4294BFDF
:10670000A8469846039B0133042B039305F1240507
:1067100001D04346BCE784B9B8F1000F03D16E49FC
:106720000320FAF761FAD8F804000028F7D0FFF741
:106730006CFF4046FFF75EFF444600210223059AA6
:106740000846FDF7B9FF6060002800F0DD8083682F
:1067500000210020C3E90001089BA3605A46079965
:1067600004F10C0004F0F2FB029A069904F1140003
:1067700004F0ECFB9DF808306377BDF82630E38326
:10678000002384F81CB0238425680FBB3379412B88
:1067900003D105360AF1FF331FE003F0E003602B5D
:1067A00006F1040618D10EAB204643F8047D50F8DC
:1067B000042F0093D2680499042300F045F90028BF
:1067C0007CD00D9A28320AEB020306441B1A05E01E
:1067D00005365346002201E053463A466068C168D8
:1067E00003EB070E8E456AD81FFA87FE0EF1FF31C4
:1067F000194489B26DB1B5F804804145C0F082807A
:10680000B5F806C0E6457DD8C6456FD161456DD166
:1068100078E01FFA83F80EF1FF314144DFF8C0A0A1
:1068200089B2AC460AEBCC05B5F806B0BBF1000F57
:1068300011D1ADB1E98021682960A5F804E0218C6F
:10684000256080684144174421849A1A31463844AF
:1068500004F07CFB04E00CF1010CBCF1340FE1D13D
:106860006368228CDB689A424ED1637F217F04F1FA
:10687000140204F10C00FDF707FDF8B18368B9F9C3
:1068800002205A8099F804201A7199F806209A710A
:1068900099F805205A710023436063682BB15A6848
:1068A0000AB11346FBE7586000E0606063680B497B
:1068B00040F201220220FDF781FA10B96068FFF76B
:1068C000A4FE2046FFF796FE1EE000BFC84200204F
:1068D000C0C62D00FEFFFF7F25CA00080000FFFF95
:1068E00058430020002C7FF404AF01E7FFF78DFE32
:1068F0002046FFF77FFE3B46524604994846FFF785
:1069000087FE01E02D6875E70FB0BDE8F08F00BF8E
:10691000037823F00F0343EA11130370437803F065
:106920000F0343EA0111417070470000082201493A
:1069300004F00CBB70CF00081022002104F004BC4E
:1069400010B508220949044604F0CEFA48B123786C
:10695000FF2B08D1607800F00F00831E5842584189
:1069600010BD012010BD002010BD00BF70CF000879
:1069700073B51546194A04460E46106851686B46B1
:1069800003C32CB3637CDB0624D4227C802A1DD075
:10699000402A1FD9D208D11F501C2944C2F10F022E
:1069A000304404F0A1FAA8B9237CD9080D44725CE4
:1069B00015F8080C03F0070302A90B44424013F832
:1069C000083C1A420CBF0120002004E0012002E034
:1069D000204600E0002002B070BD00BF32CF0008AA
:1069E0000023042A10B54370037016D0082A02D081
:1069F000022A26D118E00B7883F0020303704B784B
:106A000043708B788370CB78C3700B7903714B79AB
:106A100043718B798371CB7911E00B7883F002039A
:106A200003704B7843700223FF240022C470FE24BD
:106A3000827004714271CA5C82710B445B78C371CD
:106A400010BD184610BD00002DE9F74F1E464B68DB
:106A500000920F46D3F808A0D1F808B0019018B9F9
:106A6000C0490320FAF7C0F8019B1B68002BF7D040
:106A7000DA68272AF4D90BEB06089D6898F90130EB
:106A8000002B2B7803F00F0343F060032B701BF8EF
:106A9000063003F01803ACBF02240324082B27D0D0
:106AA00017D8002B52D118F804102846FFF730FFF2
:106AB00008EB04014B7803F00F026B7813436B7003
:106AC0008978AA78E31C0A43AA7018F803200434D2
:106AD00029E0102B2AD0182B38D100212846FFF7A7
:106AE00017FF6B7823F00F036B700023AB702CE063
:106AF00018F804309B099B0043F060032B706B78FF
:106B000003F00F01697018F8043003F00F0308EB6D
:106B100004020B436B705178AA78A31C0A43AA7035
:106B200018F803200334EB7813430EE018F8041030
:106B30002846621CFFF7ECFE6B7823F00F036B70A6
:106B40000023AB70EB70144600E0EB701BF80630CE
:106B50005B075CBF18F80430AB711BF8063003F01C
:106B6000030358BF0134022B08D0032B08D0012B9C
:106B700007D018F80430EB71013403E0402300E043
:106B8000FF23EB7198F8013003F0400202F0FF0997
:106B900072B118064ABF98F802000020000913F0ED
:106BA000300905D0FFF76EFB8146002800F03182E6
:106BB00098F8013003F07003302B42D00FD8102B1F
:106BC0001CD0202B26D0002B40F08C8008EB040139
:106BD000102205F1080004F0B9F9103482E0502BBE
:106BE0003BD006D8402B7DD105F10800FFF7A4FE6D
:106BF00078E0602B45D0702B62D073E005F108007F
:106C0000FFF794FE082208EB040105F1100004F0E0
:106C10009DF934E005F10800FFF788FE4FF0FF32E0
:106C20000023EA746FF001022A752B746B74AB7445
:106C30006B75022208EB040105F1160004F086F9D9
:106C40003CE0514605F1100011F8082BFFF7C8FE93
:106C500005F10800FFF76AFE44E0B9F1000F3FF4C8
:106C6000FFAE082208EB040105F1100004F06EF9F4
:106C700099F81020494605F1080001F0A9FB0834F5
:106C800030E0B9F1000F3FF4EBAE4FF0FF320023DC
:106C9000EA746FF001022A7508EB040102222B74DA
:106CA0006B74AB746B7505F1160004F04FF999F82D
:106CB0001020494605F1080001F08AFB023411E07A
:106CC000B9F1000F3FF4CCAE514605F1100011F8B8
:106CD000082BFFF785FE99F81020494605F10800BA
:106CE00001F076FB98F8013059070FD51A064ABF14
:106CF00098F80200002000F00F0013F00B0F05D0F1
:106D0000FFF7C0FA8146002800F0838198F801302F
:106D100003F00F030C2B00F27C81DFE813F00D0071
:106D20001600250042007A015100610082000D002A
:106D30009400A600B800C60008EB0401102205F17B
:106D4000180004F003F91034D9E005F11800FFF73A
:106D5000EDFD082208EB040105F1200004F0F6F82F
:106D60003CE000BF25CA000805F11800FFF7DEFD72
:106D70004FF0FF32002385F823206FF0010285F8E1
:106D8000242085F8203085F8213085F8223085F8D8
:106D90002530022208EB040105F1260004F0D6F8A4
:106DA0003DE09AF800109AF801200831514405F1AD
:106DB0002000FFF715FE05F11800FFF7B7FD9EE074
:106DC000082208EB040105F1200004F0BFF899F84F
:106DD0001020494605F1180001F0FAFA08348EE057
:106DE0004FF0FF32002385F823206FF0010285F871
:106DF000242008EB0401022285F8203085F8213098
:106E000085F8223085F8253005F1260004F09EF83B
:106E100099F81020494605F1180001F0D9FA02341A
:106E20006DE09AF800109AF801200831514405F1FC
:106E30002000FFF7D5FD99F81020494605F118000C
:106E400001F0C6FA5BE005F11800FFF775FDFF23BE
:106E50002B7618F804306B76611C0522414405F14D
:106E6000230004F073F8063449E005F11800FFF739
:106E700063FDFF232B7618F804306B76611C032228
:106E8000414405F1250004F061F8043437E005F1D0
:106E90001800FFF751FDFF232B7602236B7618F8BD
:106EA000043085F82730013429E005F1180099F8FD
:106EB00010A0FFF741FD99F81030402B84BF40230C
:106EC00089F81030FF232B7618F804306B7608EB26
:106ED000040349465B78AB7699F81030EB7699F865
:106EE000102005F1580001F073FA211D04224144DD
:106EF00005F1240004F02AF8063489F810A0009B5C
:106F000013B9FB681B1B01E0009B283B5BBAAB80FD
:106F10001BF806305B077ED518F8043003F0F80341
:106F2000F02B78D1019BBD68D3F800A0009BDAF864
:106F30000890344404F1010815F804B04BB90099E5
:106F4000042308220846FDF7B7FB002865D08268B5
:106F500002E009F1280200200BF00303022B14D0F9
:106F6000032B1FD015F808101170012B05EB04033B
:106F70009978517004D0D978917005341B790FE05D
:106F8000DB780434A3F5805318E015F80830A3F536
:106F900080535BBA13802B19043499789170DB7895
:106FA000D3700DE015F808301909A1F5756149BADB
:106FB00003F00F0302341180A3F575635BBA5380AD
:106FC0001BF0040F03D00021FDF768FC25E02B5DCA
:106FD0009371A31C2C446178D17118B1F968083100
:106FE000C91A01E00099283949BA9180112189F81C
:106FF00006109288A9F8042018B1019AC0F804A0DC
:10700000106053B19C1B0C9B0C9A1B6808331360D7
:1070100001E0002003E0204601E00024F3E703B094
:10702000BDE8F08F2DE9F04F4268D0F808909668DF
:10703000D268002189B0824601230846FDF73CFB57
:10704000029038B38568AB4960232B7006F1080BBA
:1070500000236B701022584603F046FF38B15846A3
:10706000FFF7E6F8804610B1437CD90601D44FF013
:107070000008337EFF2B00F0628206F11800FFF754
:10708000D7F80746002800F05A82437CDA0640F120
:10709000568201E0029858E2B8F1000F04D098F847
:1070A00011301B0703D15FB17B7C1C0708D06B78C4
:1070B00063F07F036B700023AB70032401E047464D
:1070C000022431683378727821F4704121F0FF0195
:1070D0001B01A9B943EA121313F0FF0F2B7803D158
:1070E00043F018032B7036E043F010032B707378D5
:1070F00031781B09621C43EA01132B5594B22AE034
:107100005BB203F030011209114304F101010ED109
:107110002B7843F008032B7032688BB2317812BAA7
:107120008910C2F3034242EA81122A5509E013434F
:107130002B55326889B212BAC2F30342A31C6A54B7
:107140009BB2326812BA120AEA549C1C01339BB2F9
:107150000022EA54A4B2B379112B6DD1DAF80430CD
:10716000586883681A88B3F802E052BA92B222F0E3
:107170000F0C1FFA8CFC4FF2B0018C451AD19EFA0D
:107180009EF121F00F010904090C614512D103227F
:10719000B271598849BA1FFA81FE198849BA89B271
:1071A0000EEB011101F5AA61197099795970D9791D
:1071B000997026E09EFA9EFE0EF47F4EBEF5704F4B
:1071C00004D10122B2715A8852BA0CE002F47F4213
:1071D000B2F5704F0ED10222B2711A8852BA1A70EB
:1071E0009A785A70DA789A709A79DA70DA791A712C
:1071F000052206E00022B2719A791A71DA795A7181
:107200000622B17961F00F01C2F1080EB1711A4482
:10721000C168C3EB020CCEEB01018C4504D212F81D
:107220000E1002F8011BF3E7FDF7CEFA2B7843F0BE
:1072300004032B70012303E0621C2B5594B200233E
:107240000393F379402B07D0FF2B0AD0012B0CD1ED
:107250002B7843F0010302E02B7843F002032B70FC
:1072600006E02B7843F00303F9E7621C2B5594B238
:1072700010222049584603F037FE18B96B7843F0C6
:10728000400335E0B8F1000F0CD06B7843F04003B9
:107290006B7098F8112010070AD0AB7843EA0213FC
:1072A000AB7005E05846FFF74BFB002800F040812B
:1072B00008AB0020002163E9040199F80020082AA6
:1072C00000F224814FF48A71D140C90740F11E8138
:1072D00009F108011846FFF783FBDDE90423716912
:1072E0003069994208BF904206D16B7843F0300371
:1072F0006B7021E0C0CF000804AA59464046FFF752
:1073000037FB0028F1D13369B3F17F4F05EB04005F
:107310006B7840F00381B28A52BA92B2B2F57E4FD6
:1073200040F0FC8043F020036B70022206F116014E
:1073300003F00CFE0234A4B2337EFF2B72D16B78C3
:1073400043F008026A70728BCABBF269BABB328C16
:10735000AABB727E022A0FD1326A6AB9B28C5AB9BC
:1073600096F8262042B943F00B036B7096F827205D
:107370002A55631C9CB2B4E0728C8AB996F824201A
:1073800072B943F00A036B70737E2B55601C0322A5
:1073900006F1250115FA80F003F0D8FD04349FE0D2
:1073A00096F82220002A40F0948043F009036B7085
:1073B000737E2B55601C052206F123012CE0B38B54
:1073C000ADF81030F38BADF81230338CADF81430CB
:1073D000738CADF8163004A8FEF72AFF002878D089
:1073E000437CDB0675D5027CF37E9A4271D16B78C3
:1073F00043F004036B70437C13F00F031EBFAA78A5
:107400001343AB70737E2B55631C9BB2B27EEA5460
:10741000A01C042206F1240115FA80F003F096FD69
:1074200006345DE01FB199F801303BB951E006F137
:107430001800FFF785FA0028F5D14AE057B16B78BC
:1074400043F004036B707B7C13F00F031EBFAA781C
:107450001343AB7099F8001099F8012008314944A2
:1074600004A8FFF7BDFADDE90423716A306A994286
:1074700008BF904204D16B7843F003036B7030E097
:1074800004AA06F118013846FFF772FA0028F2D173
:10749000336AB3F17F4F05EB04006B780FD1B28CE8
:1074A00052BA92B2B2F57E4F09D143F002036B702B
:1074B000022206F1260103F049FD023410E043F0F8
:1074C00001036B70082206F1200103F03FFD083430
:1074D00006E02819102206F1180103F037FD1034D8
:1074E000A4B2039B1BB1631CB2792A559CB22146FE
:1074F0000298FDF769F9DAF804105046FCF78EFFA0
:10750000029A43685360426001201EE00821B9F9E5
:10751000020000910022FCF797FCDEE643F0100326
:107520006B70082206F1100103F010FD083402E729
:1075300028191022594603F009FD1034FBE6B8F172
:10754000000F3FF4BCAD0027A9E509B0BDE8F08FFE
:1075500010B508220949044603F0C6FC48B1237857
:10756000FF2B08D1607800F00F00831E584258416D
:1075700010BD012010BD002010BD00BF70CF00085D
:10758000F8B5B0F8C631DB07044603D4154903202B
:10759000F9F72AFB00F5E0760121002504F5EE77E6
:1075A0003046FAF747FA384684F8CB51F9F798FA9B
:1075B0004FF40873A4F8F2310B4B0C49B3F90030C7
:1075C000C4F8F44104F5F872384601F017FB304670
:1075D000FAF760FA2946B4F9C401BDE8F840FCF7AF
:1075E0004DB900BF25CA00084010002080969800C1
:1075F000F8B5B0F8C631DB07044603D424490320AC
:10760000F9F7F2FA00F5E07601213046FAF712FABE
:1076100094F8CB31022B03D8013384F8CB3116E038
:10762000DD1E01F02DF80123AB403B2BB0FBF3F541
:1076300005FB13009EBF94F8CB31013384F8CB31A6
:10764000092804D93C2828BF3C20054600E00A252B
:1076500004F5EE773846F9F743FA4FF40873A4F8C7
:10766000F2310C490C4BC4F8F4416943B3F90030D2
:1076700004F5F872384601F0C1FA3046FAF70AFA12
:10768000B4F9C4010021BDE8F840FCF7F7B800BF29
:1076900025CA000840420F004010002010B50446E3
:1076A000B0F91A00FAF770FFB0F8C631DA0703D460
:1076B00010490320F9F798FA637E1B070BD40020CA
:1076C00003F086F8A8B9B4F91A00FAF75DFFBDE82F
:1076D0001040FFF755BF10220749204603F004FC75
:1076E0000028ECD02146B4F91A00BDE81040FCF7A0
:1076F000C5B810BD25CA0008C0CF00082DE9F04369
:1077000080468DB01846894614461F46FFF720FF75
:107710000546B8B910230693029308AE07AB07904D
:1077200003900093019706AB32460DF116014748CE
:1077300002F014FD002806DB069B102B0CBF35461B
:10774000002500E000253946204602F0F7FF0646F6
:10775000002D74D030B93946BDF9160002F0EEFFA5
:107760000646E0B1B6F91A00FAF70EFF18B1B0F804
:10777000C631DA0706D5737E03F03003302B08BF1D
:107780003D4600E03D4645B93846FFF7E1FE00289A
:1077900051D03D46002D3CD00EB1AF4204D0294619
:1077A000204602F0CBFF06462846FFF7D1FE58B32D
:1077B00026B1737E03F03003202B25D107AE30466F
:1077C000FCF756FD0822074689F80020A918404614
:1077D00003F0BCFB98F8003083F0020388F8003017
:1077E000CCB9BC4215D036F91400FAF7CDFE48B139
:1077F000B0F8C631DB0705D50CAB03EB440434F914
:10780000140C1FE00134ECE7737E03F03002202AF1
:1078100003D1002016E0204614E003F00703032BF9
:1078200003D104213046FBF7C9FF324649464046A2
:1078300002F0D6FF06E0FBF7ADFE0546AAE70028FA
:10784000A2D08FE70DB0BDE8F08300BF0C10002080
:1078500070B50E4618B911490320F9F7C5F900298A
:10786000F9D0B0F91A00FAF78FFE00F5EE7504466C
:107870002846F9F735F94FF40873A4F8F2310849AE
:10788000084BC4F8F44104F5F87271432846B3F983
:107890000030BDE8704001F0B1B900BF25CA000852
:1078A00040420F0040100020F8B507460D4616462E
:1078B00010211A462120FBF73CFD044660B1806888
:1078C00000236DBA0822877043710371C370C580AD
:1078D0003146104403F03AFB2046F8BD2DE9F04F45
:1078E00085B080460E9E7578022D0F4692461C4646
:1078F00040F0B8800823009300226B440321FCF77A
:10790000A3FA0028C0F2AE804046FAF73DFE2146B9
:107910008146404602F012FFBAF1870F04464ED06E
:10792000BAF1880F40F09E80B9F8C631D90740F10E
:107930009980DDE90223D6F80CB0D6F808A05B45A3
:1079400008BF524540F08E80002800F08B80B5784B
:10795000012D2ED00BD3022D40F08480404607F13C
:10796000080102F013FF4846FFF70AFE7AE009F526
:10797000E07901214846FAF75DF8F6883D4B04F1BD
:107980003807384676BAB3F90080B6B2F9F7A8F8E6
:10799000394940F21223013EA4F84E30384643469E
:1079A00004F14C02714301F029F94846FAF772F8E4
:1079B0005BE007F118014046FAF72CFE52E0B9F8F7
:1079C000C6319A074ED0B378002B4BD1083710221E
:1079D0002A49384603F088FA002843D0D4B1637EA0
:1079E0009B060CD5D4F88C20D4F8903052EA0301D1
:1079F00005D0F168B0688B4208BF824234D1B6F836
:107A00000690B9F1000F05D13946404602F0BEFE9E
:107A10004D462AE0F3882BB384B9032300930F9AD1
:107A2000109B3946404602F01BFE0446E8B1324640
:107A300000F18C0352F8080F516803C3637E0E48AF
:107A400023F0300343F030036376F188094B49BAE1
:107A500089B24143B3F9003004F1840204F17000AB
:107A600001F0CCF8002500E00125284605B0BDE86E
:107A7000F08F00BF4010002000879303C0CF0008A4
:107A800013B58A784B78402A01D8022B00E0032BEB
:107A90000ED186280ED1C878CB88C0F300145BBA0B
:107AA00000949BB2083100F00F00FEF70BFC01E0E0
:107AB000002000E0012002B010BD000008B5014622
:107AC000074800F04AFC48B910220649044803F070
:107AD0000BFA0028024818BF002008BD004808BD66
:107AE000F8440020C0CF000838B50446E1B10123B6
:107AF00080221449B0F9C401FAF764FDA0B104F57D
:107B0000E07528460121F9F795FFB4F8C63143F036
:107B10000403A4F8C6314FF4E163A4F8CC3128463D
:107B2000BDE83840F9F7B6BFB4F8C631B4F9C401BE
:107B3000044923F00403A4F8C631BDE83840FAF73D
:107B400069BD00BFA0CF000808B510220449054850
:107B500003F0CAF90028034808BF002008BD00BF91
:107B6000C0CF0008F84400202DE9F0470024054666
:107B700000F116074FF00109A2464FEAD40804F0BD
:107B8000070617F8083009FA06F633420AD0E0B2C1
:107B9000FEF778FB80F810A017F8083023EA0606F5
:107BA00007F808600134102CE7D10026AC695CB1FD
:107BB0002368AB616368A168B3F9C401FAF72AFDD1
:107BC00026606660A660F1E710222146284603F091
:107BD000BBFA2C61BDE8F0872DE9F04F87B003F1C7
:107BE000080A02905046039117461E46FFF766FFAB
:107BF0000446002800F0B480F3885BBA9AB21AB940
:107C000042F210738382ABE0DFF860918382103F11
:107C10004FF00008002F70DD08F11003039AD5180B
:107C2000D35C032B02D0222B4AD05EE00298FAF7F5
:107C3000ABFC6B780190042B42D105F1100B0822AC
:107C40004949584603F050F9002839D02A7CFF2AC8
:107C500004D16A7C02F00F02022A31D0EA78510680
:107C60002ED413062CD46A6852B359460298FAF7F8
:107C700043FDAA7804905946D9F80800059200F00F
:107C800081FB059A824209D8D9F808305B7C9A4278
:107C900004D1D9F80430019A9A4207D0334B98683E
:107CA00020B11022324903F01FF948B92F4B5A680E
:107CB00032B9019A5A60049A9A60A2691A60A36163
:107CC000AB783F2B6B7801D8022B00E0032B0CD153
:107CD000EA7804F11603C2F3C001012002F00702A2
:107CE00000FA02F2585C02435A546B7808EBC3085E
:107CF0001FFA88F8A7EBC3078CE773885BBA9BB2BF
:107D00002361B28852BA43EA02432361DAF80000E1
:107D1000DAF80410234603C356F8100F71680222E4
:107D200003C3002104F1160003F00EFA0023A3613F
:107D3000A58A104B04F11C0630465D43F8F7D0FECF
:107D400040F2232363860C4B6463B3F9003004F1E3
:107D500030022946304607B0BDE8F04F00F04EBF74
:107D600007B0BDE8F08F00BF70CF0008304500209D
:107D7000C0CF000800879303401000202DE9F04198
:107D80008846C108064614460831069A22201F4636
:107D9000FBF7CFFA0546A0B18068002164BA0171F3
:107DA0004171C480867080F80380EA6800F108049D
:107DB000083A204603F0C8F932463946204600F01A
:107DC00007FB2846BDE8F08170B505460E4614460F
:107DD00018211A462320FBF7ACFA80B183686ABAEF
:107DE0002D0C6DBA76BA5A809D80DE8022689A602A
:107DF0006268DA6054F8082F1A6162685A6170BDCF
:107E0000054BB3F90020904204D01AB90122188022
:107E100059801A71704700BF3C450020034BB3F9ED
:107E2000002082420CBF1846002070473C450020CD
:107E30000021FCF733BDF8B5074684890E46154688
:107E400000204DB900230822B96800F05FFA96F9C6
:107E50001030022B25D10DE0BD42F3D0B542F1D058
:107E60002346AA89A96800F051FAEB686D681C44A2
:107E7000A4B2E6E702194FF6EE739A42C4BF01308E
:107E800080B2B1681134204400232022083180B22E
:107E900000F03CFA4FF6FF73984203D0C04380B223
:107EA000F8BD0020F8BD000070B598B00023059320
:107EB000A3F5803306934C4B1B88ADF81C3040F281
:107EC0000523ADF80E3008216FF0850308A8049350
:107ED00001F036FF05A90420FCF70CFA01A801F017
:107EE0002BFFBDF806306FF400721344032BF5D856
:107EF000DFE803F0023B7575029D2846FCF7DCFCC9
:107F0000044608B9284667E00221FCF752FA064603
:107F100018B936490320F8F767FE606830B190F968
:107F20001030042B02D1C368082B06D0042208218C
:107F30002046FCF7DBFB00284DD000238568237426
:107F4000EB885BBA9BB2002B45D022463146FFF747
:107F500072FF4FF6FF7398423DD1698849BA2346B4
:107F600040F2012289B2042031E0029E304696F9A7
:107F70001050FCF7A1FC044608B930462CE04068DC
:107F800026460028C5D090F91030042B07D0FCF706
:107F900093FC0346F8B1706040681E46F1E7FCF7B9
:107FA0008BFCC0B1826870600023C16840680B44DC
:107FB0000028FAD15BBA93806B1C08BF63680C4938
:107FC00008BF93F9105040F2022223462846FBF7DF
:107FD000F5FE002882D12046FFF72AFF7EE703A99D
:107FE00001A801F07BFE79E7C402002025CA000841
:107FF0000000FFFF10B5044668B161B190F9103080
:10800000042B0BD14268FFF716FF50B1A36840BAAA
:10801000D880002010BD6FF00D0010BD6FF04C0037
:1080200010BD6FF0010010BD1FB50A4CB4F900304F
:1080300063B9094A0193094B029200930522082370
:108040004FF480610648F8F76FFE2080B4F9000015
:1080500004B010BD424900203ACF0008A97E0008B4
:108060004245002010B5044601784278054803F0E7
:10807000CFF86188044849BA89B2BDE8104003F0DE
:10808000C7B800BF3ECF00085BCF0008F8B5044674
:108090009DF8245025701E4605F0070310250F4655
:1080A000657006989DF8281015460AB1002F68D013
:1080B00018B1002E69D13046F8BD23B1022B02D091
:1080C0000DB9002873D0A17080B39DF82030E37003
:1080D00002289DF82130237104D0082816D00028EA
:1080E00051D120E002463249304602F0FDFE18B977
:1080F000237823F020032370637843F00803637030
:10810000737863713378A371072040E01C23637098
:10811000221D06F1080313F8011D02F8011F9E42FB
:10812000F9D10D2033E005201DB9F8BD0320002D45
:108130003DD0431C9DF81C2022549DF81D20E25484
:108140000230022D03D0082D0CD0E5B9F8BD6378BC
:1081500063F07F0363707A782254431C3A78E254C8
:108160000230F8BD637863F03F03637007F10803E2
:10817000044413F8012D04F8012BBB42F9D1083057
:10818000F8BD3846F8BD0020F8BD63B90DE075B103
:10819000BDF81C20BDF820309A42CAD1237843F0A4
:1081A00040032370CDE7022B8AD1A1708DE7F8BD83
:1081B0006ECF0008427802F00C03082B07D00C2B7E
:1081C00007D0CBB90178490614D4032302E0072372
:1081D00000E00D2312F0C0020CD00178490658BF10
:1081E0000233802A01D1981C7047C02A04D103F1C0
:1081F00008007047184670470020704770B501B1FD
:108200001AB926490320F8F7EFFC437803F00C0372
:10821000082B07D103785C0617D5C3781370037950
:10822000537012E00C2B07D103785B060FD5C3788F
:108230001370037953700AE013B16FF0150070BD2D
:1082400003785E06F9D4032302E0072300E00D2340
:10825000447814F0C00411D005786D0605D4C65CCE
:1082600016705D1C0233455D5570802C08D1C25CD0
:108270004A70034402205B780B7070BD204670BDCD
:10828000C02CDAD1034401F1080213F8010B02F803
:10829000010D8A42F9D1082070BD00BF25CA00082F
:1082A00008B501B11AB918490320F8F79DFC4378C5
:1082B00003F00C03082B09D1C378137003795370B2
:1082C00043794B7083790B70022008BD0C2B0ED1C3
:1082D000C378137010F8043F537001F1080310F8CD
:1082E000012F03F8012D8B42F9D1082008BD3BB9BD
:1082F000037813F0400F14BF6FF01500002008BD85
:108300006FF0150008BD00BF25CA0008F0B51AB30C
:10831000DC0705D511F8014B013A204492B2013334
:10832000570801EB47054C1C03350234AC4207D01B
:1083300014F803EC14F8026C06EB0E263044F4E754
:108340001A44D30703D511F8173000EB0320030CB0
:1083500080B201D01844FAE7F0BD30B54B684568EB
:1083600004680A689D4208BF944209D1C568CB6879
:1083700084688A689D4206BF94420120002030BD77
:10838000002030BD30B510B3E1B188421CD00138B7
:108390000139002210F8015F11F8014FA54202F1E6
:1083A000080303D1DAB2802AF4D10FE085EA040190
:1083B000D8B20B060AD40132D2B249008242C9B205
:1083C000F7D130BD084630BD802030BD104630BDED
:1083D000802A28BF8022F8B5D50814462A460646CA
:1083E0000F4602F0B3FD63070ED0A4EBC504725D27
:1083F000FF23C4F1080403FA04F422EA04027255CC
:108400007B5D1C4014437455F8BD00002DE9F04716
:1084100007468AB008B90020A8E00029FBD0002058
:108420004FF0FF3406462346054631F810E0BEF112
:10843000000F07D1B3F1FF3F13BF013503B2012590
:108440002DB20BE0B3F1FF3F08D0B4F1FF3F01D0F4
:10845000B54201DD2E461C464FF0FF33013008289F
:10846000E3D1581C04D0601C7DD0B54202DD7AE017
:10847000601C03D0012ED8BF4FF0FF343D480025CB
:108480006B46E8464FF03A09AC4203D183F80090BE
:10849000A5194EE015B183F80090013311F815E0ED
:1084A0001EF0F00F4FEA450C17D04FEA1E1A0EF0DF
:1084B0000F0E10F80AA010F80EE083F801E001EBAF
:1084C0000C0E83F800A09EF801E04FEA1E1E033355
:1084D00010F80EE003F801EC21E0BEF1000F10D01F
:1084E00010F80EA09E460EF802AB01EB0C0A9AF8AB
:1084F00001A04FEA1A1A10F80AA083F801A07346E7
:108500000DE001EB0C0E9EF801E01EF0F00F1FBF16
:108510004FEA1E1E10F80EE083F800E001338C4491
:1085200001359CF801E00EF00F0E10F80EE083F814
:1085300000E0072D03F10103A6DD611C05D03444E2
:10854000082C02BF3A2119700133002103F8011BE6
:10855000C8EB030393423FF65EAF4146384602F054
:10856000E9FE384602E02E461C4683E70AB0BDE825
:10857000F08700BFE0CF000810B5017801F0F003EC
:10858000602B8AB0044603D009091B4802F040FE64
:1085900022786378110149B21B0901F030001943B8
:1085A000C2F381020343C9B2144802F031FE2168CC
:1085B000134809BAC1F3130102F02AFEA188E37936
:1085C000A279104849BA89B202F022FE282204F1A9
:1085D00008016846FFF71AFF01460B4802F018FE33
:1085E000282204F118016846FFF710FF01460748EA
:1085F00002F00EFE0AB010BDF1CF00080ED0000848
:108600003FD0000854D0000881D0000895D0000861
:108610002DE9F8431546814613480F4601F094FEB4
:10862000002D08BF1025002407F1FF38A74218D0FD
:108630000E4801F089FE661C19F8040001F06CFE7A
:10864000B6FBF5F305FB13630BB1A04507D1084852
:1086500002F068FEA04502D0304601F069FE3446C3
:10866000E4E7BDE8F88300BFAED0000814D50008E9
:1086700064CA00080146014800F0A6B94449002038
:10868000124BF0B593E83400D8681E691C6084EA88
:10869000050122F000424A4082EA420280EA50008C
:1086A00050405969D86040F3000782EA802239407F
:1086B0004A4004EB12249A609A693E40604044F3B9
:1086C0000004754014405D606040F0BD44490020E6
:1086D000F8B506460F46044623783D1B412B35442A
:1086E0000ED17B4802F01EFE282D40F2EF80601C68
:1086F000FFF742FF1022A5F1290104F12900E1E072
:1087000013F0C00F06D1734802F00CFE1022294668
:108710002046D7E003F0F802C02A11D16E4802F0DB
:1087200001FE21886D4849BAC1F30A0102F070FDCB
:1087300061886B4849BA89B202F06AFD0434CBE71C
:10874000E02A17D1674802F0EDFD2188634849BA55
:10875000C1F30A0102F05CFD6188614849BA89B23F
:1087600002F056FD2179604802F052FD1022691F87
:10877000601DA7E003F0E003602B40F0A7805B489A
:1087800002F0D0FD237803F01803082B09D002D89B
:1087900063B9574808E0102B05D0182B06D155486F
:1087A00002E0554800E0554802F0BCFD237803F094
:1087B000040303F0FF0213B122B1514800E0514815
:1087C00002F0B0FD237803F00303022B06D0032B45
:1087D00006D0012B14BF4C484C4802E04C4800E046
:1087E0004C4802F09FFD637859060BD54A4802F0C9
:1087F0000FFD637803F03003102B15D00ED8C3B9EA
:10880000464814E0464802F003FD637803F0300365
:10881000102B09D002D863B9424808E0202B05D0BC
:10882000302B06D1404802E0404800E0404802F0CA
:1088300079FD637813F0080F03F004031FD05BB1D8
:108840003C4802F06FFD637803F00303013B022B09
:108850008CBF3948394822E0394802F063FD63781B
:1088600003F00303022B06D0032B06D0012B14BF09
:108870003448354813E0354811E035480FE03BB146
:10888000344802F0C5FC63789A070AD1324806E002
:10889000324802F0BDFC63789B0702D1214802F008
:1088A00041FD94F90130002B08DAA1782C4801F041
:1088B0000F02090902F0ACFC032000E00220291A93
:1088C00010222044BDE8F840FFF7A2BEF8BD00BF6B
:1088D000B7D00008D0D00008EAD0000807D10008BF
:1088E0001BD1000827D1000849D1000857D1000842
:1088F00065D10008C3D100088BD10008AAD10008B7
:10890000F6D10008EBD1000805D2000812D2000809
:108910001AD2000823D200082DD2000853D2000832
:10892000A2D20008C9D200088AD200086CD200087E
:108930007BD20008D9D200080CD300083ED300082F
:108940004BD300087FD300089BD30008B6D30008A0
:10895000D1D30008EBD3000842D3000815D4000897
:1089600040D4000830B5036845688468C168056074
:1089700085EA040223F00043534083EA430381EA7B
:10898000510183EA010242F3000583EA8223C260B7
:108990000169426929402A404C4053404460836049
:1089A00030BD036823F0004363B9436853B983685B
:1089B00043B9C36833B9542149224E234FF0590CAF
:1089C00080E80E107047000038B5036943604369C2
:1089D0008360836901600446C3600F4801256B1EF4
:1089E00003F0030305F0030254F8233054F8221077
:1089F00083EA937300FB035301354B40082D44F881
:108A00002230ECD12046FFF7CCFF2046FFF7AAFF2B
:108A1000013DFAD138BD00BF6589076C2DE9F341EE
:108A2000856804461DB919490320F8F7DDF8427836
:108A300043689340C268C2EB05086A0093424FF056
:108A400000072CBF82608360478038BF5D0886685E
:108A5000FFF716FE711BB0FBF1F202FB110005449B
:108A6000B4F91030E5604FF47A7245446A430193DB
:108A700004F11C030093A262E7623B4604F130005C
:108A800000F0C6F802B0BDE8F08100BF25CA0008BA
:108A900010B5428803789A42044600D313B963693B
:108AA000A06998472046BDE81040FFF7B7BF000017
:108AB000826843689A4210B5044603D806490320E9
:108AC000F8F792F83030F8F70BF86368A3602046A7
:108AD000BDE81040FFF7A2BF25CA0008F8B50C4654
:108AE000174606469DF818109DF81C201D461BB918
:108AF00010490320F8F778F803FA01F00E4B98427A
:108B0000F6D8002363802270656026826170FFF7CB
:108B1000B7FDC5EB8503B0FBF3F202FB1300054480
:108B2000E560A56026822462E7832046BDE8F84020
:108B3000FFF774BF25CA0008FEFFFF7F3030F7F74C
:108B4000CFBF4388013343807047000010B50188D0
:108B50004288044649BA52BA92B289B2064802F033
:108B600057FBA188E288054849BA52BA92B289B245
:108B7000BDE8104002F04CBB56D4000879D4000880
:108B8000F8F788BFB0F9001001F010B838B5044606
:108B90000020F8F711FE05460020F8F70DFE401BF7
:108BA000A042F9D338BD000030B587B004460D4669
:108BB000F7F761FC40B11DB10E490320F8F714F836
:108BC0002046FFF7E3FF13E00B4B00900390029069
:108BD000012168460493CDF814D0F8F72BFF214605
:108BE00001A82A46F7F7AEFF01216846F8F722FFF1
:108BF00007B030BD25CA0008818B000830B4034D92
:108C0000C560026130BC1380F7F77CBF858B00081C
:108C100070B41146039ABDF91050044EC66002614B
:108C200015801A4670BCF7F78DBF00BF858B000812
:108C300010B5084B0446182240F83C3B02F086F978
:108C4000082384F85630002384F8543084F85730D1
:108C500010BD00BFD0D4000837B5044600F03CFB7F
:108C600094F854301BB90321204600F060FA002527
:108C70000821684684F83650258701F051FE9DF89A
:108C80000030019A23F0010343F002038DF8003015
:108C9000009B12BA1BBA204600F000F9BDF8001084
:108CA00049BA204689B200F0E5F82046232100F0B9
:108CB00028F920461A2100F015F92946204600F02F
:108CC0003DF920460122202100F0B8F9204601227A
:108CD0004FF4807100F0B2F92A4620464FF400515B
:108CE00000F0ACF9204601224FF4804100F0A6F9D3
:108CF000204601224FF4805100F0A0F9012384F8AE
:108D00002830802220460C2100F057FA042120460A
:108D100000F065FA042100F0FD02204600F04DFA53
:108D20000321204600F05BFA032100F0F002204608
:108D300000F043FA082220460E2100F03EFA0F21EF
:108D4000204600F04CFA1621204600F0F0F903B05E
:108D500030BD10B590F857300133044680F85730D5
:108D6000204600F094FAA0F11103DBB2012BF7D9F1
:108D7000192818BF84F856001921204600F0D7F9A9
:108D8000022384F8553010BD70B51D4690F855305B
:108D90006E1C1344144680F8553013460A46F1B24F
:108DA00000F02FFA601970BD10B5012300F15502D3
:108DB0000021044600F025FA02221146204600F068
:108DC000FCF963683BB1228F120504D520460321CC
:108DD000BDE81040184710BDF8B50821044600F062
:108DE000A6F915210746204600F0F9F960F07F0248
:108DF000D2B215210646204600F0DFF906212046B2
:108E000000F095F90821204600F0E9F960F07F02B2
:108E1000D2B20821204600F0D0F90121204600F00E
:108E2000DEF903060546F8D532462046152100F046
:108E3000C4F90821204600F07AF93946204600F0AE
:108E400076F9C5F38010F8BD38B50D460221044609
:108E500000F0B3F9162D07D0204600F018FA85422D
:108E6000FAD184F8545038BD204600F010FA1F287B
:108E7000FAD0F6E710B50A0A044601F07F0180F83F
:108E80002D2080F82C10202100F097F994F82C2048
:108E900020462121BDE8104000F08FB92DE9F843AC
:108EA000054616461F4600F12D0800246FF00709FD
:108EB000E2003046394601F0E3FF09FB04F208F80E
:108EC000010F38323046394601F0DAFF04F124014F
:108ED000C2B2C9B22846013400F06FF9082CE7D1BC
:108EE000BDE8F883A1F10B020F2A07D890F83720CC
:108EF0008A4203D080F8371000F00ABA7047002089
:108F0000704737B50D0A4185CAB22221044600F0E8
:108F100054F92A462321204603B0BDE8304000F032
:108F20004CB9000008B5052100F059F9024B00F0DA
:108F30000F0033F9100008BDAED40008113109B29A
:108F40001429A8BF142121EAE171024B5A5C0521C2
:108F500000F033B999D4000808B52C2100F03FF98E
:108F6000C0F3071008BD38B50C462C21054600F0AB
:108F700036F9072C28BF072400F00F0040EA04123E
:108F8000D2B228462C21BDE8384000F016B908B509
:108F90002C2100F024F9C0F3420008BD0529A8BF28
:108FA0000521002938B50C46A8BF0C464FF02C010E
:108FB0000546B8BF072400F012F920F00E0040EA81
:108FC0004402D2B228462C21BDE8384000F0F5B862
:108FD00038B505460C4699B10A782D2100F0EDF818
:108FE0002E21284600F0FBF8637800F0F80203F029
:108FF00007031A4328462E21BDE8384000F0DDB8AB
:1090000038BD08B5092100F0EAF800F00F00400073
:109010005B3840B208BD0029C4BF494249B25B3148
:10902000C1F3430242F0C002092100F0C6B808B5FE
:10903000072100F0D4F85B3840B208BD10B5038FAB
:109040000446B2B30B43B1F5807F03870AD002D840
:10905000202925D010BDB1F5007F0ED0B1F5005FFD
:1090600020D010BD00F12E01FFF7B2FF04212046F1
:10907000FFF794FF53222F2153E02E2100F0AFF889
:1090800040F01002D2B22E21204600F096F81721AF
:10909000204600F0A4F840F00202D2B2172140E0CE
:1090A0002E212BE00E2100F09AF840F00402D2B2FB
:1090B00036E023EA0103B1F5807F03870AD002D8A6
:1090C000202921D010BDB1F5007F09D0B1F5005F96
:1090D00021D010BD4FF0FF31BDE81040FFF75EBF5B
:1090E000172100F07CF8172100F0FD02204600F067
:1090F00064F8238F9B0619D52E21204600F06FF8C7
:1091000000F0EF022E210CE02E2100F068F840F074
:109110001002D2B2F6E70E2100F061F800F0FB0277
:109120000E212046BDE8104000F047B810BD70B5D4
:1091300004460D46204600F0AAF8A0F11103DBB268
:10914000012B0646F6D91F28F4D0032D02D12A465A
:10915000082126E0A84227D0162801D1192D02E0C7
:10916000192807D1162D0AD1092211462046FFF7EA
:109170006BFE04E00F2802D1204600F094F80F2D7A
:109180000DD103212046FFF7D2FF2946204600F0EB
:1091900026F8E06CF8F786FA84F8545004E02A4682
:1091A00029462046FFF750FE304670BD90F840300B
:1091B000416CC06B0022F8F7CBB870B504460D4681
:1091C0001646FFF7F3FF334645F0C002616CE06BD3
:1091D00001F0F7FCE06BBDE87040F8F7F9B838B57E
:1091E00004460D46FFF7E2FF45F080020023616C64
:1091F000E06B01F0E6FC0546E06BF8F7E9F828467D
:1092000038BDF7B504460F4615461E46FFF7CEFF9C
:10921000616CE06B4023012201F0C2FC3B46616CB3
:10922000E06B012201F0BCFC0022E06B0196009291
:109230002B46616CF8F7E8F8E06B03B0BDE8F0404E
:10924000F8F7C6B810B50446FFF7B0FF616CE06BE5
:1092500020230122BDE8104001F0A2BC07B58DE833
:1092600006000023416CC06B0122F8F7CDF803B073
:109270005DF804FB10B50446416CC06B012300226D
:1092800001F08EFCE06BBDE81040F8F7A1B808B51E
:1092900090F854300F2B04D00121FFF7A0FF00F00D
:1092A0001F03184608BD10B50446FFF7F0FF0F284E
:1092B00011D1E06CF8F7FFF900214FF49970FFF736
:1092C00073FC01212046FFF78AFF00F01F000828E9
:1092D00084F85400F5D110BD10B50446006DF8F7C0
:1092E000EAF900213E20FFF75FFC206DF8F7DAF97C
:1092F00000213E20FFF758FC01212046FFF76FFFB9
:1093000000F01F0310F0170F84F85430F4D110BD93
:1093100038B508210446FFF70AFF08210546204614
:10932000FFF75DFF94F8373000F0E00203F01F0311
:1093300020461A430821FFF740FF29462046BDE892
:109340003840FFF7F4BE43680BB10021184770475F
:109350002DE9F0470446884616461F46FFF797FF5B
:109360008146002C00F0D3800F2840F0DF80B8F158
:10937000180F66D02046FFF796FFB8F1270F00F2CE
:109380002B81DFE818F04200290128003300290171
:1093900029013B002901290129012901290129016C
:1093A000290129012901550029018B008F007E0028
:1093B00029018400290129012901930097009B00BC
:1093C0009F002901A300AA002901290129012901DF
:1093D00029014E00BA00022F03D98B490320F7F769
:1093E00003FC31882046FFF745FD94E0082FF4D8B0
:1093F000D6E900232046FFF751FD8CE0022FECD880
:1094000031882046FFF77DFD85E0012FE5D03178DA
:10941000A1F10B030F2B00F2EC802046FFF762FD59
:1094200079E0012FD9D03378002B40F0E2806CE056
:10943000022FD2D8B6F900102046FFF77FFD022593
:10944000D9E0012FC9D83378013B052B63D8DFE879
:1094500003F00507620C1403082102E00F2100E06D
:1094600016212046FFF763FECBE0238F5A0540F11B
:10947000C8802046FFF798FCC3E02046FFF7ECFBCE
:10948000BFE0327820212046FFF7D8FD43E0012FCE
:10949000A3D831782046FFF766FD36E032784FF4E6
:1094A000806116E032784FF4007112E032784FF4A8
:1094B00000510EE032784FF480410AE032784FF4E8
:1094C000006106E032784FF4805102E032784FF4C8
:1094D00080712046FFF7B2FD17E0012F3FF67DAF08
:1094E000238FDB0503D43378052B40F2828096F975
:1094F00000102046FFF752FD07E0012F3FF66DAF49
:1095000096F900102046FFF786FD012573E06FF005
:109510001200BDE8F087B9F10F0F5DD03B4632462F
:1095200041462046BDE8F04701F0BCBAB8F1270F2C
:10953000F4D801A353F828F00B9400081D950008F7
:10954000D7930008ED9300081D9500081D950008AD
:10955000FD9300081D9500081D9500081D95000845
:109560001D9500081D9500081D9500081D95000813
:109570001D9500081D950008319400081D950008F0
:109580009D940008A5940008839400081D95000888
:109590008F9400081D950008439400081D9500084D
:1095A000AD940008B5940008BD940008C594000867
:1095B0001D950008CD940008DB9400081D95000857
:1095C0001D9500081D9500081D9500081D950008B3
:1095D00023940008FB940008B8F1180F9ED06FF098
:1095E00085050F212046FFF7A2FD15F1860F05D155
:1095F00094E76FF01505B9F10F0FF2D02846BDE8DA
:10960000F0870120BDE8F08725CA00082DE9F04168
:109610000446FFF73CFE0F2806464CD00F2120469B
:10962000FFF7DDFD022107462046FFF7D8FD7B0747
:10963000054603D5636801212046984738073AD587
:10964000162E01D0112E05D1238F590433D563680E
:1096500002212CE0192E01D0122E2CD194F8573073
:109660001BB916490320F7F7BFFA013BDBB284F8B8
:10967000573023B994F856102046FFF758FD636819
:10968000CBB1228FD20416D505F0E000202809D0F6
:1096900002D838B1BDE8F081602807D0A02803D0F7
:1096A000BDE8F081042102E0062100E00721204608
:1096B000BDE8F0411847BDE8F08100BF25CA0008A9
:1096C00013B50446416CC06BF7F714FE0121E06C42
:1096D000F7F70AFFE06CF7F7EEFF0121206DF7F7CF
:1096E00003FF206DF7F7DEFF0D4B009401220021F0
:1096F000A06CF7F733FF2046FFF7AEFA1C21204697
:10970000FFF76DFD032807D11C22002104F10C0096
:1097100001F01AFD002001E04FF0FF3002B010BD53
:10972000479300082DE9F34104460F4690461E4634
:10973000FFF788FD01220DF103012046FFF78EFDA2
:109740009DF8035005F07F05023D37B3454505D927
:109750002046FFF78FFD6FF0680521E0236A013393
:109760002362636A2B442A46394620466362FFF728
:1097700075FD022201A92046FFF770FD6EB101229E
:10978000B1182046FFF76AFD2046FFF773FD072159
:109790002046FFF724FD307002E02046FFF76AFD07
:1097A000284602B0BDE8F0812DE9F04106460D469D
:1097B0009046FFF7CEFA00273C46474512D06A682C
:1097C000A31C13447F2B05F1080514D8F36955F841
:1097D000081C2344F36130462346FFF7D5FA0137CE
:1097E0000446EAE7338F5B0502D43046FFF7DCFA24
:1097F0002046BDE8F0816FF08A00BDE8F0810000EE
:1098000008B5FFF744FD0838C0B211289ABF024BD3
:10981000185C022008BD00BFE8D400082DE9F84319
:109820000F46164698460546002800F0B780A1F17D
:109830001103152B4DD8DFE803F01827344C4C4C9E
:109840004C204C383C40444C484C4C4C4C4C4C0B01
:10985000B8F1010F03D857490320F7F7C5F90023E2
:109860007370FFF74CFB307004E0B8F1010FF2D9D0
:10987000662333800220BDE8F883B8F1000FEAD0F8
:10988000FFF7BEFF307009E0038F13F4806F03D041
:1098900001203070BDE8F883002333700120BDE85B
:1098A000F883038F13F4007FF1E7038FC3F3403392
:1098B000F3E7038FC3F38033EFE7038FC3F3C023D2
:1098C000EBE7038FC3F30033E7E7038FC3F3002312
:1098D000E3E74346324601F031F810F1860F0446C3
:1098E00060D12846FFF7D3FC0F28814611D12846C6
:1098F000FFF7D9FC162F1CD004D8012F35D0102F1C
:109900000ED046E0272F28D02F2F36D0202F1DD065
:109910003FE0162F0DD013D8012F26D0102F44D1A1
:10992000B8F1010F97D92846FFF7FCFA02243080DE
:109930002CE0B8F1000F8ED02846FFF70DFB23E096
:10994000272F0AD02F2F18D0202F2ED1B8F1000F9B
:1099500081D02846FFF71BFB16E0B8F1000F3FF45B
:109960007AAF2846FFF74DFB0EE0B8F1000F3FF449
:1099700072AF2846FFF730FA06E0B8F1000F3FF467
:109980006AAF2846FFF753FB30700124B9F10F0F7F
:1099900008D10F212846FFF7CAFB03E06FF0120041
:1099A000BDE8F8832046BDE8F8836FF08500BDE888
:1099B000F88300BF25CA0008F8B505460E46F6F73D
:1099C0004FFD364B364A1B881BB2074652F8232000
:1099D000D2F820E0BEF1000F1AD054699369A34277
:1099E00016D9631C5361D3691C4046B9136933B956
:1099F000631C04D13846F6F73BFD2046F8BD002C29
:109A00000ADB0EEBC40393E8030085E8030004E0DF
:109A10004FF0FF34002EE9D0D560166976B3336875
:109A20001361002C0CDB95695169D369691A8B426B
:109A3000A9BF691C4FF0FF351D4091610EEBC505B4
:109A4000736893E8030085E8030016F8043C052BCF
:109A500009D0002373600A21A6F10800F6F706FC7E
:109A600016F8034C00E00F243846F6F701FD0E2CE3
:109A700002D82046F6F73AFC0120F8BD002C09DA9E
:109A800010460321F6F7F2FB3846F6F7F1FCF6F73D
:109A9000C3FCF1E73846F6F7EBFCEDE7C402002023
:109AA0001003002010B583694469C2691C1BA242DF
:109AB00001DA002010BD5C1C13408461F9D4026AF5
:109AC00003C902EBC30383E80300012010BD0000BB
:109AD0002DE9F8431E46264B53F82150254B1B8891
:109AE0000380074691462DB93046F6F7C1FC4FF08A
:109AF000FF3439E02B79032B28D01F4B0146284631
:109B0000D3F80080FFF7CEFF044638B13046F6F7B1
:109B1000AFFC98F80430052B25D122E0B9F1000FF5
:109B200003D13046F6F7A4FC1EE098F80430C8F8DC
:109B30000C70052B0CBF052104214046F6F796FB5F
:109B4000414605F11000F7F7CFF807E003C8EB68CE
:109B500083E803000A212846F6F788FB3046F6F72B
:109B600087FCF6F759FC01242046BDE8F88300BFC6
:109B700010030020C4020020C802002038B50446AB
:109B8000F6F76EFC074B1B882380074B21460546E2
:109B90001868FFF787FF04462846F6F769FC204659
:109BA00038BD00BFC4020020C802002008B50F4B1A
:109BB00053F82130B3B1212202801A79032A0BD144
:109BC00003C8DA6882E8030018460A21F6F74EFB5C
:109BD000074B0120186008BD01461846BDE8084043
:109BE000FFF760BF4FF0FF3008BD00BF100300203B
:109BF000C002002070B504460D46F6F73CFC28B1C3
:109C000029462046BDE87040FFF7D0BF094B1B88AE
:109C10001BB29D4204D12046BDE87040FFF7AEBFA5
:109C2000F6F71EFC2946034601222046BDE8704097
:109C3000FFF74EBFC402002070B504460D46F6F78C
:109C40001AFC064628B129462046BDE87040FFF7B9
:109C5000ADBF0A4B1B881BB29D4204D12046BDE814
:109C60007040FFF78BBFF6F7FBFB324603462946F1
:109C70002046BDE87040FFF72BBF00BFC4020020A4
:109C80002DE9F041124F3B881BB2934206460C4629
:109C9000154603D10F490320F6F7A6FFF6F7E0FBC0
:109CA0003A880D4B12B2804653F82270052138468F
:109CB000F6F7DCFA96E80300FC60434684E803000C
:109CC000012229462046BDE8F041FFF701BF00BF51
:109CD000C402002025CA00081003002070B5044605
:109CE0000D46F6F7BDFBB4F90020114B53F82240A6
:109CF00006461CB90F490320F6F776FF2379052B9A
:109D000004D0F6F7B5FB4FF0FF3070BD95E80300C7
:109D1000E36883E803000A212046F6F7A7FA64798E
:109D20003046F6F7A5FB2046F6F7E0FA012070BDB5
:109D30001003002025CA00080121FFF73DBE0000E6
:109D400008B5074B4A1E1B681140186203D005492D
:109D50000320F6F749FF59619961DA6108BD00BF38
:109D6000C802002025CA00080121F7F763BE10B51C
:109D70000446406908B100F0A3FFE06908B100F0B3
:109D80009FFF00200022002360612061E061A0614C
:109D90002080C4E9022310BDF6F72CBE2DE9F04F58
:109DA00089B08A4615469B460446FFF7F5FFCDE984
:109DB0000401EB000393079355445346AB4205D08F
:109DC00013F8012B002AF9D0002300E0012300271B
:109DD00002936FF075030193B846B9463E46A268F8
:109DE000974270D222687D0102EB050EDEE9020186
:109DF000002908BFB0F1FF3F23D0DDE904239942D9
:109E000008BF90421DD200220023CEE9022322681F
:109E10002A44166122682A449661226856532268B1
:109E20002A44506920B100F04BFF22682A44566151
:109E300022682A44D06920B100F042FF22682A44F7
:109E4000D661039B98453CD222682A445069002879
:109E500037D007AA514600F069FF38B923681D447E
:109E6000129BCBF800500120186034E0029B13B124
:109E700002282DD1F2E7012814D12268154429695E
:109E800011F07F4F1BD0079AB2EB116F17D3B8F1C7
:109E9000000F01D0904512D20023CBF8005090461D
:109EA00001930AE002280AD1B8F1000F07D1226815
:109EB000CDF804801544CBF800504FF00109039B06
:109EC000079301378BE7129B0198C3F8009002E0DB
:109ED0000128F4D1D1E709B0BDE8F08F38B50546C7
:109EE0000C46FFF759FF4FF47A736B43C01841F1EA
:109EF0000001C4E9000138BD2DE9F04788B0972979
:109F000090461BBF109A0792424605AA8A461CBF7C
:109F1000CDF814808DF81830ADF806100292DF00ED
:109F200000F1120500F1200600F11C046FF0010998
:109F300035F9023FDBB1BAF1970F03D000976A46BB
:109F4000414607E0D8F8183019684B78DB000093D9
:109F50006A460231306800F0E9FE023007D0B5F9F8
:109F6000002003A901A8FFF78BFE4FF00009A542CE
:109F700006F10406DCD1484608B0BDE8F0872DE9BB
:109F8000F04F00F10C0787B0044638469A468B46DE
:109F90009046149EFFF7E8FE01230493B8F1000FEA
:109FA00001D0119B2BB93846F7F774FD6FF00D0007
:109FB0006AE004AB0093524605AB41462046FFF7EA
:109FC000EDFE012802D04FF000091CE01299119813
:109FD000059C00F013FE054610B96FF00B044FE02E
:109FE000E06900F06DFE139BE561721CA36102D075
:109FF00004F1080139E04FF0FF320023C4E90223E5
:10A000003DE009F10109A2689145E6D222684FEAD4
:10A0100049152A44D2E9020150EA0103F1D151461F
:10A020004046039200F0EAFD039A506122682A44F8
:10A03000516971B1109B13612268129911982A44D9
:10A04000039200F0DBFD039A139BD06122682A443F
:10A05000936122682A44D1690029D2D0A2F800B0C5
:10A06000731C216805D0294408313046FFF736FFBC
:10A0700005E00D444FF0FF320023C5E90223002420
:10A080003846F7F707FD204607B0BDE8F08F2DE909
:10A09000F04300F10C0585B0044628461F4688466B
:10A0A00091460E9EFFF760FE01230293B8F1000F68
:10A0B00000D02FB92846F7F7EDFC6FF00D002CE02B
:10A0C00002AB00934A4603AB41462046FFF766FECB
:10A0D000012802D06FF00B041BE038460C99039C5A
:10A0E00000F08CFD07460028F4D0E06900F0E8FDA0
:10A0F0000D9BA361731CE76105D004F10801304694
:10A10000FFF7ECFE04E04FF0FF320023C4E9022326
:10A1100000242846F7F7BEFC204605B0BDE8F083D2
:10A12000F0B500F10C0485B0054620460E461746F2
:10A13000FFF71AFE0123029302AB00933A4603ABEA
:10A1400031462846FFF72AFE012802D10398FFF77F
:10A150000EFE2046F7F79EFC05B0F0BD2DE9F04F4E
:10A1600000F10C0485B0054620469B468946924680
:10A170000F9EFFF7F9FD01230293B9F1000F04D000
:10A18000BBF1000F01D00E9B2BB92046F7F782FCE4
:10A190006FF0150049E016B1BAF1000F05D1204665
:10A1A000F7F778FC6FF00D003FE002AF009703ABCC
:10A1B000109A31462846FFF7F1FD0128804615D94F
:10A1C000119B00933246109B99212846FFF794FE7D
:10A1D00048B901230293009703AB109A31462846F1
:10A1E000FFF7DCFD8046B8F1010F0CD8039B5A46FF
:10A1F0005146D86900F07CFD58B92046F7F74AFC73
:10A200006FF0680011E02046F7F744FC6FF075002E
:10A210000BE0039BB3F90020A9F800200E9A9B697C
:10A2200013602046F7F736FC002005B0BDE8F08F3C
:10A23000F8B50646002546F80C5F04463046FFF7A1
:10A2400093FD04F1120204F11C0304F1300122F821
:10A25000025F43F8045F8B424FF00007F7D1237988
:10A260002761022BA2680BD1236852013946186876
:10A2700000F06AFF23689A685868D200394602E005
:10A2800020685201394600F05FFF00F0B1FD304612
:10A29000BDE8F840F7F7FEBB38B1054B0A0901F0FD
:10A2A0000F019A5C5B5C027043700220704700BF34
:10A2B000FAD4000803461A78591C0AB10B46FAE78B
:10A2C000181A7047F8B505460F4616468C18BC425A
:10A2D00006D0284614F8011DFFF7DEFF0544F6E717
:10A2E0007000F8BD07B502AB042243F8041D1946FF
:10A2F000FFF7E8FF03B05DF804FB38B505460C46F0
:10A300004CB122462946012001F072F8002802DBF8
:10A31000241A0544F4E738BD07B5014601A8FFF744
:10A32000BBFF022101A8FFF7E8FF03B05DF804FBC3
:10A3300007B501466846FFF7D5FF08216846FFF7D5
:10A34000DCFF03B05DF804FB10B50446FFF7B2FF75
:10A3500001462046BDE81040FFF7CFBFF8B50646DE
:10A3600084890F46154600206DB90023B289B16873
:10A37000FDF7CCFF4FF6C57302199A4239680EDD1E
:10A38000013080B20BE0AE42EFD02346AA89A96823
:10A39000FDF7BCFFEB686D681C44A4B2E4E73A34F7
:10A3A000204400232022083180B2FDF7AFFFC043D4
:10A3B00080B2F8BD2DE9F3410C46804603212046CA
:10A3C000F9F7F7FF054618B92E490320F6F70CFCFC
:10A3D0000221F9F7EEFF07460028F5D0EB68032BC2
:10A3E0004CD900F1080122462846AE68FFF7B6FFB7
:10A3F000002843D13378803B082B30D8DFE803F0C6
:10A40000052F2F2F2F0C151E2700AB89B968324658
:10A41000404600F081F822E0EB680093BA683346CA
:10A4200021464046F8F7DCFC19E0EB680093BA6877
:10A43000334621464046F8F755FD10E0EB6800939F
:10A44000BA68334621464046F8F734FB07E0EB682C
:10A450000093BA68334621464046F8F7F7FB317857
:10A46000234640F201220320F9F7A8FC014628B94F
:10A47000204602B0BDE8F041FAF710BA02B0BDE8DC
:10A48000F08100BF25CA000838B50D4614460021EA
:10A490001A460323FAF710F928B1836800221D70C9
:10A4A0005C709A70DA7038BD10B5044668B190F9E6
:10A4B0001030032B0CD142680831FFF74FFF50B129
:10A4C000A36840BA5880002010BD6FF00D0010BD89
:10A4D0006FF04C0010BD6FF0010010BD2DE9F04190
:10A4E000DDF81880154600220E461F46014608F189
:10A4F00008031046FFF7C8FF044650B1806876BADB
:10A500006DBA8680C58027B142463946083000F0D2
:10A510001DFD2046BDE8F081F7B506460C46002A31
:10A5200038D0072B36D99188D088083B40BA49BA31
:10A53000009389B202F1080382B28120FFF7CEFFB7
:10A54000074638B3237EFF2B04F108020CBF00211D
:10A5500004F1180100F022F8054610B9014638460A
:10A5600013E000231A4619461846F9F78DFE836852
:10A5700009495E8004464560034640F202220220FB
:10A58000F9F71CFC014628B9204603B0BDE8F040AD
:10A59000FAF784B903B0F0BD0000FFFFF8B50F462D
:10A5A0001646022328220021FAF786F8054600B352
:10A5B0008468102204F10800394617B100F0C6FC87
:10A5C00001E000F0C1FD04F118001022314616B17F
:10A5D00000F0BCFC04E000F0B7FD012384F8273054
:10A5E000602200232270FF226370A370E370A271C7
:10A5F000E3712846F8BD38B505460C4619B301F19C
:10A600007000F6F76DFA2846F7F7BEFF38B1D0F8BC
:10A6100010329C4203D100F5FC70F6F761FA04F1A8
:10A620001C00F6F75DFA04F13800F6F759FA04F168
:10A630005400F6F755FA10220021204600F084FD60
:10A6400000236383637638BD08B51022034900F008
:10A650004BFCB0FA80F0400908BD00BFC0CF000835
:10A660002DE9F74F904600901E469DF830708946C0
:10A6700009B900205CE0082BFBD80846FFF7E4FF8F
:10A680000028F6D1824604464FF0980B2A4B0BFB6C
:10A690000AF29D18494628460192FDF75EFE019A8E
:10A6A00078B1B8F1000F42D0002E40D0224B02F119
:10A6B000100041463246184400F048FC2E766F7672
:10A6C00035E02846FFF7C0FF10B1002C08BF2C462C
:10A6D0000AF1010ABAF1080FD8D1002CC9D0BDF88F
:10A6E0000030638310224946204600F02FFCB8F169
:10A6F000000F07D036B13246414604F1100000F099
:10A7000025FC2676677607F00707022F04BF032390
:10A7100084F894304FF40973A4F886304FF404732E
:10A72000C4F88840638664632465204600E02846B8
:10A7300003B0BDE8F08F00BF604900202DE9F04173
:10A7400007460E4611B90020BDE8F0810846FFF724
:10A750007BFF0028F7D10C4D0446A846B5F91A3006
:10A7600013B10FB1BB4209D131462846FDF7F5FDC3
:10A7700020B1982000FB0480BDE8F0810134082C52
:10A7800005F19805EAD1DEE76049002010B50446DE
:10A79000FFF7D4FF01462046BDE81040FFF72BBF6E
:10A7A00038B510B100F1980400E0074C074DAC42F9
:10A7B00005D22046FFF748FF18B19834F7E700208C
:10A7C00038BD204638BD00BF60490020204E002023
:10A7D00008B5FFF7E5FF10B1437E1B07F9D508BDAB
:10A7E00010B5144600B119B90B490320F6F7FCF96E
:10A7F0002AB1537E03F00703013B012B01D800204F
:10A8000010BD137E0B70127E04F1100100F09EFB50
:10A81000B4F91A0010BD00BF25CA000810B50446DF
:10A8200086B0B0F90210214800F0F2FC61792048AE
:10A8300000F0EEFCA1791F4800F0EAFC1E4800F091
:10A84000E7FC237963B11A0602D51C4800F0E0FC4E
:10A8500023795B0602D51A4800F0DAFC194800E0BB
:10A86000194800F05FFD237853B104F10802182164
:10A87000684600F0D9FA0146144800F0C9FC02E02D
:10A88000134800F04FFD63785BB122780832224410
:10A890001821684600F0C8FA01460E4800F0B8FCDE
:10A8A00002E00D4800F03EFD06B010BD0AD50008DC
:10A8B00017D5000822D500082BD5000833D500088D
:10A8C0003ED5000864CA000849D500084DD50008E7
:10A8D0005DD500086FD500087FD500087FB50C4610
:10A8E000054600B119B90D490320F6F77DF90A466E
:10A8F00001AE232100F028FC304600F04BF9002384
:10A90000B3FBF4F204FB1232F15CA85C013341406A
:10A910000C2BA954F4D104B070BD00BF25CA0008A7
:10A9200010B50446FFF7DAFF034B1A78511C197073
:10A9300023785340237010BD54020020062938B5F7
:10A9400004460D46104636D006D8032922D029D811
:10A95000B1B3022911D09DE017294AD004D80829A3
:10A9600051D0152932D095E0252948D0292900F069
:10A970008980192940F08E8035E0012B03D84849A1
:10A980000320F6F731F90A4604F12C0100F0DEFA53
:10A99000284638BD072BF2D9082204F12E0100F019
:10A9A000D5FA7AE0022BEAD1228F520701D508228C
:10A9B00004E003806CE0022BE1D1628D028067E04D
:10A9C000022BDCD194F8373013800AE0012BD6D16A
:10A9D000238F13F0200F02D00123037058E00023CF
:10A9E0000370012038BD012BC9D1238F13F0020F52
:10A9F000F1E7012BC3D194F92820027048E0022B23
:10AA0000BDD10322DAE7072BB9D9238F5B074CBFEF
:10AA10002B4602234FF000024CBF04F12E0104F13B
:10AA20002C01042B4270027018D0082B03D0022B8B
:10AA300033D1134619E00A7882F0020202704A7894
:10AA400042708A788270CA78C2700A7902714A7933
:10AA500042718A798271CA79C27119E00B7883F0E8
:10AA6000020303704B7843700223FF240022C4705A
:10AA7000FE24827004714271CA5C827119444B7861
:10AA8000C3710AE0042B7FF47AAF04F10C0111606A
:10AA9000184638BD6FF0850038BD082038BD00BFAE
:10AAA00025CA000870B515461C4619296AD8DFE882
:10AAB00001F00D6919293939496969696969696953
:10AAC000696969696969694E69616958022C03D0CD
:10AAD0002F490320F6F788F81388FF2BF8D880F861
:10AAE00037304DE0022CF3D800F12C060222002171
:10AAF000304600F029FB22462946304600F026FA6F
:10AB0000022070BD082CE3D800F12E060822002197
:10AB1000304600F019FB22462946304600F016FA6E
:10AB2000082070BD022CD3D11388022B06D0082B2D
:10AB30002BD1038F43F00403038721E0038F23F01D
:10AB400004030CE0022CC3D11388438518E012786B
:10AB5000038F12B143F0200301E023F020030387A9
:10AB6000CEE71278038F12B143F00203F7E723F028
:10AB70000203F4E7012CABD192F9003080F82830C1
:10AB8000204670BD6FF0850070BD6FF0690070BD2C
:10AB900025CA00080C22014900F0D8B9107AFF1F1D
:10ABA00010B586B006AC04F8093D012301930DF100
:10ABB000170300932346F6F727FC9DF8170006B00D
:10ABC00010BDF0B585B01F4604AB002403F8012D7D
:10ABD000012205460E4601920094F6F715FC3B460D
:10ABE000224631462846FFF7DBFF05B0F0BD0000E6
:10ABF00001210148F6F71EBF204E00202DE9F04745
:10AC000080460E46FFF7F4FF294C002514F8013C5E
:10AC10009E420AD132464146204600F065F920B9ED
:10AC2000244B122404FB053428E00135282D04F1BF
:10AC30001204EBD1204B1B68272B33D81D4B00256A
:10AC4000122202FB05F91B4F19F803A0BAF1000FFD
:10AC500025D107EB090463789E4207D010225146A4
:10AC6000A01C00F071FA07F809A06670122000FB22
:10AC7000057032464146023000F068F923780F48EB
:10AC80000133DBB2012B08BF0B4A237002BF1368EC
:10AC900001331360F6F7FEFE2046BDE8F08701356C
:10ACA000282DCED10548F6F7F5FE0020BDE8F08747
:10ACB0002A4E0020284E0020244E0020204E002046
:10ACC00010B50446FFF794FF4CB123783BB1013B2C
:10ACD000DBB223701BB9044A1368013B13600348BD
:10ACE000BDE81040F6F7D6BE244E0020204E0020CE
:10ACF00070B5154606460C46FFF77AFF72782B684A
:10AD000093420AD3B11C204600F020F973782B60DF
:10AD10000548F6F7BFFE204670BD2A600248F6F7E8
:10AD2000B9FE002070BD00BF204E00202DE9F0418B
:10AD3000174606468846FFF75BFF72783B68B3EB21
:10AD4000C20F05D1B01C002501244FF0FF3316E0DF
:10AD50002648F6F79FFE6FF00100BDE8F081591C10
:10AD600037D190F800E018F80510714537D02B4620
:10AD7000C4B1BEFA8EF46409A4B101350130954224
:10AD8000EDD33CB100233B601848F6F783FE022068
:10AD9000BDE8F0815D1C05D11448F6F77BFE204626
:10ADA000BDE8F0811E4418F80310B2784A4007212C
:10ADB00042FA01F4E40748B202D40139F8D1084656
:10ADC00000EBC3033B600948F6F764FE0120BDE8D1
:10ADD000F081002CE6D00478B4FA84F4CBE7002CA0
:10ADE000CBD0B1FA81F46409C7E700BF204E002040
:10ADF00070B5FFF7FDFE0A4C002504F5347604F823
:10AE0000025C04F8015C204610220021123400F09C
:10AE10009BF9B442F3D10348BDE87040F6F73ABE5F
:10AE20002A4E0020204E0020F0B503EB43048C4254
:10AE30004FF0000122D8017005465E1E0F464FF00C
:10AE40003A0E994219D014782409092C94BF303451
:10AE5000573494462C709CF8004004F00F04092CE1
:10AE600094BF30345734B1426C700CBF3C467446CA
:10AE7000AC70013201310335E3E7F0BD0846F0BDA7
:10AE8000D0400B1CD1409C46203AD340184352423C
:10AE9000634693401843704770B50F4E0F4D761BB5
:10AEA000B61018BF002405D0013455F8043B98476C
:10AEB000A642F9D10A4E0B4D761BF5F767F9B6108D
:10AEC00018BF002406D0013455F8043B9847A64229
:10AED000F9D170BD70BD00BF38D6000838D6000863
:10AEE00038D6000838D60008032A70B426D940EABC
:10AEF00001039B0711D004780D78AC4222D10244A3
:10AF0000431C05E013F8014B11F8015FAC4219D165
:10AF10009342F7D1002070BC70470C4603461E6870
:10AF20002568AE421846214603F1040304F10404E7
:10AF3000E1D1043A032A18462146F0D8002ADAD192
:10AF40001046E8E7601B70BC704700BF844641EACA
:10AF5000000313F003036DD1403A41D351F8043B91
:10AF600040F8043B51F8043B40F8043B51F8043BE3
:10AF700040F8043B51F8043B40F8043B51F8043BD3
:10AF800040F8043B51F8043B40F8043B51F8043BC3
:10AF900040F8043B51F8043B40F8043B51F8043BB3
:10AFA00040F8043B51F8043B40F8043B51F8043BA3
:10AFB00040F8043B51F8043B40F8043B51F8043B93
:10AFC00040F8043B51F8043B40F8043B51F8043B83
:10AFD00040F8043B51F8043B40F8043B403ABDD2F2
:10AFE000303211D351F8043B40F8043B51F8043B94
:10AFF00040F8043B51F8043B40F8043B51F8043B53
:10B0000040F8043B103AEDD20C3205D351F8043B22
:10B0100040F8043B043AF9D2043208D0D2071CBFEE
:10B0200011F8013B00F8013B01D30B880380604617
:10B03000704700BF082A13D38B078DD010F003038D
:10B040008AD0C3F10403D21ADB071CBF11F8013BFD
:10B0500000F8013B80D331F8023B20F8023B7BE74C
:10B06000043AD9D3013A11F8013B00F8013BF9D277
:10B070000B7803704B7843708B7883706046704711
:10B080008842F0B50DD98B1898420AD28118002A4F
:10B0900051D09A1A13F8014D01F8014D9342F9D19C
:10B0A000F0BD0F2A48D941EA00039B0746D100F1C1
:10B0B000100401F11003154653F8106C44F8106C9D
:10B0C00053F80C6C44F80C6C53F8086C44F8086C9A
:10B0D000103D53F8046C44F8046C0F2D03F1100379
:10B0E00004F11004E8D8A2F1100323F00F0302F0DA
:10B0F0000F0E1033BEF1030F1944034421D91E1F54
:10B100000D467446043C55F8047B46F8047F032C36
:10B11000F8D8AEF1040424F0030404342344214499
:10B1200002F0030262B1013B0A4411F8014B03F83B
:10B13000014F8A42F9D1F0BD0346F3E70346F2E737
:10B14000F0BD7246EEE700BF70B4840746D0541ECF
:10B15000002A41D0CDB2034602E0621EE4B3144699
:10B1600003F8015B9A07F8D1032C2ED9CDB245EA3A
:10B1700005250F2C45EA054519D903F1100226468D
:10B18000103E0F2E42F8105C42F80C5C42F8085C4E
:10B1900042F8045C02F11002F2D8A4F1100222F08D
:10B1A0000F0204F00F041032032C13440DD91E4675
:10B1B0002246043A032A46F8045BFAD8221F22F0FA
:10B1C00003020432134404F003042CB1C9B21C443A
:10B1D00003F8011BA342FBD170BC70471446034621
:10B1E000C2E700BF0EB410B5044683B018B183693E
:10B1F0000BB900F0B7FB06A803460190059AA168B9
:10B20000204600F071FD03B0BDE8104003B0704768
:10B210000FB410B50A4B1C6882B024B1A36913B9EE
:10B22000204600F09FFB05A803460190049AA16800
:10B23000204600F059FD02B0BDE8104004B0704750
:10B24000580200202DE9F0410E46804600283ED0ED
:10B250008369002B39D084682F4B9C4243D02F4BFD
:10B260009C4256D02E4B9C4208BFD8F80C40A38974
:10B270001B073DD52369002B3AD0013EA36816F881
:10B28000015F013BA360B5B1002B04DB23685A1CAE
:10B2900022601D70F2E7A769BB422246294640465C
:10B2A00001DB0A2DF2D100F0AFF80130E6D14FF00A
:10B2B000FF30BDE8F081002B21DB23680A22591CF6
:10B2C00021601A701046BDE8F08100F04BFBD8F801
:10B2D0001830D8F80840002BBED1404600F042FBA1
:10B2E0000D4B9C42BBD1D8F80440A3891B07C1D4A5
:10B2F0002146404600F0EAF80028BED0D7E72246B3
:10B3000040460A2100F080F80130D0D00A20BDE884
:10B31000F081D8F80840AAE7DCD50008BCD50008C1
:10B320009CD50008024B01461868FFF78BBF00BF91
:10B330005802002080EA0102844612F0030F4FD128
:10B3400011F0030F32D14DF8044D11F0040F51F8F4
:10B35000043B0BD0A3F101329A4312F0803F04BFAB
:10B360004CF8043B51F8043B16D100BF51F8044B94
:10B37000A3F101329A4312F0803FA4F101320BD1C4
:10B380004CF8043BA24312F0803F04BF51F8043B49
:10B390004CF8044BEAD023460CF8013B13F0FF0FA6
:10B3A0004FEA3323F8D15DF8044B704711F0010FD9
:10B3B00006D011F8012B0CF8012B002A08BF7047AA
:10B3C00011F0020FBFD031F8022B12F0FF0F16BFA1
:10B3D0002CF8022B8CF8002012F47F4FB3D1704769
:10B3E00011F8012B0CF8012B002AF9D1704700BF8E
:10B3F00010B4044C13460A460146206810BCF4F70A
:10B40000EBBE00BF58020020F8B50E4614460546B4
:10B4100010B18369002B41D0254B9C4243D0254B72
:10B420009C4242D0244B9C4208BFEC68A389A2698D
:10B43000A2601A0721D52369FBB122686169D31A7A
:10B440008B42F7B221DA0133A168501C0139A160A7
:10B450002060167062699A4206D0A389DB0701D585
:10B460000A2F01D03846F8BD2146284600F040F9A1
:10B470000028F7D04FF0FF37F4E72146284600F0C8
:10B4800025F80028F6D12369D7E72146284600F0A1
:10B490002FF90028EED122680123D5E700F062FAE7
:10B4A000034B9C42BBD16C68C0E7AC68BEE700BFF1
:10B4B000DCD50008BCD500089CD50008024B0A4624
:10B4C00001461868FFF7A0BF58020020384B70B53E
:10B4D0001D6806460C4615B1AB69002B42D0354BB2
:10B4E0009C4245D0344B9C4258D0344B9C4208BFC0
:10B4F000EC68B4F90C2093B219070CD52069A8B1F7
:10B5000013F001021ED0636900225B42A361A260B6
:10B51000F0B1002070BDDD0642D558072AD420695D
:10B5200042F00803A3819BB20028E9D103F4207202
:10B53000B2F5007FE4D03046214600F0B1FAA3898D
:10B540002069DDE7990758BF6269A2600028E0D151
:10B55000B4F90C301A06DDD543F04003A3814FF057
:10B56000FF3070BD284600F0FDF9124B9C42B9D166
:10B570006C68BEE7616B51B104F14403994204D099
:10B58000304600F0D1FAB4F90C20002363630023A5
:10B590002069636022F024022060C1E7AC68A8E75C
:10B5A00042F04002092333604FF0FF30A28170BDAA
:10B5B00058020020DCD50008BCD500089CD5000846
:10B5C0008B891A072DE9F0410D46804635D44A682B
:10B5D000002A6BDDEC6A002C47D003F48052002176
:10B5E00092B2D8F80060C8F80010002A62D06A6DE4
:10B5F0005F0705D569686B6B521A0BB12B6CD21AB9
:10B600000023296A4046A047441C39D0AB892A69E7
:10B610002A60DB044FF000026A6045D4696BC8F809
:10B62000006011B305F14403994202D0404600F096
:10B630007BFA00206863BDE8F0810E69AEB10C684A
:10B640000E6098070CBF4B690023A41B8B600AE0B7
:10B6500023463246AF6A296A4046B8470028A4EB21
:10B660000004064404DD002CF2DC0020BDE8F0817B
:10B67000AB8943F04003AB814FF0FF30BDE8F08170
:10B68000D8F800201D2AF3D8184BD34003F001034B
:10B6900083F00101002BEBD0AB892C696960D904E0
:10B6A0002C60BBD5002AB9D16865B7E70A6C002ABF
:10B6B00090DCDAE70123296A4046A047431C024692
:10B6C00002D0AB89EC6A93E7D8F80030002BF8D0B1
:10B6D0001D2B01D0162B02D1C8F80060C5E7AB893D
:10B6E00043F04003AB81BDE8F08100BF0100402082
:10B6F0000B6933B310B5044682B008B18369ABB1AE
:10B70000114B994219D0114B994218D0104B9942C4
:10B7100008BFE168B1F90C3013B9002002B010BDC8
:10B72000204602B0BDE81040FFF74ABF019100F08B
:10B7300019F90199044B9942E5D16168EAE7A168DA
:10B74000E8E70020704700BFDCD50008BCD5000842
:10B750009CD5000820B1054B01461868FFF7C8BF0B
:10B76000034B0449186800F043B900BF5802002099
:10B7700094D50008F1B6000800207047014900F098
:10B7800037B900BFF1B600080020704770B56823D4
:10B790004D1E03FB05F50E4605F1740100F00AFA93
:10B7A000044640B100210C30666005F1680221605A
:10B7B000A060FFF7C9FC204670BD00BF1F4B70B5ED
:10B7C0001D68AB69064613B9284600F039F84835BC
:10B7D0006B68AC68013B05D521E0013B5A1C04F1C4
:10B7E00068041CD0B4F90C20002AF6D100250123EE
:10B7F0004FF6FF72E281A38165662560A5606560F2
:10B8000025616561A5612946082204F15C00FFF706
:10B810009BFC6563A563A564E564204670BD2B6849
:10B820000BB11D46D4E704213046FFF7AFFF286077
:10B8300008B10546CCE70C23336070BD94D50008F1
:10B840003D4B3E491A682DE9F04F90424FF00003FE
:10B850008364C364036508BF012383B008BF8361A9
:10B8600081620746FFF7AAFF78603846FFF7A6FF18
:10B87000B8603846FFF7A2FF7D68F8600024042313
:10B88000AB812C606C60AC606C66EC812C616C618F
:10B89000AC61214605F15C000822FFF755FCBE684B
:10B8A000DFF89CB0DFF89CA0DFF89C90DFF89C806C
:10B8B000C5F824B001230922C5F828A0C5F82C90AA
:10B8C000C5F830802D622146F381B2813460746006
:10B8D000B460746634617461B46106F15C0008227E
:10B8E0000193FFF731FCFD68366212200222C6F890
:10B8F00024B0C6F828A0C6F82C90C6F8308021469F
:10B90000A881EA812C606C60AC606C662C616C6113
:10B91000AC6105F15C000822FFF716FC019B2D626B
:10B92000C5F824B0C5F828A0C5F82C90C5F830801B
:10B93000BB6103B0BDE8F08F94D500087DB7000867
:10B9400041C3000869C30008A5C30008C5C30008B7
:10B95000024B0349186800F04BB800BF94D50008AB
:10B96000F1B60008836903B96AE77047704700BF02
:10B97000704700BF704700BF704700BF024B0349CC
:10B98000186800F00FB800BF5802002089B70008FF
:10B99000024B0349186800F005B800BF58020020A8
:10B9A00079B700082DE9F04110F148071BD088460F
:10B9B00000267D68BC68013D0FD4A389012B05F1E9
:10B9C000FF3506D9B4F90E300133204601D0C04707
:10B9D00006436B1C04F16804EFD13F68002FE8D1E7
:10B9E0003046BDE8F0813E463046BDE8F08100BFFC
:10B9F0002DE9F84310F148071FD0884606464FF05E
:10BA000000097D68BC68013D11D4A389012B05F1B3
:10BA1000FF3508D9B4F90E3001332146304602D043
:10BA2000C04749EA00096B1C04F16804EDD13F6886
:10BA3000002FE6D14846BDE8F883B9464846BDE840
:10BA4000F88300BF70B50C46B1F90E10002990B014
:10BA500015461E4613DB01AAF4F7CCFB00280EDBCB
:10BA6000029A02F47042A2F50052B2FA82F252092E
:10BA70004FF48063002032602B6010B070BDA3894A
:10BA800000221B06326004D5402300202B6010B03A
:10BA900070BD4FF4806300202B6010B070BD00BFFC
:10BAA0008A8992070B4606D501F1470201211A60E7
:10BAB0001A6159617047F0B583B001AB6A460C4614
:10BAC0000546FFF7BFFF00990646284600F072F8CA
:10BAD000B4F90C30D0B1019A124F0099AF6243F023
:10BAE0008003A3812060206161611AB93343A3817F
:10BAF00003B0F0BD2846B4F90E10F4F780FBB4F99A
:10BB00000C300028F2D043F00103EFE79A05EFD4A0
:10BB100004F1470243F002030121A3812260226164
:10BB20006161E5E77DB7000830B481B151F8043CAC
:10BB30000439002BB8BFC9181D4B1A682AB18A42B4
:10BB40000AD908680C18A24225D04A60196030BC96
:10BB500070478B4203D81A465368002BF9D11468FA
:10BB600015198D420CD007D808680C189C4218D0C3
:10BB70004B6030BC516070470C23036030BC704791
:10BB800009680C44111999421460E0D10ACB0C44A5
:10BB900053601460DBE7146852684A602044086010
:10BBA000D4E71C685B684B60204408605160CEE7B6
:10BBB000F850002070B5CD1C25F0030508350C2D7C
:10BBC00038BF0C25002D06463BDBA94239D8274952
:10BBD0000A6852B113685B1B04D436E023685B1B10
:10BBE0001AD522465468002CF8D149681F4C002908
:10BBF00036D029463046F4F7CDFA431C21D0C41C78
:10BC000024F00304A04205D0211A3046F4F7C2FA0A
:10BC1000013016D0256004E00B2B0DD923601C44A5
:10BC2000256004F10B0020F00700231DC31A02D089
:10BC30005A42E25070BD70BD94420ED063685360AA
:10BC4000EFE70C233360002070BD0B2B03D8536843
:10BC500014460B60E5E71446E0E713461446F8E7A0
:10BC60003046F4F797FA6060C3E700BFF850002051
:10BC70009368013B002B10B4936007DBCCB21368D0
:10BC8000581C10601970204610BC70479469A3427C
:10BC900002DBCCB20A2CF2D110BCFFF7B5BB00BF5F
:10BCA00093B1F8B514460F460646D51801E0AC42EC
:10BCB00008D03A4614F8011B3046FFF7D9FF431C61
:10BCC000F5D1F8BD0020F8BD00207047936810B58D
:10BCD000144613B95360184610BD00F077FB0023DB
:10BCE000A360636010BD00BF2DE9F04F9DB0884692
:10BCF00014460393814618B18369002B00F00B8131
:10BD00008B4B984500F00D818A4B984500F00C81D3
:10BD1000894B984508BFD9F80C80B8F80C301D073E
:10BD200040F1EF80D8F81030002B00F0EA8030238B
:10BD30008DF82A302378814DDFF804A200212022DB
:10BD400009918DF82920002B00F08580252B2646AF
:10BD500003D117E0252B00F0868016F8013F002B59
:10BD6000F8D1B6EB040B76D022465B4641464846F6
:10BD7000FFF796FF01306ED0099B32785B44099340
:10BD8000002A68D000234FF0FF31721C0493079300
:10BD900006938DF853301A930591012604E0049917
:10BDA00006FA03F30B4304931446644821780522F2
:10BDB00000F08EFC621C431B0028F0D1049BD806C7
:10BDC00044BF20228DF853201907217844BF2B222D
:10BDD0008DF853202A2968D0A1F13002092A0BD806
:10BDE000079B14F8011F03EB830302EB4303A1F14C
:10BDF0003002092AF5D907932E293FD00322504853
:10BE000000F066FC48B10499CAEB0000402202FA37
:10BE100000F041EA000301340493217849488DF889
:10BE200028100622013400F053FC00285FD0464B56
:10BE3000EBB103AB00934246444B04A94846AFF331
:10BE4000008007467A1C06D0099B3B44099323785F
:10BE5000002B7FF47BAFB8F80C305B0658D4099800
:10BE60001DB0BDE8F08FB6EB040B8BD07CE7039BD5
:10BE7000073323F0070308330393E5E761782A29A2
:10BE80001DD0A1F130020023092A04F10104059319
:10BE9000B4D814F8011F03EB830302EB4303A1F1B1
:10BEA0003002092AF5D90593A8E7039A11680432EC
:10BEB0000029039215DB0791617801349CE7039B0D
:10BEC0001A680592002A03F104030393B8BF4FF0E8
:10BED000FF3204F10203AEBFA178A17805921C469F
:10BEE0008CE7494243F0020307910493E4E703AB74
:10BEF00000934246154B04A9484600F0CDF807468A
:10BF0000A0E741464846FFF7E1FA00283FF40FAFAB
:10BF10004FF0FF30A4E7FFF725FD054B98457FF470
:10BF2000F3AED9F80480F8E6D9F80880F5E600BF4A
:10BF3000DCD50008BCD500089CD50008FCD500085D
:10BF400004D6000808D6000800000000A1BC0008C4
:10BF500010B4044C13460A460146206810BCFFF793
:10BF6000C3BE00BF580200202DE9F0470C469146A1
:10BF70000969A268DDF820808A42B8BF0A46C9F87C
:10BF8000002094F8431006461F4611B10132C9F84B
:10BF90000020236899065DD5D9F800200232C9F83F
:10BFA0000020236813F0060F19461DD1E1688A1A94
:10BFB000002AD8BF194617DD04F1190A002505E04B
:10BFC000E368D9F800209B1AAB420CDD01235246EE
:10BFD00039463046C047013005F10105F0D14FF038
:10BFE000FF30BDE8F087216894F84330003318BF74
:10BFF00001238A060AD5E1185A1C302081F8430033
:10C00000224494F8451082F84310023304F14302AD
:10C0100039463046C0470130E1D0236803F00603BB
:10C02000042B29D0A36822699342C8BF4FF00009AE
:10C030002FDD9B1A99441A34002501E04D4528D084
:10C040000123224639463046C047013005F101053B
:10C05000F4D1C4E713F0060F08D1E168D9F8002045
:10C060008A1A002AD8BF1946A6DCBDE794F84330E7
:10C07000003318BF0123C9E7D9F80000E168A368BD
:10C080002269091A934221EAE179D2DCB9F1000F61
:10C09000D1D10020BDE8F0872DE9F0430C46097EA0
:10C0A00085B06E29064617460C98984604F1430C55
:10C0B0005AD01AD8632900F0128100F2D6800029E4
:10C0C0005CD0582940F0F58084F845102268036858
:10C0D000DFF864E2150603F104011ED4550653BFD0
:10C0E0001B6801601B88016019E0732900F0CF8094
:10C0F0007ED86F2900F0E480702940F0DA80226851
:10C1000042F020022260782384F845300368DFF88B
:10C110002CE2150603F10401E0D51B680160D0078D
:10C1200044BF42F020022260002B40F09080226841
:10C1300022F0200222601021002284F8432060684F
:10C14000A0600028C0F28880226822F004022260E9
:10C15000002B62D1002840F08180654608296AD012
:10C16000C5EB0C0323610CE023681A0640F1D5806F
:10C1700003686269191D01601B681A600023654627
:10C180002361CDF800803B4603AA21463046FFF7E5
:10C19000EBFE013021D02A46236939463046C0479C
:10C1A00001301AD02368039813F0020FE36819D006
:10C1B0001A1A002A16DD04F11909002504E0E368C3
:10C1C00003981A1AAA420DDD01234A463946304621
:10C1D000C047013005F10105F1D14FF0FF3005B046
:10C1E000BDE8F0839842B8BF184605B0BDE8F083BB
:10C1F000752965D078295CD1226884E76168A160DF
:10C200002D200029C3F1000384F8430021DB22F034
:10C210000402DFF824E122600A216546B3FBF1F253
:10C2200001FB123013461EF8002005F8012D002BEB
:10C23000F4D1082994D12368D90791D5626823697C
:10C240009A428DDC302305F8013C013D88E710213E
:10C2500072E7DFF8E4E00A21002BDED19EF800301F
:10C2600084F8423004F1420578E7642901D0692955
:10C270001FD122680368150603F104013AD51B6833
:10C280000160002BBADBDFF8B0E00A2157E7036852
:10C290006268191D01601D680021284600F018FA27
:10C2A000002846D0401B60602061002384F84330A2
:10C2B00067E7012384F84210236104F14205F4E7A3
:10C2C00023681A061ED503681A1D1B680260227EA9
:10C2D000DFF864E06F2A14BF0A2108212CE7036805
:10C2E0001A68191D0123016004F1420584F84220F7
:10C2F0002361DAE7550653BF1B680160B3F90030CC
:10C300000160BEE713F0400F036803F1040215BF9C
:10C3100002601B681B880260D9E713F0400F0368B6
:10C32000626903F1040101601B6814BF1A801A607E
:10C3300024E76068B8E700BF10D6000824D60008DC
:10C3400010B50C46B1F90E10F3F742FF002803DBDD
:10C35000636D0344636510BDA38923F48053A381F7
:10C3600010BD00BF002070472DE9F0411646B1F91D
:10C370000C201F46D3050C46054607D50022022394
:10C38000B1F90E10F3F731FFB4F90C20B4F90E1027
:10C3900022F48052A2813B4632462846BDE8F04155
:10C3A000F3F71ABF10B50C46B1F90E10F3F71DFFE5
:10C3B000A389421C0EBF23F4805343F4805360656D
:10C3C000A38110BDB1F90E10F3F70ABF9368002BDB
:10C3D00076D02DE9F04F8B8985B00C461907019076
:10C3E000164629D522693AB303F002081FFA88F0ED
:10C3F000356800282FD04FF00009B44FC846B24628
:10C40000B84543464A4628BF3B460198B8F1000F5D
:10C4100050D0216AA66AB047002871DDDAF80830EA
:10C420001B1A8144C0EB0808CAF80830002BE7D17A
:10C43000002005B0BDE8F08F21460198FFF746F8CF
:10C44000002840F03A81A389356803F002081FFAFA
:10C4500088F00028CFD113F001095BD14F46029636
:10C460001FB39A05D4F808802CD54745C246C0F0C2
:10C47000A48013F4906F40F0B18020685246494682
:10C48000FEF7FEFDA0682368C8EB00005344A060DF
:10C4900023603846029A93681B1A81443F1A9360BE
:10C4A000002BC5D0A389002FDBD1D5F800906F6891
:10C4B0000835D5E7D5F80090D5F8048008359FE712
:10C4C0000020704720682369984203D861698F4231
:10C4D00080F0B780B84528BFB84642464946FEF7C7
:10C4E000CFFDA3682268C8EB03034244A360226027
:10C4F000002B49D121460198FFF7FAF8002843D0D4
:10C50000B4F90C3043F040034FF0FF30A38105B085
:10C51000BDE8F08F8046029082468146B9F1000F57
:10C520002AD0029B002B4CD0206823696269C84541
:10C53000C34628BFCB4698425F4604D9A36813443C
:10C540009B4500F39080934520DB1346A76A216A40
:10C5500001985246B847071ED2DDB8EB070823D032
:10C56000B368DB1BBA44C7EB0909B360002B3FF487
:10C570005FAFB9F1000FD4D10023D5F800A0D5F8F2
:10C58000049002930835C9E7404683E75A4651466E
:10C59000FEF776FDA2682368CBEB02025B44B8EBA2
:10C5A0000708A2602360DBD121460198FFF7A0F8BD
:10C5B0000028A5D1CDF80880D2E72068B846BA4651
:10C5C0005CE74A460A21504600F082F800286FD006
:10C5D00001300123CAEB00080293A5E762692068D5
:10C5E000216902EB4208C1EB000A08EBD8780AF196
:10C5F00001004FEA680838444045424684BF8046FF
:10C6000042465B0542D511460198FFF7D3FA8346AF
:10C61000002855D052462169FEF798FCA38923F4DF
:10C62000906343F08003A381CAEB08030BEB0A007D
:10C63000C4F81480C4F810B02060A360B846BA46AD
:10C640001CE76FF00043BB4228BF3B464A4693FBC2
:10C65000F1F30198A66A01FB03F3216AB0470028B1
:10C660003FF718AF4CE71A4651460393FEF708FD13
:10C670002268039B01981A4422602146FFF738F88C
:10C68000039B00287FF43CAF1F4666E7019800F04B
:10C690006FF883460028C7D1019D21692846FFF71E
:10C6A00043FAB4F90C300C2223F080032A6029E706
:10C6B000012309F10108029336E74FF0FF30B8E695
:10C6C000019A0C231360B4F90C301BE700FCFF7FC8
:10C6D00001F0FF01102A2BDB10F0070F08D010F833
:10C6E000013B013A8B422DD010F0070F42B3F6D137
:10C6F000F0B441EA012141EA014122F007047FF050
:10C7000000070023F0E80256083C85EA010586EAA6
:10C71000010685FA47F5A3FA87F586FA47F6A5FAE2
:10C7200087F68EB9EED1F0BC01F0FF0102F00702EE
:10C7300032B110F8013B013A83EA010313B1F8D199
:10C740000020704701387047002D06BF354603387A
:10C75000073815F0010F07D1013015F4807F02BFB3
:10C76000013015F4C03F0130F0BC0138704700BF04
:10C77000F9B1F8B506461546B2B10C4600F01CF802
:10C78000854201D82046F8BD29463046FFF712FA07
:10C79000074668B12A462146FEF7D8FB30462146B7
:10C7A000FFF7C2F93846F8BDFFF7BEF92846F8BDD5
:10C7B000F8BD1146FFF7FEB951F8040C0028BEBFC2
:10C7C000091851F8043CC018043870474E4D4920F0
:10C7D00048414E444C4552004D454D204D414E413F
:10C7E00047452048414E444C45520042555320464F
:10C7F00041554C542048414E444C455200555341FC
:10C800004745204641554C542048414E444C4552E2
:10C81000004445425547204D4F4E2048414E444C20
:10C8200045520044554D4D592048414E444C4552C7
:10C83000000A49535220737461636B206F766572EE
:10C84000666C6F77656400537461636B20706F6909
:10C850006E74657220636F727275707465642C20DB
:10C86000726573657420746F20746F70206F66201A
:10C87000737461636B000A436F6E74657874206231
:10C8800065666F726520686172646661756C743A82
:10C890000020202072303A2030782530386C780A19
:10C8A00020202072313A2030782530386C780A20E8
:10C8B000202072323A2030782530386C780A2020D7
:10C8C0002072333A2030782530386C780A002020E6
:10C8D0007231323A2030782530386C780A202020A6
:10C8E0006C723A2030782530386C780A202020701D
:10C8F000633A2030782530386C780A2020707372C3
:10C900003A2030782530386C780A0A004653522F86
:10C910004641523A0020434653523A20307825305F
:10C92000386C780A0020484653523A203078253037
:10C93000386C780A0020444653523A20307825302B
:10C94000386C780A0020414653523A20307825301E
:10C95000386C780A0020424641523A20307825301F
:10C96000386C780A004D4D4641523A2030782530D7
:10C97000386C780A004D697363004558435F52452F
:10C98000543A2030782530386C780A004174746548
:10C990006D7074696E6720746F207265636F6E735B
:10C9A000747275637420737461746520666F72208D
:10C9B000646562756767696E672E2E2E00496E206A
:10C9C0004744423A0A2020736574202470633D3046
:10C9D00078256C780A20206672616D6520300A2007
:10C9E0002062740A000A49535220737461636B20F9
:10C9F0006F766572666C6F7765642062792061740A
:10CA0000206C656173742025642062797465732ECF
:10CA10000A0048415244204641554C542048414E5A
:10CA2000444C4552004641494C45442041535345EE
:10CA30005254494F4E2E0025700A002A2A2A2052AD
:10CA4000494F54206B65726E656C2070616E69632E
:10CA50003A0A25730A0A002A2A2A2068616C74653A
:10CA6000642E0A0A006D61696E28293A20546869AB
:10CA7000732069732052494F5421202856657273E0
:10CA8000696F6E3A20554E4B4E4F574E20286275B7
:10CA9000696C646469723A202F686F6D652F656CEC
:10CAA0006F7065732F50464531352F52494F5429C9
:10CAB000290A0069646C65006D61696E005F510050
:10CAC000E9CB0008F1CB0008FACB000803CC000842
:10CAD00009CC000811CC00081ACC000823CC0008AF
:10CAE0002CCC000834CC00083CCC00087374617472
:10CAF00065006E616D650009706964207C20252DDC
:10CB00003231737C20252D397351207C207072695D
:10CB1000207C20737461636B20202820757365640A
:10CB200029207C2062617365206164647220207C0E
:10CB30002063757272656E7420202020200A00091F
:10CB400020202D207C206973725F737461636B20D9
:10CB500020202020202020202020207C202D20206C
:10CB60002020202020202D207C2020202D207C20F3
:10CB7000253669202825356929207C20253130700B
:10CB8000207C20253130700A000925336869207C1B
:10CB900020252D323073207C20252D387320252E22
:10CBA0003173207C20253369207C2025366920289C
:10CBB00025356929207C2025313070207C202531C5
:10CBC0003070200A007C0053554D00092535732034
:10CBD000252D3231737C253133732536732025366C
:10CBE000692028253569290A0073746F707065649F
:10CBF00000736C656570696E6700626C206D75749A
:10CC0000657800626C20727800626C2073656E64D7
:10CC100000626C207265706C7900626C20616E79C4
:10CC2000666C00626C20616C6C666C00626C206DDE
:10CC3000626F780072756E6E696E670070656E6403
:10CC4000696E6700004400400000020003000240DB
:10CC500002000240070700260048004000000400D0
:10CC6000090C0240080C02400707002707060402CF
:10CC700001070705030200000030014007000240E1
:10CC800006000240050002400400024005000000CA
:10CC90000010000001000000003800400F040240B6
:10CCA0000E0402400D0402400C0402400500000086
:10CCB000004000000000000000000040FFFFFFFFF8
:10CCC00001000000001C0000000C0040FFFFFFFFFF
:10CCD000080000000032000002024572726F7220EC
:10CCE0007768696C6520696E697469616C697A69D5
:10CCF0006E6720454E434F4445522070696E206157
:10CD0000732065787465726E616C20696E746572EB
:10CD1000727570740A00454E434F44455220475087
:10CD2000494F20696E697469616C697A6564207322
:10CD300075636365737366756C790A0073706565F6
:10CD4000643A20256C752072706D0A0001000000A5
:10CD500003000000060C0240050C0240070C0240D4
:10CD60000A0C02405B6175746F5F696E69745F6E77
:10CD7000657469665D206572726F7220696E697490
:10CD800069616C697A696E672061743836726632DF
:10CD9000787820726164696F202325750A006174B8
:10CDA00038367266327878006970763600293A1122
:10CDB000676E72635F6E65746465763A20706F7338
:10CDC0007369626C79206C6F737420696E7465721C
:10CDD000727570742E007E7E20534E49502025328D
:10CDE00069202D2073697A653A2025337520627990
:10CDF00074652C20747970653A20004E455454595E
:10CE000050455F554E44454620282569290A004E65
:10CE10004554545950455F4E45544946202825698C
:10CE2000290A004E4554545950455F5349584C4FB8
:10CE30005750414E20282569290A004E455454591F
:10CE400050455F4950563620282569290A004E452D
:10CE500054545950455F49434D5056362028256952
:10CE6000290A004E4554545950455F5544502028D6
:10CE70002569290A004E4554545950455F554E4B7B
:10CE80004E4F574E20282569290A007E7E20504BA0
:10CE900054202020202D2025326920736E69707364
:10CEA0002C20746F74616C2073697A653A20253385
:10CEB0006920627974650A00504B5444554D503ACC
:10CEC00020646174612072656365697665643A0007
:10CED000504B5444554D503A206461746120746F36
:10CEE0002073656E643A00504B5444554D503A20BF
:10CEF000726563656976656420736F6D65746869D2
:10CF00006E6720756E657870656374656400706B1C
:10CF10007464756D7000FF020000000000000000E6
:10CF200000000000001A52504C0001020000366C54
:10CF30006F00FF7F3F1F0F07030175647000202003
:10CF400020747970653A2025336868752020636FF6
:10CF500064653A2025336868750A00202020636BD9
:10CF600073756D3A20307825303468780A00FFFFF9
:10CF7000FE80000000000000000000000000000033
:10CF8000FF010000000000000000000000000001A0
:10CF9000FF0200000000000000000000000000018F
:10CFA000FF0200000000000000000000000000027E
:10CFB000FF0200000000000000000001FF00000070
:10CFC0000000000000000000000000000000000061
:10CFD0000000000000000000000000000000000150
:10CFE00030313233343536373839616263646566DF
:10CFF00000696C6C6567616C2076657273696F6E31
:10D00000206669656C643A20256868750A00747248
:10D01000616666696320636C6173733A20307825BA
:10D02000303278202845434E3A20307825782C201D
:10D03000445343503A20307825303278290A00662C
:10D040006C6F77206C6162656C3A203078253035E2
:10D050006C780A006C656E6774683A2025687520E4
:10D06000206E657874206865616465723A20257564
:10D070002020686F70206C696D69743A2025750AEC
:10D0800000736F7572636520616464726573733ACF
:10D090002025730A0064657374696E6174696F6E2C
:10D0A00020616464726573733A2025730A0030301E
:10D0B00030303030303000556E636F6D7072657394
:10D0C0007365642049507636207061636B65740027
:10D0D0004E6F742061204C6F5750414E20284E41B6
:10D0E0004C5029206672616D6500467261676D65FE
:10D0F0006E746174696F6E20486561646572202882
:10D1000066697273742900646174616772616D206D
:10D1100073697A653A202568750A007461673A2058
:10D1200030782568750A00467261676D656E7461B6
:10D1300074696F6E2048656164657220287375623A
:10D1400073657175656E7429006F66667365743AF0
:10D1500020307825750A004950484320646973706F
:10D16000617463680054463A2045434E202B2044A6
:10D17000534350202B20466C6F77204C6162656CC6
:10D18000202834206279746573290054463A20457A
:10D19000434E202B20466C6F77204C6162656C20DB
:10D1A0002833206279746573290054463A20454338
:10D1B0004E202B204453435020283120627974653F
:10D1C00073290054463A207472616666696320636D
:10D1D0006C61737320616E6420666C6F77206C6184
:10D1E00062656C20656C69646564004E483A20692C
:10D1F0006E6C696E65004E483A204C4F5750414E58
:10D200005F4E484300484C494D3A20696E6C696E48
:10D210006500484C494D3A203100484C494D3A2070
:10D22000363400484C494D3A20323535005374614C
:10D23000746566756C20736F7572636520616464D4
:10D240007265737320636F6D7072657373696F6E4F
:10D250003A2000756E737065636966696564206164
:10D2600064647265737320283A3A29003634206268
:10D2700069747320696E6C696E650031362062696D
:10D28000747320696E6C696E6500656C69646564B1
:10D290002028757365204C32206164647265737355
:10D2A000290053746174656C65737320736F7572B4
:10D2B0006365206164647265737320636F6D70725F
:10D2C000657373696F6E3A20003132382062697479
:10D2D0007320696E6C696E65005374617465667560
:10D2E0006C2064657374696E61746F6E206D756C0B
:10D2F000746963617374206164647265737320631D
:10D300006F6D7072657373696F6E3A002020202014
:10D3100034382062697473206361727269656420B5
:10D32000696E6C696E652028556E69636173742D32
:10D330005072656669782D626173656429002020EA
:10D34000202072657365727665640053746174653C
:10D350006C6573732064657374696E61746F6E209D
:10D360006D756C7469636173742061646472657354
:10D370007320636F6D7072657373696F6E3A00200E
:10D380002020203132382062697473206361727208
:10D3900069656420696E6C696E6500202020203408
:10D3A00038206269747320636172726965642069F0
:10D3B0006E6C696E65002020202033322062697413
:10D3C00073206361727269656420696E6C696E6551
:10D3D00000202020203820626974732063617272FB
:10D3E00069656420696E6C696E650053746174656B
:10D3F00066756C2064657374696E61746F6E20610C
:10D4000064647265737320636F6D707265737369A2
:10D410006F6E3A200053746174656C657373206499
:10D42000657374696E61746F6E2061646472657394
:10D430007320636F6D7072657373696F6E3A20004D
:10D440005343493A20307825782C204443493A20E8
:10D45000307825780A002020207372632D706F7257
:10D46000743A202535687520206473742D706F72AE
:10D47000743A20253568750A002020206C656E6797
:10D4800074683A202568752020636B73756D3A20A7
:10D49000307825303468780A000F0F0F0E0E0E0E0C
:10D4A0000D0D0C0C0B0B0A09080706050300030001
:10D4B000030002000200010001000000FFFFFEFF68
:10D4C000FDFFFCFFFBFFF9FFF7FFF4FFEFFF00009C
:10D4D000A997000825970008C19600080D96000836
:10D4E0001D98000851930008060202020202020180
:10D4F00002030402020202020204303132333435E4
:10D500003637383941424344454669665F7069643D
:10D510003A202575202000727373693A2025752002
:10D5200020006C71693A2025750A00666C6167738A
:10D530003A200042524F41444341535420004D553C
:10D540004C54494341535420003078300073726387
:10D550005F6C32616464723A2025730A00737263EF
:10D560005F6C32616464723A20286E696C290064D1
:10D5700073745F6C32616464723A2025730A0064CC
:10D5800073745F6C32616464723A20286E696C292E
:10D59000000000005C0200204300000000000000CA
:10D5A000000000000000000000000000000000007B
:10D5B000000000000000000000000000000000006B
:10D5C000000000000000000000000000000000005B
:10D5D000000000000000000000000000000000004B
:10D5E000000000000000000000000000000000003B
:10D5F000000000000000000000000000232D302B80
:10D6000020000000686C4C006566674546470000D6
:10D610003031323334353637383941424344454668
:10D62000000000003031323334353637383961622A
:08D63000636465660000000060
:10D638000451002000000000980300204000000072
:10D648000000000000000000B3CA0008B8CA0008C3
:10D6580001010101140000000000000900000000A1
:10D66800000000002D5F00086B5F0008555F000890
:10D678007D5F00082B5F000800000000000000002C
:10D6880000000000010000005C0200200000000013
:10D69800DCD50008BCD500089CD5000800000000B7
:10D6A80000000000000000000000000098D50008FD
:10D6B8000000000000000000000000000000000062
:10D6C8000000000000000000000000000000000052
:10D6D8000000000000000000000000000000000042
:10D6E80000000000000000000000000028210000E9
:0400000508000529C1
:00000001FF
